:020000040800F2
:2000000000000120057C00080D7A0008117A0008197A0008217A0008257A0008000000002F
:200020000000000000000000000000002D7A0008317A000800000000357A0008397A0008EC
:20004000557C0008557C0008557C0008557C0008557C0008497A0008557C0008557C0008E6
:20006000557C0008557C0008557C0008557C0008557C0008557C0008557C0008557C0008B8
:20008000557C0008517A0008557C000800000000000000000000000000000000557C000802
:2000A0005D7A0008697A0008997A0008F57A0008557C0008017B0008457B0008517B0008EB
:2000C0005D7B0008557C0008557C0008557C0008557C0008697B0008757B000800000000F8
:2000E000817B0008557C0008557C000800000000000000000000000000000000A17B000826
:2001000000000000557C0008557C0008557C00080000000000000000000000000000000054
:20012000557C0008557C0008557C0008557C0008557C000800000000000000000000000082
:20014000000000000000000000000000557C0008557C0008557C0008557C0008557C000862
:20016000557C0008557C0008000000000000000000000000000000000000000000000000CD
:2001800000000000557C00080000000000000000557C0008FFFFFFFFFFFFFFFFFFFFFFFFB9
:2001A00010B5054C237833B9044B13B10448AFF300800123237010BD200600200000000057
:2001C00080F0000808B5034B1BB103490348AFF3008008BD000000002406002080F0000890
:2001E000034613F8012B002AFBD1181A0138704701F0FF01102A2BDB10F0070F08D010F840
:20020000013B013A8B422DD010F0070F42B3F6D1F0B441EA012141EA014122F007047FF0E1
:2002200000070023F0E80256083C85EA010586EA010685FA47F5A3FA87F586FA47F6A5FA04
:2002400087F68EB9EED1F0BC01F0FF0102F0070232B110F8013B013A83EA010313B1F8D123
:200260000020704701387047002D06BF35460338073815F0010F07D1013015F4807F02BFE9
:20028000013015F4C03F0130F0BC0138704700BF81F0004102E000BF83F0004330B54FEA72
:2002A00041044FEA430594EA050F08BF90EA020F1FBF54EA000C55EA020C7FEA645C7FEA8D
:2002C000655C00F0E2804FEA5454D4EB5555B8BF6D420CDD2C4480EA020281EA030382EAF7
:2002E000000083EA010180EA020281EA0303362D88BF30BD11F0004F4FEA01314FF4801C7F
:200300004CEA113102D0404261EB410113F0004F4FEA03334CEA133302D0524263EB43034C
:2003200094EA050F00F0A780A4F10104D5F1200E0DDB02FA0EFC22FA05F2801841F10001BA
:2003400003FA0EF2801843FA05F359410EE0A5F120050EF1200E012A03FA0EFC28BF4CF00E
:20036000020C43FA05F3C01851EBE37101F0004507D54FF0000EDCF1000C7EEB00006EEBD8
:200380000101B1F5801F1BD3B1F5001F0CD349085FEA30004FEA3C0C04F101044FEA445270
:2003A00012F5800F80F09A80BCF1004F08BF5FEA500C50F1000041EB045141EA050130BDD5
:2003C0005FEA4C0C404141EB010111F4801FA4F10104E9D191F0000F04BF01460020B1FA70
:2003E00081F308BF2033A3F10B03B3F120020CDA0C3208DD02F1140CC2F10C0201FA0CF033
:2004000021FA02F10CE002F11402D8BFC2F1200C01FA02F120FA0CFCDCBF41EA0C019040B0
:20042000E41AA2BF01EB0451294330BD6FEA04041F3C1CDA0C340EDC04F11404C4F1200203
:2004400020FA04F001FA02F340EA030021FA04F345EA030130BDC4F10C04C4F1200220FA89
:2004600002F001FA04F340EA0300294630BD21FA04F0294630BD94F0000F83F4801306BF42
:2004800081F480110134013D4EE77FEA645C18BF7FEA655C29D094EA050F08BF90EA020FA7
:2004A00005D054EA000C04BF1946104630BD91EA030F1EBF0021002030BD5FEA545C05D151
:2004C0004000494128BF41F0004130BD14F580043CBF01F5801130BD01F0004545F0FE4166
:2004E00041F470014FF0000030BD7FEA645C1ABF194610467FEA655C1CBF0B46024650EA9B
:20050000013406BF52EA033591EA030F41F4002130BD00BF90F0000F04BF0021704730B5CF
:200520004FF4806404F132044FF000054FF0000150E700BF90F0000F04BF0021704730B5E0
:200540004FF4806404F1320410F0004548BF40424FF000013EE700BF42004FEAE2014FEAC0
:2005600031014FEA02701FBF12F07F4393F07F4F81F06051704732F07F4208BF704793F0EE
:200580007F4F04BF41F40021704730B54FF4607401F0004521F000411CE700BF50EA01023A
:2005A00008BF704730B54FF000050AE050EA010208BF704730B511F0004502D5404261EB1F
:2005C00041014FF4806404F132045FEA915C3FF4D8AE4FF003025FEADC0C18BF03325FEACE
:2005E000DC0C18BF033202EBDC02C2F1200300FA03FC20FA02F001FA03FE40EA0E0021FA12
:2006000002F11444BDE600BF70B54FF0FF0C4CF4E06C1CEA11541DBF1CEA135594EA0C0FE4
:2006200095EA0C0F00F0DEF82C4481EA030621EA4C5123EA4C5350EA013518BF52EA033567
:2006400041F4801143F4801338D0A0FB02CE4FF00005E1FB02E506F00042E0FB03E54FF056
:200660000006E1FB03569CF0000F18BF4EF0010EA4F1FF04B6F5007F64F5407404D25FEA92
:200680004E0E6D4146EB060642EAC62141EA55514FEAC52040EA5E504FEACE2EB4F1FD0C56
:2006A00088BFBCF5E06F1ED8BEF1004F08BF5FEA500E50F1000041EB045170BD06F0004666
:2006C00046EA010140EA020081EA0301B4EB5C04C2BFD4EB0C0541EA045170BD41F480118A
:2006E0004FF0000E013C00F3AB8014F1360FDEBF002001F0004170BDC4F10004203C35DAC8
:200700000C341BDC04F11404C4F1200500FA05F320FA04F001FA05F240EA020001F000426A
:2007200021F0004110EBD37021FA04F642EB06015EEA430E08BF20EAD37070BDC4F10C0441
:20074000C4F1200500FA04F320FA05F001FA04F240EA020001F0004110EBD37041F10001FF
:200760005EEA430E08BF20EAD37070BDC4F1200500FA05F24EEA020E20FA04F301FA05F289
:2007800043EA020321FA04F001F0004121FA04F220EA020000EBD3705EEA430E08BF20EA31
:2007A000D37070BD94F0000F0FD101F00046400041EB010111F4801F08BF013CF7D041EA17
:2007C000060195F0000F18BF704703F00046520043EB030313F4801F08BF013DF7D043EA92
:2007E0000603704794EA0C0F0CEA135518BF95EA0C0F0CD050EA410618BF52EA4306D1D176
:2008000081EA030101F000414FF0000070BD50EA410606BF1046194652EA430619D094EAE4
:200820000C0F02D150EA013613D195EA0C0F05D152EA03361CBF104619460AD181EA0301B6
:2008400001F0004141F0FE4141F470014FF0000070BD41F0FE4141F4780170BD70B54FF035
:20086000FF0C4CF4E06C1CEA11541DBF1CEA135594EA0C0F95EA0C0F00F0A7F8A4EB0504D2
:2008800081EA030E52EA03354FEA013100F088804FEA03334FF0805545EA131343EA12638B
:2008A0004FEA022245EA111545EA10654FEA00260EF000419D4208BF964244F1FD0404F597
:2008C000407402D25B084FEA3202B61A65EB03055B084FEA32024FF480104FF4002CB6EBE5
:2008E000020E75EB030E22BFB61A754640EA0C005B084FEA3202B6EB020E75EB030E22BF02
:20090000B61A754640EA5C005B084FEA3202B6EB020E75EB030E22BFB61A754640EA9C00A2
:200920005B084FEA3202B6EB020E75EB030E22BFB61A754640EADC0055EA060E18D04FEADF
:20094000051545EA16754FEA06164FEAC30343EA52734FEAC2025FEA1C1CC0D111F4801FCA
:200960000BD141EA00014FF000004FF0004CB6E711F4801F04BF01430020B4F1FD0C88BF48
:20098000BCF5E06F3FF6AFAEB5EB030C04BFB6EB020C5FEA500C50F1000041EB045170BD10
:2009A0000EF0004E4EEA113114EB5C04C2BFD4EB0C0541EA045170BD41F480114FF0000E01
:2009C000013C90E645EA060E8DE60CEA135594EA0C0F08BF95EA0C0F3FF43BAF94EA0C0FA0
:2009E0000AD150EA01347FF434AF95EA0C0F7FF425AF104619462CE795EA0C0F06D152EA01
:200A000003353FF4FDAE1046194622E750EA410618BF52EA43067FF4C5AE50EA41047FF44D
:200A20000DAF52EA43057FF4EBAE12E74FF0FF3C06E000BF4FF0010C02E000BF4FF0010C19
:200A40004DF804CD4FEA410C7FEA6C5C4FEA430C18BF7FEA6C5C1BD001B050EA410C0CBF4B
:200A600052EA430C91EA030F02BF90EA020F0020704710F1000F91EA030F58BF994208BFE5
:200A800090422CBFD8176FEAE37040F0010070474FEA410C7FEA6C5C02D150EA013C07D13D
:200AA0004FEA430C7FEA6C5CD6D152EA033CD3D05DF8040B704700BF8446104662468C4644
:200AC0001946634600E000BF01B5FFF7B7FF002848BF10F1000F01BD4DF808EDFFF7F4FFED
:200AE0000CBF012000205DF808FB00BF4DF808EDFFF7EAFF34BF012000205DF808FB00BF6F
:200B00004DF808EDFFF7E0FF94BF012000205DF808FB00BF4DF808EDFFF7CEFF94BF0120AA
:200B200000205DF808FB00BF4DF808EDFFF7C4FF34BF012000205DF808FB00BF4FEA410CBA
:200B40007FEA6C5C02D150EA013C0AD14FEA430C7FEA6C5C02D152EA033C02D14FF0000026
:200B600070474FF0010070474FEA410212F5001215D211D56FF47873B3EB625212D94FEAA1
:200B8000C12343F0004343EA505311F0004F23FA02F018BF404270474FF00000704750EA8C
:200BA000013005D111F0004008BF6FF0004070474FF00000704700BF4A0011D212F50012D5
:200BC00011D20DD56FF47873B3EB62520ED44FEAC12343F0004343EA505323FA02F07047A5
:200BE0004FF00000704750EA013002D14FF0FF3070474FF0000070474FEA4102B2F1E04364
:200C000024BFB3F5001CDCF1FE5C0DD901F0004C4FEAC0024CEA5070B2F1004F40EB830052
:200C200008BF20F00100704711F0804F21D113F13872BCBF01F00040704741F480114FEA53
:200C40005252C2F11802C2F1200C10FA0CF320FA02F018BF40F001004FEAC1234FEAD323DB
:200C600003FA0CFC40EA0C0023FA02F34FEA4303CCE77FEA625307D150EA01331EBF4FF075
:200C8000FE4040F44000704701F0004040F0FE4040F40000704700BF53B94AB9002908BFA3
:200CA00000281CBF4FF0FF314FF0FF3000F072B9ADF1080C6DE904CE00F006F8DDF804E0B8
:200CC000DDE9022304B070472DE9F047089E04468846002B4BD18A42154667D9B2FA82F2E5
:200CE0004AB1C2F1200701FA02F320FA07F7954047EA030894404FEA154E230CB8FBFEF7BF
:200D00001FFA85FC0EFB178843EA084307FB0CF1994209D9EB1807F1FF3080F01B8199424C
:200D200040F21881023F2B445B1AA4B2B3FBFEF00EFB103344EA034400FB0CFCA44509D942
:200D40002C1900F1FF3380F00781A44540F2048102382C4440EA0740A4EB0C0400271EB1E3
:200D6000D4400023C6E900433946BDE8F0878B4209D9002E00F0EB800027C6E90001384622
:200D80003946BDE8F087B3FA83F7002F47D18B4202D3824200F2FA80841A61EB0303012067
:200DA0009846002EE0D0C6E90048DDE702B9FFDEB2FA82F2002A40F08F80491B4FEA154E9B
:200DC0001FFA85F80127B1FBFEFC230C0EFB1C1143EA014308FB0CF1994207D9EB180CF11E
:200DE000FF3002D2994200F2CD808446591AA3B2B1FBFEF00EFB101443EA044408FB00F80D
:200E0000A04507D92C1900F1FF3302D2A04500F2B6801846A4EB080440EA0C409FE7C7F117
:200E2000200CBB4022FA0CFE4EEA030E01FA07F420FA0CF521FA0CF34FEA1E482543B3FB3C
:200E4000F8F92C0C08FB19331FFA8EFA44EA034309FB0AF49C4202FA07F200FA07F10BD95A
:200E60001EEB030309F1FF3080F087809C4240F28480A9F1020973441B1BADB2B3FBF8F028
:200E800008FB103345EA034400FB0AFAA24508D91EEB040400F1FF336BD2A24569D90238FB
:200EA000744440EA0940A0FB0289A4EB0A044C45C2464B4654D351D0002E69D0B1EB0A05C0
:200EC00064EB030404FA0CFCFD40FC404CEA0505C6E90054002747E7C2F1200320FA03F7BB
:200EE000954001FA02F021FA03F34FEA154E3843010CB3FBFEF71FFA85F80EFB173341EA44
:200F0000034107FB08F38B4204FA02F407D9691807F1FF3C2FD28B422DD9023F2944CB1AD4
:200F200081B2B3FBFEF00EFB103341EA034100FB08F38B4207D9691800F1FF3C17D28B4221
:200F400015D902382944C91A40EA07473BE73746304609E70746E7E61846FBE64145ABD240
:200F6000B8EB020A69EB0E0201381346A4E76046E9E7184695E76746D1E781467CE7023828
:200F80002C4447E7ACF1020C2B442FE7384608E73746E9E6704700BF10B5254A254B13603D
:200FA0008CB080234FF6FF71936110460023D160536003930793019393601361CDE9043334
:200FC0000693CDE90833CDE90A3302930AF080FF10B1194B01221A7000234FF4005203A950
:200FE0001348CDE90323CDE905330BF0AFFA10B1114B01221A7000230524502207A90C489C
:201000000993CDE907420B930BF046FB10B10A4B01221A70002301A90548CDE901330BF099
:2010200069FC10B1044B01221A700CB010BD00BFF01C002000040040C922002030B52B4A71
:201040002B4B136042F2CF038FB05360802340F2E731936110460023D16093600393019307
:2010600007931361CDE9043306930293CDE90833CDE90A33CDE90C330AF02AFF10B11D4B22
:2010800001221A704FF4805303A9184803930BF05DFA10B1174B01221A7014480AF0B8FFBC
:2010A00010B1144B01221A70002301A90F48CDE901330BF01FFC10B10E4B01221A70002355
:2010C000602542F2107407A91A46084809930B93CDE907540BF03CF910B1064B01221A7039
:2010E000024806F037FB0FB030BD00BFA81C0020000C0040C9220020284AF8B592E803003C
:20110000274C284D2378284E28604FEA114C1C22A98085F806C043F02003A5F114004FF6C9
:20112000FF7711462370378006F096FDA5F1180445F8180C264684460FCE1C4FDFF888E03F
:2011400007F11C050FC596E80F0085E80F000FCCBD68CEF800C0164EDFF870C03E606E1C80
:2011600007F13C050FC5C7E901C694E80F0085E80F0000BF0F4E104D1049114800240A2368
:20118000142234802C700BF099FC00BF0D4B012220461A7008F080F800BFF8BD14FB000814
:2011A000CC220020E02300202A000020F8190020785634121C0000208824002020FB000844
:2011C000982400204E2500200C060020466D6574094B82B00022ADF806005A625A62596A54
:2011E000BDF80620914205D200BF596ABDF806209142F9D302B07047004401400000000080
:201200002DE9F843344B1C788CB300224FF45041324809F0E3F800224FF47071304809F030
:20122000DDF800BF2AA7D7E90067DFF8B890DFF8AC80142548460AF0CBFA2021404609F0BA
:20124000D1F800BF002400BF01342046FFF762F932463B46FFF74AFC0028F4D16B1E13F089
:20126000FF05E7D100BFBDE8F84308F097BD22464FF480711A4809F0B1F8224680211848BE
:2012800009F0ACF822464021154809F0A7F822464FF40041114809F0A1F822464FF48041B0
:2012A0000E4809F09BF822464FF400510B4809F095F822464FF48051084809F08FF82246C3
:2012C0004FF40071064809F089F8AAE7AFF300800000000080841E413C06002000040240D4
:2012E00000080240A41B002010B5204B1C786CB100224FF450411E4809F070F800224FF4C2
:2013000070711C48BDE8104009F068B822464FF48071184809F062F822468021154809F0CC
:201320005DF822464021134809F058F822464FF400410F4809F052F822464FF480410C48A5
:2013400009F04CF822464FF40051094809F046F822464FF48051064809F040F822464FF426
:2013600000710448BDE8104009F038B83C060020000402400008024070B59E4E3378002BF9
:2013800073D09D4DFFF7B0FF9C4A2B789C48D45CE30754BF01220022802109F01FF8A00744
:2013A00054BF012200221021964809F017F8610754BF012200222021924809F00FF82207BA
:2013C00059BF01221146002201218F4809F006F8E3064CBF002201228B48022108F0FEFF45
:2013E000A0064CBF002201220421874808F0F6FF61064CBF002201224FF48061824808F079
:20140000EDFF22064CBF0022012210217C4808F0E5FF00BF7D4A13780133DBB20F2B137008
:201420000BD9002313703378002B3CD02B78032B13D8DFE803F060574F4775493278097894
:201440009942F0D22C78631CDBB242B9072B2B7001D900232B7000BF70BD0133DBB2032B04
:201460002B70F8D900232B70F5E70821654808F0AFFF60B9604D67492A7831F9123013F162
:20148000090F6CDB013B21F8123000BF7AE700BF594D604B297833F91120092A57DC01328F
:2014A00023F811206EE701224FF40061544808F095FF2C78072C2ED8DFE804F0888078265E
:2014C0007069625A01224FF440714E4808F086FF3278B7E70122C0214A4808F07FFF32784F
:2014E0002C78B0E701224FF44041474808F076FF32782C78A7E701224FF44051424808F079
:201500006DFF32782C789EE701224FF400713D4808F064FF2C78404B1B782341DB0714D5E4
:201520003E4B1A78224112F0010260D03C494FF47A720023D1E90001FFF7AEFB00214FF463
:20154000FA70994208BF904248D332787BE7354A012310788B400343DBB2137012E73148C8
:201560000121037801FA02F223EA020202708CE701224FF40041244808F030FF2C78CAE75A
:20158000012240211F4808F029FF2C78C3E7012280211C4808F022FF2C78BCE701224FF404
:2015A0008071184808F01AFF2C78B4E701224FF48051154808F012FF2C78ACE701224FF450
:2015C0000051114808F00AFF2C78A4E701224FF480410D4808F002FF2C789CE700224FF430
:2015E0000061074808F0FAFE32782C782BE700BFF5E700BF3C060020B21600200400002023
:201600000000024000080240000402404306002000000020D01700200C1C0020B01B002035
:2016200090240020F4190020594970B5D1E90045621C45F10003C1E90023FFF79DFE554A2F
:2016400013889BB21BB11388013B9BB21380524A13889BB21BB11388013B9BB213804F4A7F
:2016600013889BB21BB11388013B9BB213804C4A13889BB21BB11388013B9BB21380494A6B
:2016800013889BB21BB11388013B9BB21380464A13889BB21BB11388013B9BB21380434B56
:2016A0001A781AB11A78013AD2B21A70404B1A6812B11A68013A1A603E4B1A781AB11A7873
:2016C000013AD2B21A703C4B1A6812B11A68013A1A603A4A13889BB21BB11388013B9BB262
:2016E0001380374A13889BB21BB11388013B9BB21380344A13889BB2012B00F018811388B5
:201700009BB2002B3ED1304A13889BB243B113884FF6FF71994203D01388013B9BB2138037
:201720002A4A13889BB243B113884FF6FF71994203D01388013B9BB21380254C2578012D68
:2017400052D0002D00F09B804FF40041214808F03FFE214B1A78824204D0204A18701388EA
:20176000013313801E4A1388013B9BB2002B40F0DC801A491B480C8804804FF47A700B80C9
:20178000108070BD1388013B9BB21380BBE700BF9024002030230020DA24002028000020C7
:2017A000F21900201A000020E4190020E619002024000020C023002020000020EC1C0020D9
:2017C0009C1C0020E82300202A0000201C0000203C06002000000240F8170020B0160020C7
:2017E00014000020381D00204FF40051844808F0EFFD844A92F90030002800F0A280D81D44
:20180000BBBF814A137803F1FF3303F0DF03137001217B4808F0DCFD7C4A92F9003000281B
:2018200040F0B680072BC5BF774A1378013343F0800313700221724808F0CAFD744A92F9EE
:201840000030002840F09A80072BC5BF6E4A1378013343F0010313700421694808F0B8FD7C
:201860006C4A92F90030002840F08280072B00F3C080257801331370002D7FF465AF01210E
:201880005F48654E08F0A4FD96F90030002852D0D81DC0F29180013B604C33700221584846
:2018A00008F096FD00285CD000BF96F90130072B00F38E80013373700421514808F088FD45
:2018C000002847D000BF96F90230072B6ADC0133B370534A23791178C3F3400399420DD007
:2018E0002379C3F34003137000BF237913F0040F236814BF013303F1FF332360494A2379F5
:201900001178C3F3800399423FF41EAF2379C3F38003137000BF237913F0020F236814BF05
:2019200003F1FF33013323600EE7138070BD3E4B00221A70E7E6072B44DC01333370374C67
:20194000ACE7072BC5BF304A1378013343F0200313705DE796F90230DA1D3EDB013BB370B8
:20196000B7E796F90130D91D21DB013B7370A3E7DD1D37DB013B13702578E2E6DE1DBBBFC9
:20198000214A137803F1FF3303F0FE03137063E7D91DBBBF1C4A137803F1FF3303F07F036E
:2019A000137047E7237943F00403237191E7237960F3410323717FE7184C237965F300030C
:2019C00023716BE7154C237943F00103237165E7237943F0020323716EE7237960F38203DC
:2019E000237176E7084A2578137803F0BF031370A7E6054A2578137843F040031370A0E6C1
:201A000000080240B6160020F4190020B5160020B4160020B316002040060020901C002073
:201A2000F0170020F1170020F823002070B500BF4FF48071094808F0CBFC68B9084A09492F
:201A4000536A0E68084D094C43EA06432B60012308605062237070BD00BF70BD000002407C
:201A60000000014034230020081C0020981A0020284B1A78002A43D00020274A274930B471
:201A8000187010680B68264C1B1A002BB8BF5B4242F20F7083422CDC224B15681068224A9F
:201AA000186010781A680D6002FB00F21F481A601968007891FBF0F200FB12121C491D4D12
:201AC000D2B20A7019686A7D91FBF0F11A48196019680160C2F3411200212170D10712D4FE
:201AE000920703D51A6869680A441A60186830BC70472378012BCFD85A1C2270094BF5E791
:201B0000084B186870471A686968521A1A60186830BC7047981A0020081C0020F41700209E
:201B2000E1170020981C0020DE240020E9240020EA240020C8230020081B002000BF024AE3
:201B400013680133136070473423002000BF0549054A0B8801339BB20B80138801339BB21E
:201B600013807047F02300200C00002070B500BF40210A4808F02CFC68B9094A0949536A82
:201B80000E88094D094C43EA06432B60012308805062237070BD00BF70BD00BF00000240F8
:201BA00000040040F0230020E81C00203425002000BF024A1368013313607047BC2200202F
:201BC0000B4B0C4A1868116870B401380A4E18601C68736B094D0A4803EB0443591A13600E
:201BE0000123002429600370546070BC704700BFBC220020E8170020004801403C1D00202C
:201C0000C822002010B50446FEF7EAFA214682B20A230248BDE810400AF050BF98240020E6
:201C2000F8B5444B444A454D45482C780A21197013889BB2591C89B211801188C4547F29E1
:201C400088BF00233F4C88BF13803C493E4801220AF0E4FF2388C72B07D82A783B4E5D1C8A
:201C6000ADB20A2A2580F25400D0F8BD384F39490023062230463B7073550BF017FE30B331
:201C80000622354930460BF011FE002838D00622324930460BF00AFE002838D00622304901
:201CA00030460BF003FE20B306222E4930460BF0FDFDC0B32C49052230460BF0F7FD3146EA
:201CC00060BB07F59660C8220BF002FE0CE03146C82207F1C8000BF0FBFD2449244B012015
:201CE0004FF4FA6208701A80224A002315802380F8BD314607F54870C8220BF0E9FDF3E7E7
:201D0000314607F5C870C8220BF0E2FDECE7314607F51670C8220BF0DBFDE5E73846C82297
:201D20000BF0D6FDE0E7314607F57A70C8220BF0CFFDD9E7E6190020DC240020D8240020E5
:201D4000101C0020FE1700203823002044060020441D002000F1000808F1000810F1000899
:201D600018F1000820F1000828F10008F8230020E8230020041C0020014610B50A220446F0
:201D80002D480BF0A5FD2D4B0021C3E900112278002A50D02D3AD2B24F2A9CBF2849895CE2
:201DA00019706278002A46D02D3AD2B24F2A96BF234900228A5C5A70A278002A3BD02D3AD3
:201DC000D2B24F2A96BF1E4900228A5C9A70E278002A30D02D3AD2B24F2A96BF1849002278
:201DE0008A5CDA702279002A25D02D3AD2B24F2A96BF134900228A5C1A716279DAB12D3A84
:201E0000D2B24F2A96BF0E4900228A5C5A71A2798AB12D3AD2B24F2A96BF094900228A5CDD
:201E20009A71E2793AB12D3AD2B24F2A96BF044900228A5CDA7110BDE819002004000020E6
:201E4000B0F0000838B50A2205460C46014646480BF03EFD454B0021C3E900112A78002ADF
:201E600050D02D3AD2B24F2A9CBF4149895C19706A78002A46D02D3AD2B24F2A96BF3C492B
:201E800000228A5C5A70AA78002A3BD02D3AD2B24F2A96BF364900228A5C9A70EA78002A43
:201EA00030D02D3AD2B24F2A96BF314900228A5CDA702A79002A25D02D3AD2B24F2A96BF22
:201EC0002B4900228A5C1A716A79DAB12D3AD2B24F2A96BF264900228A5C5A71AA798AB134
:201EE0002D3AD2B24F2A96BF214900228A5C9A71EA793AB12D3AD2B24F2A96BF1C4900221E
:201F00008A5CDA71E20903D01A7862F07F021A70600603D55A7862F07F025A70A10603D5B7
:201F20009A7862F07F029A70E20603D5DA7862F07F02DA70250703D51A7962F07F021A718E
:201F4000600703D55A7962F07F025A71A10703D59A7962F07F029A71E20703D5DA7962F0FA
:201F60007F02DA7138BD00BFE819002004000020B0F000082DE9F0435A4E87B0014604463B
:201F8000132201A80BF0A4FC737D13F00C0F46D001A8FEF725F9002304E011F8142C2E2A40
:201FA00000F09780DAB206A99042114403F10103F3D800238DF80C3001A8FEF711F9013830
:201FC000C0B243B25D1C00F08A8006AA1A4412F8141C302940F0818012F8151C2E297CD077
:201FE000202007E012F8141C302944D112F8151C2E2940D0013BDDB26BB202F8140C591CF9
:020000040800F2
:2020000006AA1A44EED101A8FEF7EAF80138C0B2FF2500BF737D03F00C03082B36D14FF07A
:2020200000094D46C8462646012705E00135EDB23270661909F1010901A8FEF7D1F85FFAC3
:2020400089F306AA98421A440ED912F8142C2E2AECD1C3F1080007FA00F048EA0000C0B285
:2020600000BF4FFA80F8E5E70023337000BF404607B0BDE8F08301A8FEF7B2F80138C0B247
:2020800000BF737D03F00C03082BC8D0451B6DB2002D1CDD0027202601A8FEF7A1F8C0B209
:2020A000431E5BB2002B0EDD0DF103020238D118C0B201AA091A134413F8012C1A7003F822
:2020C000016D9942F8D101377FB2BD42E4D100BFA5E700238DF80D306EE70546D0E7FF2526
:2020E000CEE700BFC823002070B52DED028B4CF24F339A4288B005460E461ED9324B9A42D2
:2021000037D832483249A0FB023080094FF47A736C4603FB1023024620460BF08FFB40F2ED
:20212000057006F095FE224631462846012306F0F9FB08B0BDEC028B70BD10EE100AB0EE75
:20214000408AFEF709FADFED237AB4EEE78AF1EE10FA02460B4621DADFED1F7AB4EEE78A4C
:20216000F1EE10FA0DDA6C4620461C490BF066FBD5E71B4C1B4984FB0204D017C0EBA44034
:20218000C6E70DA3D3E90023FEF73EFA6C4602460B46204614490BF051FBC0E708A3D3E973
:2021A0000023FEF731FA6C4602460B4620460F490BF044FBB3E700BFFCA9F1D24D62503F9A
:2021C0008DEDB5A0F7C6B03E40420F00D34D6210B8F100080024744900007A44DCF100083D
:2021E00083DE1B43ACF10008D0F10008C4F10008F8B5634B1D780E46002D40F0D380614B55
:20220000984200F31782B0F57A7FC0F280815E4B5E4C5F4983FB0023C217C2EBA3124FF4ED
:202220007A7303FB120320460BF008FB2046FFF7A1FE0A222146C7B256480BF049FB564BB5
:202240002278C3E90055002A56D02D3AD2B24F2A9CBF52498D5C62781D70002A4CD02D3A3C
:20226000D2B24F2A9CBF4D49895CA27888BF00215970002A40D02D3AD2B24F2A9CBF4749B7
:20228000895CE27888BF00219970002A34D02D3AD2B24F2A9CBF4149895C227988BF00212F
:2022A000D970002A28D02D3AD2B24F2A9CBF3B49895C627988BF00211971EAB12D3AD2B238
:2022C0004F2A9CBF3549895CA27988BF0021597192B12D3AD2B24F2A9CBF3049895CE279BF
:2022E00088BF002199713AB12D3AD2B24F2A96BF2A4900228A5CDA71FA0903D01A7862F048
:202300007F021A70790603D55A7862F07F025A70BA0603D59A7862F07F029A70FD0603D58A
:20232000DA7862F07F02DA703C0703D51A7962F07F021A71780703D55A7962F07F025A715A
:20234000B90703D59A7962F07F029A71FA0703D5DA7962F07F02DA7141F2326006F078FD7A
:202360000021084601230E4A06F0DCFAC0B2324601230021083006F0D5FAC0B200BFF8BD94
:202380003C0600203F420F00D34D62100418002074F10008E819002004000020B0F0000823
:2023A000C0F10008994B984200F30082984B984200F37083974B984200F3B48242F20F73F3
:2023C000984200F38B83B0F57A7F80F27983924C9249024620460BF031FA2046FFF7CAFD66
:2023E00021460A22C5B28E480BF072FA8D4B22780021C3E90011002A56D02D3AD2B24F2A92
:202400009CBF8949895C62781970002A4CD02D3AD2B24F2A9CBF8449895CA27888BF00210E
:202420005970002A40D02D3AD2B24F2A9CBF7E49895CE27888BF00219970002A34D02D3ACE
:20244000D2B24F2A9CBF7849895C227988BF0021D970002A28D02D3AD2B24F2A9CBF724996
:20246000895C627988BF00211971EAB12D3AD2B24F2A9CBF6C49895CA27988BF0021597169
:2024800092B12D3AD2B24F2A9CBF6749895CE27988BF002199713AB12D3AD2B24F2A96BF34
:2024A000614900228A5CDA71EA0903D01A7862F07F021A70690603D55A7862F07F025A70B4
:2024C000AA0603D59A7862F07F029A70EF0603D5DA7862F07F02DA702C0703D51A7962F059
:2024E0007F021A71680703D55A7962F07F025A71A90703D59A7962F07F029A71EA0703D5D6
:20250000DA7962F07F02DA7141F232606DE0424C4649024620460BF091F90A2221464048CD
:202520000BF0D6F93F4B2278C3E90055002A56D02D3AD2B24F2A9CBF3B498D5C62781D70C9
:20254000002A4CD02D3AD2B24F2A9CBF3649895CA27888BF00215970002A40D02D3AD2B2A2
:202560004F2A9CBF3049895CE27888BF00219970002A34D02D3AD2B24F2A9CBF2A49895C19
:20258000227988BF0021D970002A28D02D3AD2B24F2A9CBF2449895C627988BF00211971EF
:2025A000EAB12D3AD2B24F2A9CBF1F49895CA27988BF0021597192B12D3AD2B24F2A9CBF25
:2025C0001949895CE27988BF002199713AB12D3AD2B24F2A96BF144900228A5CDA71DA7940
:2025E00062F07F0241F23260DA7106F031FC00210F4A0846012306F095F9C0B23246012357
:202600000021083006F08EF9C0B2F8BD7F9698003F420F009F86010004180020A4F1000881
:20262000E819002004000020B0F0000880F1000888F10008564F574C574987FB0027C21749
:20264000C2EBA742013303FB120320460BF0F6F82046FFF78FFC0A222146C7B24F480BF0C9
:2026600037F94F4B2278C3E90055002A56D02D3AD2B24F2A9CBF4B498D5C62781D70002AD8
:202680004CD02D3AD2B24F2A9CBF4649895CA27888BF00215970002A40D02D3AD2B24F2A02
:2026A0009CBF4049895CE27888BF00219970002A34D02D3AD2B24F2A9CBF3A49895C227996
:2026C00088BF0021D970002A28D02D3AD2B24F2A9CBF3449895C627988BF00211971EAB19E
:2026E0002D3AD2B24F2A9CBF2E49895CA27988BF0021597192B12D3AD2B24F2A9CBF2949FE
:20270000895CE27988BF002199713AB12D3AD2B24F2A96BF234900228A5CDA71FA0903D0CE
:202720001A7862F07F021A707C0603D55A7862F07F025A70B80603D59A7862F07F029A705C
:20274000F90603D5DA7862F07F02DA703A0703D51A7962F07F021A717D0703D55A7962F0A8
:202760007F025A71BC0703D59A7962F07F029A71F80703D5DA7962F07F02DA7141F2326074
:2027800006F066FB002108460123074A33E700BF83DE1B430418002068F10008E8190020A8
:2027A00004000020B0F00008B4F100085549564B564A81FB0041C517C5EB2131A3FB014344
:2027C0005B096427524C82FB000207FB13135149C5EBA24220460BF031F82046FFF7CAFBEC
:2027E00021460A22C5B24C480BF072F84B4B22780021C3E90011002A56D02D3AD2B24F2A14
:202800009CBF4749895C62781970002A4CD02D3AD2B24F2A9CBF4249895CA27888BF00218E
:202820005970002A40D02D3AD2B24F2A9CBF3C49895CE27888BF00219970002A34D02D3A0C
:20284000D2B24F2A9CBF3649895C227988BF0021D970002A28D02D3AD2B24F2A9CBF304916
:20286000895C627988BF00211971EAB12D3AD2B24F2A9CBF2A49895CA27988BF00215971A7
:2028800092B12D3AD2B24F2A9CBF2549895CE27988BF002199713AB12D3AD2B24F2A96BF72
:2028A0001F4900228A5CDA71EA0903D01A7862F07F021A706F0603D55A7862F07F025A70EC
:2028C000AC0603D59A7862F07F029A70E80603D5DA7862F07F02DA70290703D51A7962F05D
:2028E0007F021A716A0703D55A7962F07F025A71AF0703D59A7962F07F029A71ED077FF52B
:202900003DAF37E7AD8BDB681F85EB5183DE1B43041800208CF10008E8190020040000208D
:20292000B0F00008784B7949794D7A4C83FB0023C217C2EB6313A1FB0371C90801EB8101F2
:2029400085FB0050A3EB41037349C2EBA01220460AF074FF2046FFF70DFB21460A22C5B279
:202960006E480AF0B5FF6E4B22780021C3E90011002A56D02D3AD2B24F2A9CBF6949895C1C
:2029800062781970002A4CD02D3AD2B24F2A9CBF6449895CA27888BF00215970002A40D0B8
:2029A0002D3AD2B24F2A9CBF5E49895CE27888BF00219970002A34D02D3AD2B24F2A9CBF14
:2029C0005849895C227988BF0021D970002A28D02D3AD2B24F2A9CBF5249895C627988BFA2
:2029E00000211971EAB12D3AD2B24F2A9CBF4D49895CA27988BF0021597192B12D3AD2B2DC
:202A00004F2A9CBF4749895CE27988BF002199713AB12D3AD2B24F2A96BF424900228A5C69
:202A2000DA71EA0903D01A7862F07F021A706C0603D55A7862F07F025A70A80603D59A7845
:202A400062F07F029A70E90603D5DA7862F07F02DA702A0703D51A7962F07F021A716F07F3
:202A600003D55A7962F07F025A71AC0703D59A7962F07F029A71E80703D5DA7962F07F02A4
:202A8000DA7141F2326006F0E3F9002108460123254AB0E51E49254A81FB0043C517C5EB9C
:202AA000A313A1FB03411B4C890982FB00024FF47A7707FB1133C5EBA24220461C498AE6BF
:202AC000134B144C1A4983FB0023C217C2EBA3124FF47A7303FB1203204639E715490A4B7D
:202AE0000B4A81FB0041C517C5EBA101A3FB0143084C82FB00025B09642707FB1313C5EB1A
:202B0000A21220460C4923E71F85EB51CDCCCCCCD34D6210041800209CF10008E8190020A7
:202B200004000020B0F00008C0F1000883DE1B4394F10008676666668CF100082DE9F0415F
:202B4000604D88B02B780446E8460F4640462246002B40F0B3805C490AF070FEB4F57A7FF5
:202B60002AD35A4E2B78B44294BF08264826012B27D013B9564B9C4227D90A225549564852
:202B80000AF0A6FE554B56490022C3E9001241F2326006F05DF9002108460123514A05F044
:202BA000C1FEC0B23A4601230021083005F0BAFEC0B208B0BDE8F0812B78012B4FF00006E6
:202BC000D7D142F20F739C42D7D841460A2242480AF07EFE414B9DF800200021C3E9001138
:202BE000002A5DD02D3AD2B24F2A9CBF3E49895C9DF801201970002A52D02D3AD2B24F2A64
:202C00009CBF3949895C9DF8022088BF00215970002A45D02D3AD2B24F2A9CBF3249895CAC
:202C20009DF8032088BF00219970002A38D02D3AD2B24F2A9CBF2C49895C9DF8042088BF20
:202C40000021D970002A2BD02D3AD2B24F2A9CBF2549895C9DF8052088BF00211971FAB17C
:202C60002D3AD2B24F2A9CBF1F49895C9DF8062088BF002159719AB12D3AD2B24F2A9CBF51
:202C80001949895C9DF8072088BF002199713AB12D3AD2B24F2A96BF134900228A5CDA716C
:202CA000B20903D05A7862F07F025A7030077FF56EAF1A7962F07F021A7168E70B490AF0C1
:202CC000BDFD4BE73C06002030F100083F420F00FFE0F5053CF10008E8190020040000209A
:202CE0003F3E795038F10008B0F0000834F1000870B52DED028B6E4B1C7888B0B0EE408ACF
:202D00000546B5EE400A002C40F0E280F1EE10FA00F0D78110EE100AFDF71EFCDFED6A7AB6
:202D2000B4EEE78AF1EE10FA02460B4680F21684DFED667AB4EEE78AF1EE10FAC0F2F48123
:202D400059A3D3E90023FDF75FFC0B460246594968460AF073FD6846FFF70CF90A22694672
:202D6000C6B255480AF0B4FD544B9DF80020C3E90044002A5DD02D3AD2B24F2A9CBF5049A0
:202D80008C5C9DF801201C70002A52D02D3AD2B24F2A9CBF4A49895C9DF8022088BF002167
:202DA0005970002A45D02D3AD2B24F2A9CBF4449895C9DF8032088BF00219970002A38D07F
:202DC0002D3AD2B24F2A9CBF3D49895C9DF8042088BF0021D970002A2BD02D3AD2B24F2AD6
:202DE0009CBF3749895C9DF8052088BF00211971FAB12D3AD2B24F2A9CBF3149895C9DF809
:202E0000062088BF002159719AB12D3AD2B24F2A9CBF2B49895C9DF8072088BF00219971C9
:202E20003AB12D3AD2B24F2A96BF254900228A5CDA71F20903D01A7862F07F021A707106F9
:202E400003D55A7862F07F025A70B20603D59A7862F07F029A70F40603D5DA7862F07F02B5
:202E6000DA70300703D51A7962F07F021A71710703D55A7962F07F025A71B20703D59A79A3
:202E800062F07F029A71F40703D5DA7962F07F02DA7141F2326005F0DBFF002108460123E9
:202EA000084ADAE0AFF30080FCA9F1D24D62503F3C06002050F10008E8190020040000204E
:202EC000B0F00008C0F100080024744900007A44F1EE10FA00F0D08010EE100AFDF73CFB86
:202EE0005FED077AB4EEE78AF1EE10FA02460B4680F270825FED0B7AB4EEE78AF1EE10FA3F
:202F000080F2B281814968460AF098FC6846FFF731F869460A22C4B27D480AF0D9FC7D4B8C
:202F20009DF800200021C3E90011002A5DD02D3AD2B24F2A9CBF7849895C9DF80120197003
:202F4000002A52D02D3AD2B24F2A9CBF7249895C9DF8022088BF00215970002A45D02D3A38
:202F6000D2B24F2A9CBF6C49895C9DF8032088BF00219970002A38D02D3AD2B24F2A9CBF45
:202F80006549895C9DF8042088BF0021D970002A2BD02D3AD2B24F2A9CBF5F49895C9DF82E
:202FA000052088BF00211971FAB12D3AD2B24F2A9CBF5949895C9DF8062088BF002159711C
:202FC0009AB12D3AD2B24F2A9CBF5349895C9DF8072088BF002199713AB12D3AD2B24F2AE9
:202FE00096BF4D4900228A5CDA71E20903D01A7862F07F021A70600603D55A7862F07F0203
:203000005A70A10603D59A7862F07F029A70E20603D5DA7862F07F02DA70260703D51A79B1
:2030200062F07F021A71600703D55A7962F07F025A71A10703D59A7962F07F029A71E20728
:2030400003D5DA7962F07F02DA7141F2326005F0FFFE0021314A0846012305F063FCC0B29C
:203060002A4601230021083005F05CFCC0B200BF08B0BDEC028B70BD0A22294924480AF0C6
:2030800027FC244B00244FF07C51C3E900146FF07F0241F23260DA7105F0DAFE2146204624
:2030A00001231E4A05F03EFCC0B221462A460123083005F037FCC0B200BF08B0BDEC028B69
:2030C00070BD0A22174912480AF002FC114B4FF07C51C3E900416FF0400241F23260DA71DF
:2030E00005F0B6FE214601230C4A204605F01AFCC0B22A4621460123083005F013FCC0B2BA
:2031000000BF08B0BDEC028B70BD00BF60F10008E819002004000020B0F0000888F100084F
:2031200048F1000844F10008A54968460AF086FB6846FEF71FFF0A226946C6B2A1480AF003
:20314000C7FBA14B9DF80020C3E90044002A5DD02D3AD2B24F2A9CBF9C498C5C9DF8012083
:203160001C70002A52D02D3AD2B24F2A9CBF9749895C9DF8022088BF00215970002A45D0CC
:203180002D3AD2B24F2A9CBF9049895C9DF8032088BF00219970002A38D02D3AD2B24F2AF3
:2031A0009CBF8A49895C9DF8042088BF0021D970002A2BD02D3AD2B24F2A9CBF8349895CFD
:2031C0009DF8052088BF00211971FAB12D3AD2B24F2A9CBF7D49895C9DF8062088BF00210B
:2031E00059719AB12D3AD2B24F2A9CBF7749895C9DF8072088BF002199713AB12D3AD2B252
:203200004F2A96BF714900228A5CDA71F20903D01A7862F07F021A70700603D55A7862F0A4
:203220007F025A70B10603D59A7862F07F029A70F20603D5DA7862F07F02DA70340703D573
:203240001A7962F07F021A71700703D55A7962F07F025A71B10703D59A7962F07F029A713C
:20326000F2077FF5F2AEECE653A3D3E90023FDF7CBF90B460246564968460AF0DFFA68467B
:20328000FEF778FE69460A22C4B24E480AF020FB4D4B9DF800200021C3E90011002A5DD045
:2032A0002D3AD2B24F2A9CBF4849895C9DF801201970002A52D02D3AD2B24F2A9CBF434903
:2032C000895C9DF8022088BF00215970002A45D02D3AD2B24F2A9CBF3C49895C9DF8032001
:2032E00088BF00219970002A38D02D3AD2B24F2A9CBF3649895C9DF8042088BF0021D9709E
:20330000002A2BD02D3AD2B24F2A9CBF2F49895C9DF8052088BF00211971FAB12D3AD2B22A
:203320004F2A9CBF2949895C9DF8062088BF002159719AB12D3AD2B24F2A9CBF2349895C1A
:203340009DF8072088BF002199713AB12D3AD2B24F2A96BF1D4900228A5CDA71E20903D024
:203360001A7862F07F021A70620603D55A7862F07F025A70A60603D59A7862F07F029A703C
:20338000E00603D5DA7862F07F02DA70210703D51A7962F07F021A71620703D55A7962F0A9
:2033A0007F025A71A60703D59A7962F07F029A71E4077FF56EAD68E5FCA9F1D24D62503FDE
:2033C00050F10008E819002004000020B0F0000860F100085AA3D3E90023FDF715F90B462F
:2033E0000246594968460AF029FA6846FEF7C2FD69460A22C4B255480AF06AFA544B9DF836
:2034000000200021C3E90011002A5DD02D3AD2B24F2A9CBF4F49895C9DF801201970002AB2
:2034200052D02D3AD2B24F2A9CBF4A49895C9DF8022088BF00215970002A45D02D3AD2B221
:203440004F2A9CBF4349895C9DF8032088BF00219970002A38D02D3AD2B24F2A9CBF3D4987
:20346000895C9DF8042088BF0021D970002A2BD02D3AD2B24F2A9CBF3649895C9DF80520FB
:2034800088BF00211971FAB12D3AD2B24F2A9CBF3049895C9DF8062088BF002159719AB13A
:2034A0002D3AD2B24F2A9CBF2A49895C9DF8072088BF002199713AB12D3AD2B24F2A96BF23
:2034C000244900228A5CDA71E20903D01A7862F07F021A70660603D55A7862F07F025A70CC
:2034E000A00603D59A7862F07F029A70E10603D5DA7862F07F02DA70220703D51A7962F04B
:203500007F021A71660703D55A7962F07F025A71A00703D59A7962F07F029A71E10703D5B9
:20352000DA7962F07F02DA7141F2326005F090FC002108460123084A8FE500BFAFF300809A
:203540008DEDB5A0F7C6B03E58F10008E819002004000020B0F00008B4F1000858A3D3E94F
:203560000023FDF751F80B460246514968460AF065F96846FEF7FEFC0A226946C6B24D482D
:203580000AF0A6F94C4B9DF80020C3E90044002A5DD02D3AD2B24F2A9CBF48498C5C9DF832
:2035A00001201C70002A52D02D3AD2B24F2A9CBF4249895C9DF8022088BF00215970002AD1
:2035C00045D02D3AD2B24F2A9CBF3C49895C9DF8032088BF00219970002A38D02D3AD2B267
:2035E0004F2A9CBF3549895C9DF8042088BF0021D970002A2BD02D3AD2B24F2A9CBF2F49CE
:20360000895C9DF8052088BF00211971FAB12D3AD2B24F2A9CBF2949895C9DF8062088BF56
:20362000002159719AB12D3AD2B24F2A9CBF2349895C9DF8072088BF002199713AB12D3AC4
:20364000D2B24F2A96BF1D4900228A5CDA71F20903D01A7862F07F021A70720603D55A7880
:2036600062F07F025A70B40603D59A7862F07F029A70F00603D5DA7862F07F02DA703107B7
:2036800003D51A7962F07F021A71720703D55A7962F07F025A71B40703D59A7962F07F0226
:2036A0009A71F0077FF540AF3AE700BFAFF3008050F10008E819002004000020B0F000086D
:2036C0008DEDB5A0F7C6B03E2DE9F0412DED028BBD4BDFEDBE7A93F8008088B0B0EE408ACB
:2036E00006460F461546B4EEE70AB8F1000F43D1F1EE10FA80F24B81DFEDB57AB4EEE70ABA
:20370000F1EE10FA80F2A281DFEDB27AB4EEE70AF1EE10FA80F29A81DFEDAF7AB4EEE70AA2
:20372000F1EE10FA80F2A08110EE100AFCF714FFF2EE047AB4EEE78AF1EE10FA02460B46FC
:2037400080F2AE81F7EE007AB4EEE78AF1EE10FA6C46ACBFA149A24920460AF06FF841F281
:20376000326005F075FB4146404601239D4A05F0D9F85FFA80F85BE0F1EE10FA80F24A8142
:20378000DFED937AB4EEE70AF1EE10FA35DADFED917AB4EEE70AF1EE10FA2EDADFED8E7A96
:2037A000B4EEE70AF1EE10FA27DA10EE100AFCF7D3FEF2EE047AB4EEE78AF1EE10FA80F2E4
:2037C0007381F7EE007AB4EEE78AF1EE10FA0B466C46ACBF84498549024620460AF02EF8C3
:2037E00041F2326005F034FB0021084601237D4A05F098F85FFA80F81AE0DFED7D7A68EE1D
:20380000277A6C4617EE900AFCF7A6FE0B467949024620460AF012F841F2326005F018FB8D
:20382000002108460123744A05F07CF85FFA80F82046FEF79FFB21460A22C4B26F480AF04E
:2038400047F86F4B9DF800200021C3E90011002A5DD02D3AD2B24F2A9CBF6A49895C9DF899
:2038600001201970002A52D02D3AD2B24F2A9CBF6449895C9DF8022088BF00215970002AEF
:2038800045D02D3AD2B24F2A9CBF5E49895C9DF8032088BF00219970002A38D02D3AD2B282
:2038A0004F2A9CBF5749895C9DF8042088BF0021D970002A2BD02D3AD2B24F2A9CBF5149C7
:2038C000895C9DF8052088BF00211971FAB12D3AD2B24F2A9CBF4B49895C9DF8062088BF72
:2038E000002159719AB12D3AD2B24F2A9CBF4549895C9DF8072088BF002199713AB12D3AE0
:20390000D2B24F2A96BF3F4900228A5CDA71E20903D01A7862F07F021A70620603D55A78BB
:2039200062F07F025A70A00603D59A7862F07F029A70E10603D5DA7862F07F02DA70220726
:2039400003D51A7962F07F021A71600703D55A7962F07F025A71A10703D59A7962F07F0288
:203960009A71E20703D5DA7962F07F02DA71384605F06EFA3246294608F10A00012304F02D
:20398000D1FFC0B208B0BDEC028BBDE8F081DFED207A60EE277A6C4617EE900AFCF7DCFD6F
:2039A00002460B462046184909F048FF41F2326005F04EFA414640460123144A04F0B2FF31
:2039C0005FFA80F834E700BF3C060020002474490050C34700401C4600007A4440F2000805
:2039E00048F200083CF2000850F2000858F200086F12833A60F1000828F20008E8190020D9
:203A000004000020B0F0000818F20008DCF40008BD3786355FED027A60EE277A6C4617EED3
:203A2000900AFCF799FD02460B462046214909F005FF41F2326005F00BFA002108460123AB
:203A40001D4A04F06FFF5FFA80F8F1E6DFED1B7A68EE277A6C4617EE900AFCF77DFD024697
:203A60000B4620461649D5E6DFED147A60EE277A6C4617EE900AFCF76FFD02460B4620467D
:203A8000104909F0DBFE41F2326005F0E1F94146404601230C4A04F045FF5FFA80F8C7E62A
:203AA0006C462046094958E66C4602460B462046004993E660F10008DCF400086F12833A7C
:203AC00020F200082CF2000828F2000834F2000810B5254C86B0204608F058FA234B93F940
:203AE0001530002B0BDBFDF757FA1F4808F07EFA2268D36843F04103D36006B010BD00233F
:203B00001B4903934FF6FF720293CDE904330093C4E9013323610193204680232160E2601B
:203B2000A36108F0D5F910B1124B01221A7000234FF4005202A90C48CDE90223CDE9043371
:203B400008F004FD10B10B4B01221A70002369460548CDE9003308F0CDFE0028C5D0054BD0
:203B600001221A70C1E700BFF01C0020C823002000040040C922002070B54FF080432DED6A
:203B8000028B1A69500600F18B80614A1388614D614C9BB213B92B60236000BF28685F4EFF
:203BA000FCF7B8FC58A3D3E90023FCF72DFDFDF723F85B4A08EE100A20682B6882ED008A8F
:203BC000C01AFCF7A7FC50A3D3E90023FCF71CFDFDF712F8236830601846FCF79BFC4AA3A9
:203BE000D3E90023FCF710FDFDF706F807EE900A4C4BF5EE407AF1EE10FA186059D0DFEDDB
:203C00004A6A9FED4A7A28EE268AC7EE276A88EE277A474B474848491A7880ED007AC1EDA4
:203C2000006A002A51D00020444A4549187010680B68444C1B1A002BB8BF5B4242F20F7069
:203C400083423BDC404B15681068404A186010781A680D6002FB00F23D481A6019680078A8
:203C600091FBF0F200FB12123A493B4DD2B20A7019686A7D91FBF0F13848196019680160FE
:203C8000C2F3411200212170D10732D4920735D41B68F3B9BDEC028B314B00221A6070BD40
:203CA00019691B4A21F0400143F69820196110806CE79FED2C7AF0EE476AAAE72378012B64
:203CC000C0D85A1C2270204BE2E71F4B1B68002BE0D0FDF7CDFE07EE900ADFED146A204B45
:203CE000B8EEE77ABDEC028BC6EE877AC3ED007A70BD1A686968521A1A60C9E71A6869683F
:203D00000A441A60C4E700BF198661188661883FDA240020E0190020A01C0020041B002059
:203D20003C240020F42300200000C84200247449981A0020E0240020E4240020081C00207F
:203D4000F4170020E1170020981C0020DE240020E9240020EA240020C8230020081B002081
:203D6000EC2300200000000070B5032803D8DFE800F0023A1F57384808F008F9FDF75EF9BC
:203D8000354808F033F90021334808F09FF9334B334A344834494FF47A741C6042F63C053C
:203DA000012342F20F74D562546303700B7070BD29482A4C2D4D08F0E9F8FDF73FF926484B
:203DC00008F014F90021244808F080F9244B28492448254A2560D962264D5D630124642188
:203DE0000470117070BD1C481C4C08F0CFF8FDF725F9194808F0FAF80021174808F066F9E2
:203E0000174B1848184A642540F214512560D96240F2E7350A2401215D630470117070BD1E
:203E20000D480E4C144D08F0B1F8FDF707F90A4808F0DCF80021084808F048F9084B0F496A
:203E40000848094A42F210762660D96201240A215D630470117070BDA81C00202C250020BD
:203E6000000C0040DE240020E9240020A08601006C430F003F420F009F860100CC870100B8
:203E80000D4B93F91530002B00DB70470B4A137803F0FF01002BF8D130B40948094C642364
:203EA0001370436A2588084A43EA054313602180416200BF30BC7047C8230020C023002037
:203EC000000400400C000020C022002070B5554C94F91430092B86B001D006B070BD524D1C
:203EE000524A2B78117899420AD02B78DBB2022B13702AD04E4A1278012A01D1180622D438
:203F000094F91530002BE8DA00BF494B1B78002B3AD1484948480A79047802F001029442DB
:203F2000DBD00A790979C2F300020270CA07D4D5424943484A6A0588424C42EA0542226054
:203F400003804B62C9E7D907DAD5637D3E4EC3F3C01282F0010262F3C7133046637508F014
:203F600015F894F91530002B28DBFDF715F8364808F03CF832683549D36842F2107043F04F
:203F80004103D3600880BBE7314B2A7819789142A3D02A781A7000BF1B78802B01D0012B65
:203FA0009BD100BF254A2648536A0188254C43EA014300212360018051628EE700231F49F9
:203FC0000093CDE90233CDE90433C6E90133336101934FF6FF72802330463160F260B361A5
:203FE00007F076FF10B11B4B01221A7000234FF4005202A914480292CDE90333059308F0B2
:020000040800F2
:20400000A5FA10B1134B01221A70002369460E48CDE9003308F06EFC0028A8D00D4B0122A7
:204020001A70A4E7C8230020F4190020FA1700203C060020901C0020FD170020000400405C
:204040000C000020C0220020F01C00202A000020FB170020C92200202DE9F04FDFF8FC90C7
:20406000DFF8FCA037493848BBB000250A23192289F8005008F022FDDAE9006704F0A4FF2C
:20408000002856D0314CDFF8DCB00DF1200899F8003021684BF833100BEBC30362685A60BC
:2040A0002B4807F095FBDAE90001801BE679617906900596E0782679A7790391A17863789E
:2040C00022780091CDE9010622490497404609F0B5FB4046FCF784F80A2382B241461A4884
:2040E00008F0ECFC237801352D2BEDB207D199F800300133DBB2092B89F800301FD8DAE91F
:20410000006704F07FFF0028C1D199F800302A461149404609F092FB4046FCF761F841461C
:2041200082B20A23084808F0C9FC00BF3BB0BDE8F08F99F8003002460DF12008E8E72A46D5
:20414000E6E700BF68FA00089824002038250020A41B002084FA0008C4FA0008E8240020B9
:2041600090240020B41B00202DE9F04182B000BF6B4F6C495C220023009218463A4605F0CF
:2041800095F800286DD000BF0422B818664909F08DFB002868D100BF644C654EDFF8C4C169
:2041A0000FCC35460FC594E80F0085E80F0030461C2250F8043BCCF80030114603F04CFD0C
:2041C0005C4B186000BF1B6832689A4235D000BF0A231A2258495948DFF87C81103408F089
:2041E0006DFC0FCCB446ACE80F0094E80F0098F80040DFF874C185E80F001C223368CCF85E
:204200000030A5F10C0044F00804114688F8004003F022FD4A4B186000BF1B6832689A429E
:204220004FD100BF7B6947484749002201337B6102800A7000BF022006E00A2312224349BA
:204240003E4808F03BFC012000BF414A737D12786FF30413012A737503D1DBB26FF3010371
:20426000737502B0BDE8F081314E3A4933483A4C344D0A231F2208F021FC0A231E2237499A
:204280002E4808F01BFC727D2078397E002302F0E00263F3461272754FF40042F2822A4A62
:2042A000337540F0040041F00201C6E90133C6E9033320702B801370397600BF00BF00BF7C
:2042C00069E700BF0A23222225491C481D4C08F0F5FB0A231E222149184808F0EFFB98F892
:2042E0000030727D397E184843F0040388F8003002F0E002002341F0020163F346124FF482
:2043000000457275C6E90133C6E903333375F58239762380037000BF00BF032094E700BFEA
:20432000F8190020B41B0020CCF90008141A0020C823002078230020F4F9000898240020AB
:20434000A01A00202A0000208824002034FA00083C060020D4F90008CC2200208CF200086C
:2043600010FA000830250020341D00202DE9F04F89B092469B46884604F06AFD04F076FD6E
:20438000064604F079FD011D4046CFB2CDF81880FBF726FF04465046FBF722FF05465846F2
:2043A000FBF71EFFAC4238BF2C46844238BF0446023404FB06F404EBD47358100397C0F178
:2043C0004000BDF80C90079382B2A2F1040801250027A4B20FFA88F84FEA890104922346F1
:2043E00005910A464046CDE90075102104F012FB059A2346CDE900574046102104F00AFB2F
:2044000023464046CDE900550822102104F002FB0499039A0C44A4B2A4F1090022FA05F3C4
:20442000CDE90075C6F34702122100B204F0F2FAC9F57F40FC3020444A463B46102100B289
:2044400004F080FADDF818800499079B404601EB6304FBF7C5FEA4B206FB00F0A4EB50008E
:204460003B464246102100B204F05CFA5046FBF7B7FE00FB06F0A4EB500009F11401524652
:204480002B4600B204F04EFA5846FBF7A9FE039A00FB06F0A4EB500002F10A0100B2A94080
:2044A0002B465A4609B0BDE8F04F04F03BBA00BF2DE9F0432DED028B04468BB003F012FF2D
:2044C0000A2C00F23F82DFE814F04F0020015A019E016903DA03E901FE01160289020B00DE
:2044E000CA4D297811F0010440F05084C849C9480A2209F0EDF9C84B4FF04032C3E900223B
:2045000041F2326004F0A4FC0123C44A2146204604F008FA40F2057004F09AFC287810F07C
:2045200001004FF0010300F05885BD4ABD4EBE4C2021002004F0F6F9BC4BDFEDBD7A93ED80
:20454000007A67EE277A17EE900AFCF705F802460B46B848B84909F071F90123B54A2821F3
:20456000002004F0DFF920E1B44B1A684CF24F339A4200F3C384B24BB24893ED000AFEF781
:20458000B7FB04B240F2057004F062FC20460123AD4A002104F0C6F902AD40F2057004F01B
:2045A00057FCAA4BAA4A93ED008A20210123002004F0B8F9DFEDA77AB4EEE78AF1EE10FAA2
:2045C000064618EE100A80F26A85FBF7C5FFDFEDA27AB4EEE78AF1EE10FA02460B4680F269
:2045E0001786F7EE007AB4EEE78AF1EE10FAC0F24E869A49284609F021F9F0B201232A46A3
:20460000202104F08FF9964B964A93ED008A28210123002004F086F9DFED8E7AB4EEE78A2B
:20462000F1EE10FA064618EE100A80F22985FBF793FFDFED897AB4EEE78AF1EE10FA02466E
:204640000B4680F2F285F7EE007AB4EEE78AF1EE10FAC0F204868149284609F0EFF8F0B2CF
:2046600001232A46282104F05DF97F4B7F4A93ED008A30210123002004F054F9DFED757AE5
:20468000B4EEE78AF1EE10FA064618EE100A80F21585FBF761FFDFED707AB4EEE78AF1EEAC
:2046A00010FA02460B4680F2CD85F7EE007AB4EEE78AF1EE10FAC0F2DE856849284609F00B
:2046C000BDF82A46F0B20123302104F02BF9684B544E18684D4DFBF73FFF02460B465548B1
:2046E000644909F0ABF80123524A3821002004F019F941F2166004F0ABFB204601235E4ABD
:20470000494C102104F00EF94FE04C4B1A684CF24F339A4200F31784534B4A4893ED000AAC
:20472000002241F23261FEF7CFFF04B241F2166004F08EFB0123514A1021204604F0F2F8BE
:2047400040F2057004F084FB01234D4A2046002104F0E8F84B4B1A68B2F57A7F00F2F78503
:2047600000F03A8602AD2846474909F067F82A4620460123082104F0D5F800F002BC334B74
:20478000424893ED000A274E274C204D002241F23261FEF799FFFDF76BF9294B024693EDA7
:2047A000000A28210020FDF79FFC327894F91430012A00F0D080002B00F06F82052B00F0E5
:2047C0006C82A38A23F4FE43092B00F0668241F2166004F03DFB2E4B1B889BB2002B40F0C1
:2047E0008F822B78DB0700F17E822A4B1B889BB2002B40F06E82012003F0F2FC0BB0BDEC1C
:20480000028BBDE8F083164B2348BAE7401D002084F90008E8190020040000207CF90008C2
:2048200090F900083C060020C82300209C1A00200000C8422418002094F90008081B002066
:20484000E4240020C0F60008F8F800083C24002000F900080024744900007A4474F20008EC
:20486000041B002004F90008F423002008F90008E024002010F9000820F9000828F9000835
:20488000F0F800082C2500200CF2000830F90008EC1C00209C1C002038F90008A74BA84865
:2048A00093ED000AA74EA84CFEF722FA054640F2057004F0CDFA28B20123A44AA44D0021C9
:2048C00004F030F871E7A34B9D4893ED000A9D4E9D4C002241F23261FEF7F6FE054640F2E5
:2048E000057004F0B5FA28B201239B4A984D002104F018F859E7994B914893ED000A00220A
:2049000041F23261FEF7E0FE04B240F2057004F09FFA8E4A20460123002104F003F8904BC7
:204920001A68B2F57A7F00F23C8300F05E8302AD28468C4908F082FF2A4620460123082145
:2049400003F0F0FF7F4E804C3278814D94F91430012A7FF430AF3BB1052B05D0A38A23F4E1
:20496000FE43092B7FF433AF637DC3F341139A0700F1D881002B3FF42AAF00BF40F20570FB
:2049800004F066FA784B1A684CF24F339A4200F399814FF0FF3005F0EDF9744BD3E90067AA
:2049A0004FF0FF3005F0D8F9304639464FF47A720023FCF771F900214FF4FA70994208BFAF
:2049C000904280F07F8194F91400002840F07A810123674A192103F0A5FFF8E65A4C94F9EA
:2049E0001530002BC0F20E83DFF8AC8198F80030002B00F0D48200225E4B88F800205E4EB8
:204A00001B685E4A3360336812785D495D48097803FB02F33360326892FBF1F301FB132324
:204A2000627DDBB20370C2F34113D807326892FBF1F2326000F16384990703D53368A2681E
:204A4000134433603E493068FDF7D2FB07B240F2057004F0FDF901233F4A3846002103F003
:204A600061FF3F4B1A68B2F57A7F00F21C8400F08B8402AD28463B4908F0E0FE01232A468E
:204A80000821384603F04EFF41F2166004F0E0F901233D4A1021384603F044FF41F2166080
:204AA00004F0D6F90123394A1021384603F03AFF40F2057004F0CCF998F800302BB3002291
:204AC0002C4B88F800201B682C4A3360336812782B492C48097803FB02F33360326892FBF8
:204AE000F1F301FB1323627DDBB20370C2F34113326892FBF1F23260DA0700F106849F071A
:204B000003D53368A268134433603068002840F0278301231E4A302103F004FF0022064653
:204B200000231C49284608F089FE2A46F0B20123302103F0F7FE034E054D36E6E4240020AA
:204B4000C0F600083C060020C8230020F8F80008401D0020F4230020F0F80008EC2300205F
:204B60002C2500200CF20008081B002090240020BCF90008E81C0020C4220020DE2400209E
:204B8000E9240020DF24002068F9000870F9000808F9000880F2000834250020834B844E4F
:204BA0001868844CFBF7D8FC377802460B46002F00F02E818049204608F040FE2046FDF70A
:204BC000D9F921460A22C5B27C4808F081FE7C4B22780021C3E9001152B12D3AD2B24F2A18
:204BE0009CBF7849895C62781970002A40F02F81EA0903D01A7862F07F021A706F0603D545
:204C00005A7862F07F025A70AC0603D59A7862F07F029A70E80603D5DA7862F07F02DA7077
:204C2000290703D51A7962F07F021A716A0703D55A7962F07F025A71AF0703D59A7962F0CE
:204C40007F029A71EC0703D5DA7962F07F02DA7141F2326004F0FCF80021084601235A4AA8
:204C60005A4C5B4D03F05EFEFCF702FF594B024693ED000A28210020FDF736FA95E5FCF733
:204C8000F7FE5549FDF7B4FA04B240F2057004F0DFF820460123514A3EE6637D13F0600F1C
:204CA0003FF495AD00BF4E4B1A684CF24F339A424C4A32DC94F91410137879BB63F03F0360
:204CC000137084E500231846474A192103F02AFE7DE5464BA3F11402A3F1280133F82A0CC6
:204CE000FFF744FB87E5424B42491A78314808F0A5FD01232F4A3021622003F013FE74E589
:204D000094F914203C492B4808F098FD0123294A00216C2003F006FE63E5137803F03F030A
:204D2000137054E500BF40F2057004F091F82C4B1A684CF24F339A4221DC4FF0FF3005F0DF
:204D400019F82E4BD3E900674FF0FF3005F004F8304639464FF47A720023FBF79DFF002151
:204D60004FF4FA70994208BF904208D294F9140028B90123224A192103F0D4FD27E50023F9
:204D800018461F4A192103F0CDFD20E51D4BDFED1E7A93ED000A1D4820EE270A082241F2F9
:204DA0001661FEF791FCFFF7B5BB00BFE02400203C0600202418002044F90008E81900208D
:204DC00004000020B0F000083CF90008C8230020401D0020E4240020C0F60008F0F800086C
:204DE000081B0020B01B0020BCF900081625002040240020C8F90008C4F900089024002087
:204E0000B4F900089C1A00200000C8427CF90008B549204608F012FD2046FDF7ABF80A22EC
:204E20002146C5B2B14808F053FDB14B2278C3E90077002A3FF4DCAE2D3AD2B24F2A9CBFF4
:204E4000AC498F5C62781F70002A3FF4D1AE2D3AD2B24F2A9CBFA749895CA27888BF002117
:204E60005970002A3FF4C4AE2D3AD2B24F2A9CBFA049895CE27888BF00219970002A3FF4E5
:204E8000B7AE2D3AD2B24F2A9CBF9A49895C227988BF0021D970002A3FF4AAAE2D3AD2B23A
:204EA0004F2A9CBF9349895C627988BF00211971002A3FF49DAE2D3AD2B24F2A9CBF8D4953
:204EC000895CA27988BF00215971002A3FF490AE2D3AD2B24F2A9CBF8649895CE27988BFF0
:204EE00000219971002A3FF483AE2D3AD2B24F2A00F2F3807F498A5CDA7179E6FCF7B8FD30
:204F00007D49FDF775F904B240F2057003F0A0FF01237A4A2046002103F004FD784B1A68D2
:204F2000B2F57A7F00F2F78100F0498202AD2846744908F083FC01232A460821204603F045
:204F4000F1FCFFF72ABB704B6B4893ED000A002241F23261FEF7B8FB04B241F2166003F0AF
:204F600077FF0123694A1021204603F0DBFC40F2057003F06DFF20460123654A002103F030
:204F8000D1FCFCF775FD634B634E93ED000A634C634D024628210020FDF7A6F805E4614EBC
:204FA00050E5614B614F5D6A614B624E6249A7FB05C08009A3FB00C3DB0803EB8303A6FB49
:204FC0000556A0EB4300A7FB027202AD00909209730B284608F032FCAEE4584A4E4E4F4C3B
:204FE000202103F09FFCFFF7E0BB4F4B4F4A5B6A5349A2FB032302AD9B092846012208F01E
:205000001DFC99E44F4E504D736A28883A4943EA0040FDF793FD40F2057003F019FF40F2DB
:20502000057003F015FF726A2B88716A2D883F48394E41EA054142EA0342A0FB01539B0952
:20504000A0FB02024FF47A7000FB131392093F493F48334D08F0F2FB01233D4A2021002048
:2050600003F060FC3B4B3C491A68394808F0E6FB0123374A2821002003F054FCFFF795BB63
:20508000FBF76AFA16A3D3E90023FBF7BDFA02460B462846314908F0D1FBFFF7E0BAFBF7B2
:2050A0005BFA0FA3D3E90023FBF7AEFA02460B4628462A4908F0C2FBFFF79FBAFBF74CFABA
:2050C00007A3D3E90023FBF79FFA02460B462846224908F0B3FBFFF7F4BA0022DA7187E527
:2050E0008DEDB5A0F7C6B03E40F20008E819002004000020B0F00008C0F60008F0F8000861
:205100002C2500200CF20008EC23002028F90008F8F80008E42400203C060020C823002033
:20512000401D0020C4220020000C0040D34D6210CDCCCCCC5917B7D1E8F10008A8F900085B
:20514000FCF10008000400400C0000204CF9000824180020C02200205CF9000860F2000888
:2051600098F800302BB30022AD4B88F800201B68AC4A336033681278AB49AC48097803FB3F
:2051800002F33360326892FBF1F301FB1323627DDBB20370C2F34113D807326892FBF1F279
:2051A000326000F12781990703D53368A26813443360D6ED007ADFED9E8A9E4AF8EE677ADD
:2051C000012388EEA78A3021002003F0ABFB064618EE100AFBF7C0F9B4EEE88AF1EE10FAE6
:2051E00002460B467FDADFED947AB4EEE78AF1EE10FA80F2D780F7EE007AB4EEE78AF1EECD
:2052000010FAC0F2FC808D49284608F017FB8CE47FA3D3E90023FBF7F7F902460B462846AE
:20522000874908F00BFBFFF7E8B979A3D3E90023FBF7EAF902460B462846814908F0FEFA78
:20524000FFF70DBA72A3D3E90023FBF7DDF902460B4628467A4908F0F1FAFFF732BA002224
:20526000784BFBF7D1F902460B462846764908F0E5FAFFF7F4B90022724BFBF7C5F9024698
:205280000B462846704908F0D9FAFFF71ABA00226C4BFBF7B9F902460B4628466A4908F0D2
:2052A000CDFAFFF7AAB9694BDFF8B0C15D6A684BDFF8ACE16749ACFB05908009A3FB00934E
:2052C000DB0803EB8303AEFB055EA0EB4300ACFB02C202AD009092094FEA5E33284608F028
:2052E000ADFAFFF7CBBB4CA3D3E90023FBF78CF902460B462846584908F0A0FA15E4336878
:20530000A2689B1A3360FFF79DBB3368A2689B1A3360FFF7FABB4D4B504E5D6A4C4B504F22
:205320004C49A6FB05C08009A3FB00C3DB0803EB8303A7FB0557A0EB4300A6FB026202ADB1
:20534000009092097B0B284608F078FAF3E53F4B424E5D6A3E4B424F3E49A6FB05C080097B
:20536000A3FB00C3DB0803EB8303A7FB0557A0EB4300A6FB026202AD009092097B0B2846D6
:2053800008F05CFAFFF7F3B9304B344A5B6A3549A2FB032302AD9B092846012208F04EFAFA
:2053A000FFF76CBB1AA3D3E90023FBF72DF902460B462846224908F041FAFFF7B6BB234BA2
:2053C000264A5B6A2749A2FB032302AD9B092846012208F033FAAEE51C4B204A5B6A2149C9
:2053E000A2FB032302AD9B092846012208F026FAFFF7BDB93368A2689B1A3360D9E60022B4
:20540000104BFBF701F902460B46FFF78ABB00BFFCA9F1D24D62503F8DEDB5A0F7C6B03E92
:20542000E81C0020DE240020E9240020DF2400200024744908F9000800007A4474F20008C0
:2054400068F2000800408F4080F20008000C0040CDCCCCCCE8F1000860F20008D34D621017
:205460005917B7D1FCF1000830B5002399B0CDE90E33CDE90333CDE90533CDE90833CDE976
:205480000A3329490093109302930793086C274A40F080500864096C01F080510091009946
:2054A0000193136823F4404343F400431360136803F4404301934FF4803109234FF48000EA
:2054C00002220C930D9104231390012454210CA8019DCDE91142CDE91431CDE9162306F0CC
:2054E0007DF908B1124B1C700222002311460F24039202A84FF4805202940493CDE9052364
:2055000006F080FB10B10A4B01221A7002224FF4007307A807920A9306F032FC10B1044B64
:2055200001221A7019B030BD0038024000700040C9220020000000002DE9F04F2DED028BD7
:20554000D1B000BFB14BB24D9A68B24942F480529A605A6842F007025A60DA6842F00102E3
:20556000DA609A6842F001029A609A6842F002029A609A6842F004029A609A6842F008021C
:205580009A60DA6842F48032DA60DA6842F40032DA60DA6842F48022DA60281D042208F012
:2055A00085F9002840F08585AB6801339A4AAB60536F980000F17585984B0993964B5B6F66
:2055C000190104D5099A137843F002031370924A099B1978536F43F080735367CA0702D594
:2055E000EB680133EB6000BF00240DF1780B04F02DFBFFF739FFCBE90144CBE90344864E63
:2056000012941E94336B864843F004033363336B03F004031293129B1394336B43F0800311
:205620003363336B03F080031393139B1494336B43F001033363336B03F001031493149B6E
:205640001594336B43F002033363336B03F002031593159B1694336B43F008033363336B8D
:2056600003F008032246169348F6F031169B04F0B5FE012202216B4804F0B0FE22464FF41E
:205680000B61684804F0AAFE22464FF23741664804F0A4FE012746F2070359466048209785
:2056A000CDE91E3404F02CFD48F6F03359465C4821944FF00208CDE91F741E9304F020FD18
:2056C000082359465648CDF88080CDE91E344FF0110904F015FD59465248CDF87880CDE98A
:2056E0002074CDF87C9004F00BFDB02359464D482194CDE91F741E9304F002FD4FF23743E5
:20570000594649482194CDE91F741E9304F0F8FC4FF40063594643482194CDE91F941E9323
:2057200004F0EEFC414B3E4820974FF480525946CDE91E2304F0E4FC22460421282004F07A
:20574000D5FA282004F008FB1194336B43F400133363336B03F400132246042111934846B1
:20576000119B04F0C3FA484604F0F6FA224604212F2004F0BBFA2F2004F0EEFA2C4B2D49BD
:20578000C3F8048040F6FF72184619609A6005F0FBFF294C00B127702849294B0B604FF611
:2057A000FF738022CB60084600238A614B601A9317931E93CBE90133CBE90333CBE90533DD
:2057C0008B600B61CDE91B331D93189306F080FB08B1012323704FF480531AA917481A934D
:2057E00006F0B4FE08B101232370144806F010FC08B101232370002317A91048CDE9173388
:2058000007F078F8F0B1012323701BE0002004E00C060020CCF9000800380240CC22002043
:2058200000080240000002400004024000002110A41B002000300040C9220020581A002079
:20584000000800400023602041F270761E901A465946B048209322931F9606F079FD08B15D
:20586000012323704EF6602304225946A9481F9306F06EFD08B101232370A64801F06AFF29
:20588000A54BA649A64A19605A604FF48041002218461961C3E90222C3E90522C3E9072290
:2058A00004F0D4FE08B101232370FBF7C7FB9D499D4B0B604FF6FF738022CB6008460023D0
:2058C0008A614B60CDE91A33CDE91C331E93CBE90133CBE90333CDE917338B60C1E90433DB
:2058E00006F0F6FA08B10123237000234FF400521AA98C481A92CDE91B331D9306F026FE89
:2059000008B1012323700521002350221E9185481F9259462093229306F0BEFE08B1012399
:205920002370002317A97F48CDE9173306F0E2FF08B1012323707D4B7D4A1A604FF4612214
:205940000C215A60184600225961C3E902221A61C3E9062207F010F808B101232370754BD8
:20596000754A1A604FF416520C215A60184600225961C3E902221A61C3E9062206F0FCFF12
:2059800008B101232370FBF707FB6C4A00234FF080411046C2E900131E93CBE90133CBE969
:2059A0000333CDE91A33CDE91C33CDE91733C2E902331361936106F0AFFB08B10123237051
:2059C0000421002350221E915C481F925946CDE92033229306F060FE08B1012323700023C5
:2059E00001261A461AA955481A93CDE91C331B9606F0F0FB00B12670022304221AA94F4890
:205A0000CDE91A3306F0E6FB08B101232370002317A94A48CDE9173306F06CFF08B1012389
:205A20002370DFF82091464BC9F8003048460023C9F804301E93CBE90133CBF80C30C9E9D9
:205A40000233C9F81030C9F8183006F041FA08B1012323703B4806F05FFB08B10123237023
:205A6000002301261A46594636481E93CDE920331F9606F0AFFB00B12670334B334A1A6094
:205A800053204FF6FF7280215860DA601846002299619A601A6106F01BFA002801F076843D
:205AA0000123237000BFFBF7ABFB294B29491B684FF0006252F8040B8A420344FAD124482B
:205AC000254A264903600A601368254A254813602021012204F082FC4FF48041224804F019
:205AE00077FC002801F0F783204B0C932048FCF789F80C9B1B78002B41F0E5831D4B1E4AEC
:205B00001E49584607F09AFE114E154F5846FCF779F835E0581A00200C1B002000540040AA
:205B2000801A0600FC2300200000014098240020004400403823002000100140482400208D
:205B40000048014080230020601B002000440140100000208038010840580108E41700202C
:205B6000B816002000040240000802403C060020ACF20008E0F20008ECF20008F8F20008ED
:205B800032683B689A4201F09683AC49AC4C584607F054FE5846FCF735F8D5E902133268E3
:205BA00038680B44134421682A6903440B44134418462B6107F0EAFD00BF07F00BFEA14A24
:205BC000A1490D9182FB0032C317C3EB2213322202FB13030B600A682B610F320A600A68E4
:205BE0004FF47A7303FB02F30B6000BF099B97491878D5E90223C0F3400500F00100CDE9C2
:205C00000005584607F01AFE5846FBF7FBFF9048FBF7F8FF0C9B1B78002B01F04783012B3B
:205C20000CBF8C488C48FBF7EDFF8C4806F0CCF9FEF712FA00BF8023894E0093012500236E
:205C40001846884A8849357003F030FB874A8649002003F075FBFEF787FA024620B9099924
:205C60000B7843F010030B70099B1B78DB0701F115837F4B0F931846C368DFF83882013383
:205C8000C3607C4B0021A8F80010197000BF0169C36800915846784907F0D0FD5846FBF728
:205CA000B1FF099B1B78DF0602D57448FBF7AAFF6B4F6E4A6C490025082600962B462846FB
:205CC0003D7003F0F3FA00BF012328463B7003F0E3FA00962B462846644A634903F0E6FAC9
:205CE00000BF00BF664806F081F92946644806F0EDF9634BE18A1A680C9B51631B78002B5D
:205D000041F0C7825F48FCF737F8099B1B7813F0100501F0A7825C4B9878D9781A791E78A6
:205D20005D7860F07F0061F07F0162F07F029870D970587999791A71DA7966F07F0665F0D9
:205D40007F0560F07F0061F07F0162F07F021E705D7058719971DA710C9B1D78012D01F078
:205D60004E824021012001F08FFF322003F09AFF41F2326003F06CF8099B1B7803F00C0220
:205D8000042A01F034821F0707D50021012308463E4A02F0C7FD099B1B785E0705D50021C4
:205DA000084601233A4A02F0BDFD012002F018FA607D384F384EDFF800A100F00300FDF7D3
:205DC000D3FF364B1A681846D36843F04103D36006F00CF9324806F0F7F84FF08043012529
:205DE0004FF0FF3C31214FF0540E002240F20120C3F82CC09A6298611962C3F808E01D608A
:205E0000FDF766FE274806F0F1F8274BD9F800C09D614FF6FF7200201D629862DA621D60D3
:205E2000DCF80C302149224843F003032A46CCF80C3006F0F3FEA14600E100BF60F300080C
:205E4000C82300201F85EB51200000208CF30008BCF30008D8F30008E8F30008601B002088
:205E60004E25002048170020B41B0020C8170020F819002088240020F8F3000828F400080E
:205E8000581A002050F400080400002060F400086CF400080C1C0020901C0020FC230020E9
:205EA000482400208023002000480140D8240020382300202A0000200008024001239340E8
:205EC00040F23112134240F0178113F0CE0F40F088849D0540F1CC8099F91530002B80F281
:205EE0000B81099B1B78DC0640F1CB80A14B1B680A9323B9099B1B78980600F1AE810D9BFC
:205F00001B68C3B99C4B1A689C4B1B689A4212D09B49584607F092FC5846FAF761F90A23D4
:205F200082B25946974806F0C9FD0A2003F0BAFE00BFFBF765F9FDF7C9FF3368032B02DCAC
:205F4000336803331ADA326899F81430002AB8BF033203EBA2035BB2002BC0F2B1800A2B54
:205F6000C8BF002389F81430002342F210723360A8F80020844A4FF4FA63138083498448ED
:205F80000B7802789A4243D00B78DBB2202B037000F09A80082B40F0BB8099F81520C2F324
:205FA0008103013303F00303032B00F0248463F383020021012B89F81520ADF8801000F067
:205FC0004084022B40F01E84724B93E807005B4603C31A70704940F6B83040F20573142217
:205FE0006E4C20806E48841E20F8023C07F070FC14226C4904F1160007F06AFC142259460E
:020000040800F2
:2060000004F12A0007F064FC42F21073A8F8003065490C88A4B25CB999F815306422DD0697
:206020000A8040F155810C9B1D78012D00F011845E4B1B889BB2002B00F0C4815C4805F04E
:20604000C7FB00224FF40061504604F0C7F930BF012250464FF4006104F0C0F9554B1C8831
:20606000A4B2002C76D099F81420092A7FF626AF3B7823F008033B70099B1B78DC063FF54D
:2060800035AF4D4B1C88A3B20A93002B00F08B83B8F800309BB2002B7FF428AFFBF72CF80D
:2060A00024E7464A0992137843F001031370FFF785BA434B6B600023EB600123FFF776BA1F
:2060C0000A2389F814304FE700BF0C9B1A7899F8143001335BB2002A40F0B9800A2B40F38F
:2060E000B98089F81420284A4FF4FA63138042F21073A8F800308BE74FF48071314804F073
:2061000067F93B780028B4D043F008033B70E8E6012B40F0F88699F9143043B1052B06D05F
:20612000B9F8143023F4FE43092B7FF471AF99F8153097F90020C3F3411181F0010060F3F8
:206140004613C90789F8153040F1B78322F040023A70CCE7174A1B484FF4FA7320211380EC
:2061600004F040F91848FAF73BF84B461A46A1462DE000BF2400002010000020B816002068
:2061800084F4000898240020EC1C0020F4190020FC1700209CF40008C0F400089C1C0020EF
:2061A000EE240020C0F600083023002028000020A41B0020F21900201C000020CC220020E0
:2061C000466D6574000002400C1E00200134E3B235498342194432D291F8C8102C29F5D1BD
:2061E00009F101095FFA89F9B9F1070FEED12E48991C0144054691F8C8000133303805EBA9
:20620000030E092805F1C80505EB030C00F24F8300BF9EF8C83091F8C810303B303903EB46
:20622000830301EB430321490B70214B0A92C3F800C000BF1F48F9F7D3FF0A9AC6E71C4B9E
:206240001B689146002B3FF40EAF00BF0BE7092BC8BF002389F8143045E7082300930A98E9
:20626000154B164C164D174918705A460346256003F01CF80E9000BF0F4B0A9801251D7090
:2062800003F00AF8284603F00DFD00BF0E9B2BB104220D491FA807F009FB18B10B4A0023DB
:2062A000137000BF00BF2AE6441D002040240020001800200C1E00204E250020240000206F
:2062C000E0930400B41B0020CCF9000818000020B14901224FF080430A80B0499A6B0A6042
:2062E0000A68AF490A60AF4A5B6B13601368AE4A136000BFFDF740FCAC484FF4007104F027
:2063000067F8AB4A1378834204D01070A94A4FF4FA631380A74B1B889BB2002B00F07A8266
:20632000A54B9FEDA68A1868FAF7F4F898A3D3E90023FAF769F9FAF75FFC07EE900A27EEF7
:20634000888AF7EE007A9FED9E7A9E4B77EEC87A186067EE877A9C4BBDEEE77A83ED008ADD
:2063600017EE100A994B0028C3ED007AB8BF4042FAF7E0F80022964BFAF7B8FB954A1378F5
:2063800028B1B5EE408AF1EE10FA40F056856FF300031370904B1B7823B1904B1B78002B00
:2063A00040F074848E4B1B889BB2002B7FF440AE99F81400FEF77CF88A4B1B889BB2002B62
:2063C0007FF43CAE884B87491B784FF496720A80002B40F02782854B93E80300844B83E8C9
:2063E00003000C9B1B78002B40F02482814B824A8249834807F022FA7D48F9F7F1FE7C4BB3
:206400007F49184407F03AFADFF850C2044665460FCDE3607B4B20609D426160A260AC4656
:2064200004F11004F3D1BCE80700BCF80030A381754B20606160A2601B78642B00F09384B0
:206440000A2B00F02383FBF713FB704A704913681468A4B202461B0C0094694807F0EEF91F
:206460006749634807F013FA99F91530002B80F25F83684B1A68B2F57A7F00F2EC8200F042
:20648000A78365495E4807F0D9F95D495848634D07F0FDF9624B1868FAF75EF802460B46C5
:2064A0005748604907F0CAF95549514807F0EFF95D4B1868FAF750F802460B4650485B498E
:2064C00007F0BCF94E494A4807F0E1F9584B1868FAF742F802460B464948564907F0AEF961
:2064E0004749434807F0D3F9534B1868FAF734F802460B464248514907F0A0F940493C4829
:2065000007F0C5F94E4B1868FAF726F802460B463B484C4907F092F93949354807F0B7F9C5
:20652000494B1868FAF718F802460B463448474907F084F932492E4807F0A9F9444B2C6880
:2065400015491A78304B09881B782D4800910134019440492C6007F071F92949244807F091
:2065600096F93D4B93E803001A4BADF860101B7817900022D907CDF8622000F14D8299F937
:206580001530002BC0F253826AE000BFAFF30080198661188661883FA41C002044240020AB
:2065A000E0190020541A0020A01C002000040240F9170020E41900203C1D0020BD3786359D
:2065C0000000C8427C230020C42300209C1A002000002440401D0020C8220020301D0020BD
:2065E0001A00002028000020E017002004F500080C070020E0F20008ECF200080CF5000805
:20660000881800209CF50008E9240020081C002048F600082C250020C4F60008AC16002055
:20662000F4230020D8F60008E4240020F0F60008EC23002008F700083C24002020F7000862
:20664000041B002038F70008E02400204CF70008DE24002060F7000898F000087CF50008CB
:206660000C9B1B78002B6BD1A24ACDF86E30A24BDFEDA27A1B7892E80300A14A1A9092ED31
:20668000007AADF86C10DA0767EE277A12D5BDEEE77A17EE103A1A1D082A40F2FF8303F135
:2066A0000902122A40F20F84002BB8BF5B42322B00F31184904B1B7817AA17EE900A03F0E9
:2066C000010306920793F9F747FFCDE904018D4B18681AAB0293F9F73FFF8B4B1A68CDE9A5
:2066E00000018A498A4807F0A9F88949894807F0CEF8894B93E80300884BCBF800001B8871
:20670000ADF87C100022B3F5617FCDF87E2000F27583824B1B889BB2002B40F09383B9F872
:2067200016207E4B7E491B880192A2F50042009277485A4607F082F87549764807F0A7F810
:20674000784B93E80300099B1A901B78ADF86C1000229B06CDF86E2000F15781099B3168DA
:206760001B7899F9142070480290C3F34013CDE9001267486D491AAA07F060F864496548D3
:2067800007F085F80C9B1C78002C00F0FB80684A604801231370F9F723FD5E4982B265481A
:2067A00006F01AFA4AE4644C6449624814250A230622258006F082F9614B1D78ED00EDB229
:2067C00000BF0F9A5F490A982B462A4403F014F900BF632D00F2E381594A1378013313709E
:2067E00056E44FF48051584803F0F2FD3B7800283FF43FAC88E46FF38302002389F81520A4
:20680000ADF88030514B93E807005B4603C31A70FFF7E0BB3A4A002313603A4A13604C4ADC
:206820001360B7E53B4A4B4B13600C9B1B78002B3FF4DCAD484B494A4949354806F0FEFF72
:20684000DAE5484B93E807005B4603C31A70FFF7C1BB00BF41F2166002F0FAFA4FF0FF3045
:2068600003F088FA404BD3E900234FF0FF30CDE90A2303F071FADDE90A23104619464FF49F
:206880007A720023FAF708FA002199424FF4FA7008BF904234BF23462B46344A10214020D8
:2068A00002F040F8012001F09BFCFFF7C1BB9EF8C8302F49303B0B70B7E42E4902F07F0222
:2068C0000968C9F8041042F040020121DBB261F346133A702849294A08681168284AC9F8F8
:2068E0000C00126889F81530C9F81010C9F80820FFF7FDBBA4F00008401D00200000C842B1
:206900009C1A0020C42300203C1D0020F8F70008881800200C070020F0F70008E41900202B
:2069200044F80008A8F70008E81900207CF80008E0170020982400201C00002048FA000856
:2069400088240020B41B002000000240B4F400087C2300201B5B7300E0F20008ECF2000822
:2069600044F50008A8F4000890240020FCF4000840240020081C002044240020541A002088
:20698000C422002002229849984806F0A1FF02229749984806F09CFF97499848022206F027
:2069A00097FF974BCDF87E4093E80300954BCBF800001B78ADF87C10042B00F24B82022BDC
:2069C00000F273828D4A0292033A0192033A8E4900928E485A4606F031FF8D48F9F700FC92
:2069E0008B4B8A49184406F049FF8A4A12780346002A40F00B82884A1068127918601A71EE
:206A00008649834806F043FFC1E67D4B93E803001A90ADF86C10A1E6814B93E8030099F989
:206A200015301790002BADF86010BFF619AE7D4B7D4C5A6A7D4B7E4918887E4B1B68248832
:206A4000009442EA0042714806F0F8FE6F49704806F01DFF04E6784B784C586A784B794D51
:206A6000A4FB00C18909A3FB01C3DB0803EB8303A4FB0242A1EB4301A5FB0040430B0091F9
:206A800092097149614806F0D9FEFEE4FAF7F0FF6E4A6F4B6F491B78156814682D0CA4B224
:206AA0000246CDE90054594806F0C8FE5749584806F0EDFE99F91530002BFFF6DAAC664AD9
:206AC000137843B300231370644B654C1B68654A236023681078644A03FB00F323602068BD
:206AE000117899F8152090FBF1F301FB13035F48DBB20370C2F34113226892FBF1F222609A
:206B0000DA0700F1F0819B0705D55549D9F808200B6813440B60524B55491A68534B1B78FC
:206B20003A4806F08BFE3949394806F0B0FEA0E4494A137843B300231370484B484C1B68C5
:206B4000484A236023681078474A03FB00F323602068117899F8152090FBF1F301FB1303B0
:206B60004248DBB20370C2F34113DD07226892FBF1F2226000F1A181980705D53849D9F844
:206B800008200B6813440B60354B3A491A681F4806F054FE1D491E4806F079FE69E40A9D37
:206BA000354A364980234FF6FF7000932B462080284602F07BFB0A2316223149314805F0B9
:206BC0007DFF099A137865F345131370FFF760BA194B1A4A5B6A2C490C48A2FB03239B090B
:206BE000012206F02BFE50E46B200020BC1600206D200020BF1600206F200020C216002039
:206C0000F0F7000840240020C0F80008881800200C070020E0170020E4F80008441D0020D2
:206C2000A8F7000800040040381D00200C000020B0F70008C0220020000C0040D34D621039
:206C4000CDCCCCCC5917B7D194F60008081C0020EA240020FCF5000834250020E81C002071
:206C6000C4220020DE240020E9240020DF24002030F6000878F60008C8160020B41B00200B
:206C800050FA000898240020ACF60008B24A0023137000BF4FF40071B04803F099FBB04A8E
:206CA0001378834204D01070AE4A4FF4FA631380AC4B1B889BB2002B00F0E580AA4B9FED1D
:206CC000AB8A1868F9F726FCA1A3D3E90023F9F79BFCF9F791FF07EE100A27EE088AB7EE68
:206CE000007A37EE487ADFEDA27AA24B67EE277A1860BDEEE77AA04B17EE100A83ED008AE0
:206D00009E4B0028C3ED007AB8BF4042F9F712FC00229B4BF9F7EAFE9A4A137828B1B5EE76
:206D2000408AF1EE10FA40F0E4806FF3000313708D4B954A1B68934200F2948000BF934B72
:206D40001988B9F816304FF6FF72501A834280F2A3800B449BB21A468D49A9F816300968F7
:206D60004A63FFF71FBBFAF783FE8A4A8A4B8B491B78156814682D0CA4B20246CDE900543A
:206D8000874806F05BFD8649864806F080FD99F91530002BFFF66DAB834A137843B3002346
:206DA0001370824B824C1B68824A236023681078814A03FB00F323602068117899F81520BA
:206DC00090FBF1F301FB13037C48DBB20370C2F34113D807226892FBF1F2226000F18D800C
:206DE000990705D57249D9F808200B6813440B606F4B73491A68714B1B7891E6714B93E83B
:206E00000300CBF80000ADF87C1088E46E4906F035FD6E4906F032FD6D4906F02FFD6D49C6
:206E200006F02CFD6C4906F029FD6C4906F026FD6B4A034610681860E2E543F00103137025
:206E4000FFF7A8BA674B93E80300CBF80000ADF87C1064E45B4A92E80300CBF80000ADF8E4
:206E60007C10AFE5404B604A1B6893427FF69AAA00BF464AB9F81630128893420BD99B1A5E
:206E80009BB21A4668E73D4A002313603A4A1360384A13604CE7002213465DE7494B93E8EC
:206EA00003001A90ADF86C1004E44E4A92E80300CBF80000ADF87C1084E52368D9F8082026
:206EC0009B1A236060E6494B93E803001A90ADF86C10FFF7EFBB464B93E803001A90ADF859
:206EE0006C10FFF7E7BB2368D9F808209B1A236011E643F0010313701AE72368D9F808208C
:206F00009B1A236074E7802B40F0908099F9143043B1052B06D0B9F8143023F4FE43092BA2
:206F20007FF476A899F8152097F90010C2F3411383F0020083F0030360F3461213F00203B0
:206F400089F8152056D101F07F013970FFF7CFB8198661188661883FC822002000040240A7
:206F6000F9170020E41900203C1D0020BD3786350000C8427C230020C42300209C1A0020F6
:206F800000002440401D0020FFBC010516000020581A0020081C0020EA240020ACF500086C
:206FA000881800200C07002034250020E81C0020C4220020DE240020E9240020DF240020C9
:206FC000E0F50008A8F700080C1E0020D41E00209C1F0020642000202C210020F4210020B0
:206FE000ECF8000898F0000800BD0105E8F70008F0F70008D2B263F34612C14B89F8152088
:207000001868C04BC9F8040021F040011B68C9F80C3061F07F013970BB4BBC4909681B68D5
:20702000C9F81010C9F80830FFF761B8102B4AD199F81530B6485C1C04F0030464F301036F
:20704000022C89F8153000F0B88000F29B80012C67D104F09BFFF9F7F1FFAD4804F0C6FF86
:207060000021AB4805F032F8AA48AB4B6421016040F2145240F2E731DA625963A74B1C70B7
:20708000A74B0A221A7099F8152002F003020023022ACDE91F33CDE921335ED06CD8012A8D
:2070A00062D0A04B93E803000B0CCBF80000ADF87C108DF87E3040F6B83040F205731422F9
:2070C0009949FEF78DBF402B14D199F815303A78C3F3001181F0010161F3041389F815304A
:2070E000DB064CBF42F0200302F0DF033B7000BFFEF78EBF042B7EF48BAF99F91530002BF2
:20710000FEF686AF99F9143023B9092389F81430FEF7EDBF092B04BF002389F81430FEF72E
:20712000E6BF04F033FFF9F789FF794804F05EFF0021774804F0CAFF7648774A4FF47A71B0
:20714000016042F63C0342F20F71D3625163744A01231370714A137095E7744B93E807005A
:207160005B4603C31A70A6E7714B93E80300CBF80000ADF87C109EE76E4B93E803008BE834
:20718000030098E704F002FFF9F758FF6048614C04F02CFF00215E4804F098FF5E4B664A12
:2071A000664942F210702060DA6259635C4901220A705A4A0A23137065E704F0E7FEF9F749
:2071C0003DFF534804F012FF0021514804F07EFF5048514B5A4901605A4A5B49DA62596330
:2071E0004F4901220A704D4A642313704BE7002108460123554A01F095FBFEF7D6BD20210B
:20720000284600F041FD524B022232201A7002F049FD01F067F841F2326001F019FE099B3C
:207220001A7812F00C0117D0110707D500212B46484A084601F076FB099B1A78530705D594
:20724000002108460123444A01F06CFB012000F0C7FF00BFFEF7ACBD2B46404A084601F087
:2072600061FBF3E741F2326001F0F2FD099B1B781E0705D529463748FAF7E4FD099B1B7806
:2072800058077EF569AD00213348FAF7DBFDFEF763BD3348FAF770FDFEF737BD31490F91B0
:2072A0000B6901330B610846FEF7E6BC2E48FAF7A9FCFEF7BABC2D4B2D482E4C0D93FAF766
:2072C000A1FCFEF793BC2C4B2C4A2D49584606F0B5FAFEF719BC2B4B2B480C9301224FF46F
:2072E00080411C4603F07AF8012002F0DBFC4FF48041254803F06CF801232370FEF7F6BBF7
:20730000081C002044240020C4220020541A0020A81C00202C250020000C0040E92400203F
:20732000DE240020D0F40008F4F40008E0F40008D8F40008ECF40008CC8701009F8601005D
:20734000A08601006C430F003F420F0050F40008B819002060F400086CF4000878F4000843
:207360005CF40008F8190020C8F300082000002078F30008C8230020E0F20008ECF2000843
:207380002CF300083C060020000802402378002B3EF48BABFEF786BB014B01221A70704706
:2073A000C922002010B582B0114B002400945A6C42F480425A645A6C02F480420092009A91
:2073C00001941A6C42F080521A641B6C03F0805301930420019B02F077FC22462146052016
:2073E00002F084FC052002B0BDE8104002F0B4BC00380240F0B502682E4B89B000249A42B2
:20740000CDE90344CDE90544079401D009B0F0BD294F01943B6B43F002033B633B6B03F07C
:20742000020301934FF4C073019A039312220123CDE9042303A90423032506461F48CDE973
:20744000065302F05DFE02943B6C1D4D1D48EC6043F400133B643B6C286003F40013029377
:207460004FF000714022029B6C614FF480632846C5E90644C5E90844C5E901122B6102F0CB
:20748000B9FC98B97563002204211F20AE6302F02DFC1F2002F060FC00220421202002F056
:2074A00025FC202002F058FC09B0F0BDFFF774FFE8E700BF00540040003802400004024074
:2074C000A41A0020B860024070B503687D4A90B000249342CDE90B44CDE90D440F9420D045
:2074E000794A93425FD0794A934200F09880784A934209D0774A934200F0CF80764A93424B
:2075000000F0A28010B070BD744B07941A6C42F008021A641B6C03F008030793079B10B051
:2075200070BD6E4B01945A6C6D4842F001025A645A6C02F001020192019A02941A6B42F02C
:2075400001021A631B6B03F00103022502930BA901234FF488520F93CDE90B25029E02F063
:20756000CFFD22462946182002F0C0FB182002F0F3FB22462946192002F0B8FB192002F08B
:20758000EBFB224629461A2002F0B0FB1A2002F0E3FB224629461B2002F0A8FB1B2002F079
:2075A000DBFB10B070BD4D4B03941A6C4C4842F002021A641A6C02F002020392039A0494C5
:2075C0001A6B42F001021A631A6B02F001020492049A05941A6B42F008021A631B6B03F076
:2075E0000803022505930BA94023059A0F95CDE90B3502F085FD04230BA93A480B930C9561
:207600000F95CDE90D4402F07BFD224603211D2002F06CFB1D2002F09FFB10B070BD2F4B03
:2076200006941A6C42F004021A641B6C03F004032246069304211E20069B02F057FB1E206C
:2076400002F08AFB10B070BD244B09945A6C264842F480225A645A6C02F480220992099A54
:207660000A941A6B42F002021A631B6B03F002030A930BA903234FF400720225CDE90B257D
:207680000F930A9E02F03CFD224629461A2002F02DFB1A2002F060FB34E7104B08945A6CEB
:2076A00042F400325A645B6C03F400330893224602211920089B02F019FB192002F04CFB39
:2076C00020E700BF000001400004004000080040000C004000440140004801400038024043
:2076E00000000240000C02400004024030B5026889B00023B2F1804FCDE90333CDE90533BD
:20770000079301D009B030BD02F50E320193116C0F4841F001011164116C01F0010101910F
:2077200001990293136B43F001031363136B03F0010302930222012303A94FF40044029DCB
:207740000793CDE9034202F0DBFC09B030BD00BF0000024010B502681D4988B000238A4268
:20776000CDE90333CDE9053307931AD019498A4201D008B010BD184A0293136B174843F020
:2077800001031363136B03F0010302930122022303A9029C0793CDE9032302F0B1FC08B006
:2077A00010BD0D4A0193136B0D4843F002031363136B03F0020301934022022303A9019CB6
:2077C0000793CDE9032302F09BFC08B010BD00BF00080040000C0040003802400000024016
:2077E0000004024008B5304A0368934223D02F4A934233D02E4A93424AD02E4A934206D0FE
:207800002D4A93423DD02D4A934207D008BD02F50B32136C23F00803136408BD02F5704271
:207820002748536C23F4802353644FF40071BDE8084002F03BBD02F59C322248536C23F01D
:20784000010353644FF4885102F030FD182002F091FA1B20BDE8084002F08CBA02F50D32E7
:207860001848136C23F002031364402102F01EFD1548042102F01AFD1D20BDE8084002F085
:2078800079BA02F57442536C23F40033536408BD02F50C321E20136C23F004031364BDE85B
:2078A000084002F067BA00BF000001400004004000080040000C0040004401400048014087
:2078C0000004024000000240000C024070B50368484A8AB000249342CDE90544CDE907447D
:2078E000099449D0444A934201D00AB070BD434B03941A6C424D42F400321A641A6C02F41B
:2079000000320392039A04941A6B42F001021A631B6B03F0010304930C230593022305A986
:2079200006934FF0030C072306463648049ACDE908C302F0E5FB344828604FF00061402275
:207940004FF480632846EC60C5E90544C5E907446C62C5E901122B6102F04CFA002845D1C6
:207960003563002204212620AE6302F0BFF9262002F0F2F90AB070BD204B01945A6C2148EE
:2079800042F010025A645A6C02F010020192019A02941A6B42F001021A631B6B03F00103A3
:2079A00002934FF40071122201230326029D0591072505A90692CDE90736099502F0A0FB38
:2079C000022305A94FF480620E480794CDE90523CDE9086502F094FB22460421252002F078
:2079E00085F9252002F0B8F90AB070BDFFF7D4FCB6E700BF001001400044004000380240C9
:207A0000D022002000000240A0600240704700BF08B5F9F7F5FBFEE708B5F9F7F1FBFEE75A
:207A2000FEE700BF08B5F9F7EBFBFEE7704700BF704700BF704700BF08B5F9F7F5FDBDE884
:207A4000084002F01DB900BF00BFF9F7D9BB00BF014802F07BBA00BFD0220020014804F0D7
:207A60009FBE00BFFC23002008B5094B1B681A69D20702D5DB68DB0707D4054804F090FE15
:207A80000448BDE8084004F08BBEFAF757F8F4E7FC230020601B0020144B1B681A695206BE
:207AA00010B502D5DB685C0618D4114C23681A69900702D5DA68910713D41A69D20702D5CC
:207AC000DB68DB0707D4094804F06AFE0848BDE8104004F065BEFAF76BF8F4E7F9F7A6FFD9
:207AE000E3E7FAF76DF82368E7E700BFFC23002080230020014804F053BE00BFFC23002000
:207B000010B50F4C23681A69D00702D5DA68D10711D41A69520602D5DB685B0604D408480C
:207B2000BDE8104004F03CBEFAF720F80448BDE8104004F035BEFAF709F82368E9E700BF25
:207B4000F01C0020014804F02BBE00BF581A0020014802F097BF00BF0C1B0020014803F0AF
:207B6000A5BC00BF0C1B0020014805F0BBB800BF38230020014805F0B5B800BF982400206D
:207B800008B5064B5B69DB0401D5FCF779F94FF48050BDE8084002F02FBC00BF003C0140E0
:207BA000014802F0D3B900BFA41A00200C4A08B5136833B118446946884208D8106018466C
:207BC00008BD084B1360184469468842F6D905F04FF90C2303604FF0FF33184608BD00BF54
:207BE000B419002058250020054BD3F888204FF0006142F47002C3F888209960704700BF1E
:207C000000ED00E0DFF834D0002103E00C4B5B58435004310B480C4B42189A42F6D30B4AE8
:207C200002E0002342F8043B094B9A42F9D3FFF7DBFF05F023F9FDF77FFC704700000120A2
:207C400010520108000000200C0600202006002058250020FEE7000081B110B4084C014410
:207C600010F8013B83EA1263884254F8233083EA0222F5D110465DF8044B70471046704760
:207C800050FB0008704700BF2DE9F0438FB0C54D0EABAE2203F81B2D2A7800930124022633
:207CA0008946234602FA04F18046002202960194BD4802F08BFD0EABD52203F81C2D297872
:207CC0000093A14023460022CDE90146B64802F07DFD0EAB802203F81D2D29780093A14089
:207CE00023460022CDE90146AF4802F06FFD0EABA82203F81E2D29780093A140234600223E
:207D0000CDE90146A84802F061FD0EAB3F2203F81F2D29780093A14023460022CDE9014628
:207D2000A14802F053FD0EABD32203F8202D29780093A14023460022CDE901469A4802F0B1
:207D400045FD0EAB002703F8217D29780093A14023463A46CDE90146934802F037FD0EABB3
:207D6000402203F8222D29780093A14023463A46CDE901468C4802F029FD0EAB8D2203F80D
:207D8000232D29780093A14023463A46CDE90146854802F01BFD0EAB142203F8242D2978E5
:207DA0000093A14023463A46CDE901467E4802F00DFD0EAB202203F8252D29780093A1404A
:207DC00023463A46CDE90146774802F0FFFC0EAB297803F8267DA14000933A462346CDE906
:207DE0000146714802F0F2FC0EABA12203F8272D29780093A14023463A46CDE901466A482B
:207E000002F0E4FC0EABC82203F8282D29780093CDE90146A14023463A46634802F0D6FC33
:207E2000B9F1200F00F0EE802978B9F1600F4FEA41010EAB4FF0DA0200F0BA8003F80F2DA1
:207E4000594800933A462346CDE9014602F0BEFC0EAB122203F8102D297800934900234651
:207E60003A46CDE90146504802F0B0FC0EAB812203F8112D29780093CDE9014623464900D7
:207E80003A46494802F0A2FC0EA8CF2300F8123D29780090CDE9014623463A464900424868
:207EA00002F094FC0EABD92203F8072D2978009301240226A14023460022CDE901463A48F1
:207EC00002F084FC0EABF12203F8082D29780093A14023460022CDE90146334802F076FCB8
:207EE0000EABDB2203F8092D29780093A14023460022CDE901462C4802F068FC0EAB402219
:207F000003F80A2D29780093A14023460022CDE90146254802F05AFC0EABA42203F80B2D2B
:207F200029780093A14023460022CDE901461E4802F04CFC0EABA62203F80C2D297800931B
:207F4000A14023460022CDE90146174802F03EFC0EAB2E2203F80D2D29780093A140234671
:207F60000022CDE90146104802F030FC0EABAF2203F80E2D29780093CDE901462346A14031
:207F80000022094802F022FCB8F1000F05D0074B93F80080B8F1000F6CD000BF0FB0BDE85D
:207FA000F08300BF310000200C1B0020B919002003F8132D654800933A462346CDE90146A4
:207FC00002F004FC0EAB297803F8146D490000933A462346CDE901465C4802F0F7FB0EABD6
:207FE000812203F8152D29780093CDE90146234649003A46554802F0E9FB0EA8AF2300F84B
:020000040800F2
:20800000163D45E70EABDA2203F8172D29780093A14023463A46CDE901464C4802F0D6FB9B
:208020000EAB297803F8186DA14000933A462346CDE90146454802F0C9FB0EAB812203F872
:20804000192D29780093A14023463A46CDE901463E4802F0BBFB0EA88F2300F81A3D297859
:208060000090CDE9014623463A46A140374802F0ADFB17E70EAB212203F8012D2978009339
:20808000CDE90146A140234642463048304F02F09DFB0EAB297803F8028DA140CDE90146CE
:2080A000424600932948234602F090FB0EAB7F2203F8032D29780093CDE90146A14023464E
:2080C0004246224802F082FB0EAB222203F8042D29780093CDE90146A140234642461B48B0
:2080E00002F074FB0EAB297803F8058DA140CDE90146424600931548234602F067FB0EA86F
:20810000072300F8063D297800901048CDE9014623464246A140814602F058FB07F58068B2
:208120000A264FF4807429780097CDE90146490007F5807701234022484602F047FBB84522
:20814000F1D100BF0FB0BDE8F08300BF0C1B00203400002083B27F2B28D830B48CB23F2C01
:2081600022D81D4D2D78022D27D0032D1FD0012D04D1C4F17F0501461C4628B20029B8BF52
:208180000731C910802504F0070311FB05000124124D04FA03F3A2425BB2295618D0022A1E
:2081A00013D021EA03032B5430BC70477047C3F13F039CB2084621B2E0E7C4F13F04A4B278
:2081C000C3F17F0000B221B2D8E74B402B54EBE70B432B54E8E700BFB819002034000020AC
:2081E0002DE9F0473B4B1D7886B01DB1284606B0BDE8F087384F39483978394C06AB2122A1
:2082000003F8012D01264FF00208B140CDE9016800932A46334602F0D9FA06AB397803F817
:20822000025DB140CDE9016800932A4633462B4802F0CCFA06AB7F2203F8032D397827488B
:208240000093CDE90168B14033462A4602F0BEFA06AB222203F8042D397820480093CDE965
:208260000168B14033462A4602F0B0FA06AB397803F8055DB140CDE9016800932A463346D4
:20828000164802F0A3FA06AA072302F8063D397812480092CDE901683346B1402A4682467C
:2082A00002F094FA04F580694FF00A084FF4807639780094CDE90168490004F58074012314
:2082C0004022504602F082FAA145F1D1284606B0BDE8F087B9190020310000200C1B0020C6
:2082E000340000204FF480620021014804F0EABD340000202DE9F04F95B0044610460F91D2
:208300000593FFF7BFFC6E4B0E901A8841F23261A3B28A42019383B200F0238241F216612C
:208320008A424AD0202800F0EC82664A125C0132D2B203924FEAC308039B03F1FF3A5FFA1F
:208340008AF21FFA88F800927BB35F4BBDF83C70984407F1080B059B1FFA8BFB83F001099A
:20836000CDF808B09A46DDE9004B18F8016F3DB246FA04F313F0010F0FFA8BFC04F1FF341E
:2083800052462946604602BF4A4660462946E4B2FFF7E0FE0BF1010BFF2C1FFA8BFBE7D1D6
:2083A0000137029BBFB2BB42DDD1BDF80C00019B184400B215B0BDE8F08F203B43495B0135
:2083C0009AB28B18885C10921A790092DA7903921A7C07925A7C08929A7C0992DA7C0A92D9
:2083E0001A7D93F80CA093F80EB00B925A7D99785D7993F8098093F80A905F78DE789C7990
:2084000093F808E093F80BC0CDF810A0CDF818B093F80DA093F80FB00C929A7D0D92009A21
:2084200045EA02220292039A47EA002742EA0424187E049A0090587E4AEA022A069A054627
:20844000187F11904BEA022BDDE9072040EA02220392987F5A7F12921390DA7F46EA0126CB
:2084600048EA0E2ED97D93F81A804CEA092C93F81B90DDE9093040EA03230493DDE90B308B
:2084800040EA032306930D9B41EA03230099079345EA01210891129949EA082509950D46E1
:2084A000119945EA01210A911399002042EA0122012310210B9200901A46CDE90C4114E032
:2084C00032000020084F01082F4B010850FF0008002900F04081009B002A18BF4B46009376
:2084E00043460130102800F0DC80C0F10F0147FA00F818F0010F47FA01F818BF0022029C5B
:20850000039D18F0010F46FA00F918BF002346FA01F819F0010F18BF002244FA00F918F0E6
:20852000010F44FA01F80C9C18BF002319F0010F18BF002244FA00F918F0010F18BF0023F7
:2085400044FA01F819F0010F18BF00224EFA00F918F0010F18BF00234EFA01F819F0010F25
:2085600018BF00224CFA00F918F0010F18BF00234CFA01F819F0010F18BF00224AFA00F923
:2085800018F0010F18BF00234AFA01F819F0010F18BF00224BFA00F918F0010F18BF00232A
:2085A0004BFA01F819F0010F18BF0022049C18F0010F45FA00F918BF002345FA01F819F040
:2085C000010F18BF002244FA00F918F0010F44FA01F8069C18BF002319F0010F18BF00225E
:2085E00044FA00F918F0010F44FA01F8079C18BF002319F0010F18BF002244FA00F918F007
:20860000010F44FA01F8089C18BF002319F0010F18BF002244FA00F918F0010F44FA01F8DD
:20862000099C18BF002319F0010F18BF002244FA00F918F0010F44FA01F80A9C18BF002363
:2086400019F0010F18BF002244FA00F918F0010F44FA01F80B9C18BF002319F0010F18BFF1
:20866000002218F0010F44FA00F844FA01F118BF002318F0010801F001015FFA80F93FF457
:2086800027AF002964D10A46002B3FF42AAF009CC9F10F01091B0130C9B210280D917FF4A0
:2086A00024AF0E9B202B00F01D81009B02930D9B002B4AD05A1EBDF83C80109B0199069282
:2086C00003F1010908F110039BB203934B1E51FA82F704938D4A059B914483F00102BFB2B6
:2086E0000592CDF800909A46009ABDF8104012F8013C1578DDF81890BDF814B045EA0325EE
:20870000029B1D41ADB20FFA88F645FA09F313F0010F0FFA84FC04F10104524631466046F2
:2087200002BF5A4660463146A4B2FFF713FDA74209F1FF39E9D1009B023308F10108009325
:20874000039B1FFA88F84345CED1BDF834002EE600231A46C5E60099002A18BF49460091D6
:2087600092E76B4A6B491578019ABDF83C406A4E9B019BB201F14000013A03EB010EC318D8
:20878000069393B20793059B4FF00108C4F17F0783EA0803BFB24FF080099C46A7F14003D0
:2087A0009EF800209EF8010002971BB2039339B223B240EA022000930F22079B04912BE05E
:2087C0007F2B24D83F2C22D8022D70D0032D66D0012D61D0DDF800A0059FBAF1000FD3466E
:2087E000B8BF0AF1070B4FEAEB0B1BFB09110AF0070A08FA0AFA012F4FFA8AFA16F901B0C8
:2088000045D0022F32D02BEA0A0A06F801A0013A0133511C9BB22ED040FA02FA1AF0010FD1
:2088200019B2CDD17F2BF2D83F2CF0D8022D51D0032D47D0012D42D0DDF800A0BAF1000F22
:20884000D346B8BF0AF1070B4FEAEB0B1BFB09110AF0070A08FA0AFABCF1010F4FFA8AFA81
:2088600016F901B013D0BCF1020FCCD18AEA0B0A06F801A0CBE7029F069B0EF1020E01349A
:20888000013F7345A4B2BFB288D110208FE54AEA0B0A06F801A0BAE78A4604999CE7019909
:2088A000C1F1310A92440FFA8AFA009994E70199DDF80CA0C1F17101114409B28CE78A46C2
:2088C0000499BBE70199C1F1310A92440FFA8AFA0099B3E70199DDF80CA0C1F171011144A8
:2088E00009B2ABE70D4B1878F7F724FE0C4B0022F7F78AFEF8F760F900230293C3B20D932F
:20890000D6E6064A1278039214E500BF50FF0008B8190020300B0108340000203000002044
:208920000000044070B5144612784AB10E461D462B463146FFF7DEFC14F8012F002AF7D152
:2089400070BD00BF002A5FD02DE9F04F1FFA80FC2E4CBCF17F0F83B089B294F800E03AD847
:20896000CCF17F0424B2CCF13F081FFA88F80094DFF89C90C1F13F040FFA88FB0027019470
:208980004FF0800ABDB26C18A4B23F2C20D8BEF1020F26B223D0BEF1030F31D0BEF1010F56
:2089A00027D00546002EB8BF0736F61016FB0A5504F007060124B440012B64B219F905604A
:2089C00013D0022B14BF26EA0404744009F805400137BA42D6D1002003B0BDE8F08F019C33
:2089E000641BA4B226B2009DDCE7344309F80540EEE7C1F17F04651B2DB264460646D1E796
:208A0000354644465E46CDE700207047B8190020340000202DE9F04F87B093469DF844405F
:208A20009DF840500095002C40F0F1808DB2002B00F0BF81DFF814C43F2D87B29CF800E04D
:208A400044D8C5F17F0212B2C5F13F0A0492C7F17F021FFA8AFACDE90112A146DFF8E883A2
:208A60000FFA8AF403941FFA89F4E21992B27F2A28D8BEF1020F16B200F0C381BEF1030FDD
:208A800000F08681BEF1010F00F0B381019C2A46002CB8BF0734E410802114FB016600996D
:208AA000012402F0070204FA02F2012952B218F9064000F09A81022914BF24EA0202624062
:208AC00008F8062009F101094B45CCD10BEB050E1FFA8EFE0FFA8EF20192BBF1000F00F0CA
:208AE000F4807F2F9CF8006048D8C7F13F08C7F17F021FFA88F812B20FFA88F10292DFF8BE
:208B00004893009C0491C5F13F024FF0000C0392CDF814801FFA8CF16A1892B23F2A29D853
:208B2000022E0FFA82FA00F07E81032E00F03D81012E00F071810146BAF1000FB8BF0AF12E
:208B4000070A4FEAEA0A4FF080081AFB081102F0070A012202FA0AF2012C52B219F901A0E0
:208B600000F05581022C14BF2AEA020282EA0A0209F801200CF1010CDC45CBD1DC19A4B26A
:208B80000FFA84FA1BB1BEF13F0F40F2A7807F2C39D8C4F17F0CC4F13F0424B2AA4F0194D4
:208BA0000FFA8CFC0020C5F13F094FF080084FF0010E82B2AB189BB23F2B21D8022E1BB24D
:208BC00000F01A81032E00F0E080012E00F035815146002B1A46B8BFDA1DD210009C12FB99
:208BE000081203F007030EFA03F3012C5BB2B95600F02081022C14BF21EA03034B40BB54DA
:208C000001308345D5DC002007B0BDE8F08F002AF9D08E4ADFF830A292F8009084B21FFAD2
:208C200081FEC4F17F020492CEF13F020292CEF17F02AC4603920026002B3FD0B2B20EEBD1
:208C4000020189B23F290FFA81F837D803980299891A821A09B212B200910192002081B272
:208C60000A1992B27F2A26D8B9F1020F12B200F08780B9F1030F7DD0B9F1010F77D04146DF
:208C800000290D46B8BFCD1DED10802715FB072201F00701012505FA01F1BCF1010F49B252
:208CA0001AF902505FD0BCF1020F14BF25EA010169400AF8021001308342D0D101365E4550
:208CC000BAD1002007B0BDE8F08FDC19A4B2BEF13F0F9CF800600FFA84FA94D8CEF13F02DF
:208CE00012B2CEF17F0E04920FFA8EF20592DFF858C10294C7F17F02002003924FF0800E6D
:208D00004FF0010981B2CA1992B27F2A22D8022E12B25DD0032E42D0012E63D00199009C11
:208D200000298846B8BF01F107084FEAE80818FB0E2201F0070109FA01F1012C49B21CF92D
:208D400002804AD0022C14BF28EA010181EA08010CF8021001308342D4DC029CBBF1000FD9
:208D60007FF415AF4FE729430AF80210A3E71146019A85E7C4F13F02511A09B242467FE714
:208D8000049A521A12B200997AE71946019B20E7C7F13F02121B92B214B2019E78E6C7F124
:208DA0003F02511A09B2019AB9E75146DDE904A2C2E602EB050E1FFA8EFE0FFA8EF20192A5
:208DC000BBF1000F3FF41FAFDFF880C087B288E6039A521A12B20499A1E741EA08010CF8EF
:208DE0000210B7E71146059A99E7224308F8062068E63446049E4BE6A9EB02031BB261461A
:208E0000E7E6029A141B26B25246039C40E642EA0A0209F80120ADE6C5F17F02511A09B23B
:208E20003A46824688E6039A521A92B20FFA82FA029981E60B43BB54E2E6C5F17F018A1AA9
:208E400011B25346C5E600BF34000020B8190020034A0449044B1080020A08701A707047C9
:208E6000320000203625002035250020014B1878704700BF35250020014B1878704700BF8D
:208E8000362500202DE9F04FDFF830A1DFF830819AF8003083B01A460193002388F8003016
:208EA000002A54D1044600F0B9F900284FD0002C5CD1F02000F0AAF801200446F8F788F95A
:208EC000DFF80091394F2546002600F0A5FD834600F0A2FDBBF1010F4CD08345BA5D50D14F
:208EE00099F8003032480121AB42017058D9144214BF0846002000283FD1082D54D82D4BDE
:208F000001951D7022EA0402BA5500F0C5FD64005A20F8F75DF9013514F0FF04EDB232D05A
:208F2000072ED2D9402D14D998F800308BB9019B89F8003013B901238AF800301E4A1B4938
:208F4000136809780133136019B101200BE0DFF87490184B00241C7089F800408AF8004027
:208F600000F0E2FD204603B0BDE8F08FEC2000F04DF8A1E70128D5D0BA5D2243BA550120A2
:208F8000C3E75846BEE7B95D98F8000000F052F90136F6B2072E88F80000C3D8012494E734
:208FA0000CBF01200020A6E70195ABE7382500204025002042250020482500204325002052
:208FC000412500204425002038B5002000F064F907480849084A094D094C002303700B707A
:208FE000137018462B602370BDE83840FFF74ABF4025002043250020422500204825002035
:20900000442500200020FFF73DBF00BF38B50546082405F0010000F03FFD631E13F0FF04E9
:209020004FEA5505F5D138BD38B50825002400F0F3FC64086B1E44EAC01413F0FF05E4B231
:20904000F5D1204638BD00BF2DE9F0413C4F3B780646F3B90824552505F0010000F01CFD0E
:20906000631E13F0FF044FEA5505F5D106F1080716F8015B082405F0010000F00DFD631E03
:2090800013F0FF044FEA5505F5D1BE42F0D1BDE8F0812C4A0178107888422CD150787178AB
:2090A000884228D19078B178884224D1D078F178884220D13079117988421CD170795179F4
:2090C000884218D1B0799179884214D1D279F179914210D1DB074FF008040DD5A52505F0C4
:2090E000010000F0D9FC631E13F0FF044FEA5505F5D1BDE8F0810824692505F0010000F014
:20910000CBFC631E13F0FF044FEA5505F5D10123DFF834803B70771E073617F8015F08F80D
:20912000015F082405F0010000F0B6FC631E13F0FF044FEA5505F5D1BE42EED1BDE8F08156
:209140004C250020BC190020BB1900202DE9F0412F4B02781978914205462ED15978427821
:2091600091422AD181789A78914226D1C178DA78914222D101791A7991421ED141795A799F
:2091800091421AD181799A79914216D1DB79C279204F9A4238D13B78DB074FF0080434D57E
:2091A000A52505F0010000F077FC631E13F0FF044FEA5505F5D1BDE8F081164F0824692676
:2091C00006F0010000F068FC631E13F0FF044FEA5606F5D10123DFF840803B706E1EEF1D64
:2091E00016F8013F08F8013F3578082405F0010000F052FC631E13F0FF044FEA5505F5D1F4
:20920000B742EDD1BDE8F08108246926D8E700BFBC1900204C250020BB19002008B5044BC2
:2092200000221A7000F080FCBDE8084000F07CBC4C25002041404B08C80748BF83F08C03C4
:209240005A08D90744BF82F08C02D2B25308D20744BF83F08C03DBB25A08DB0744BF82F0C6
:209260008C02D2B25308D00744BF83F08C03DBB25A08D90744BF82F08C02D2B25308D2071B
:2092800044BF83F08C03DBB25808DB0744BF80F08C00C0B2704700BF024B187000B17047D6
:2092A00000F042BC4C250020704700BF2DE9F8438046894616461F469DF8205000F034FCED
:2092C00070B31E4B1B7823BBB8F1000F2ED14846FFF73CFFF020FFF799FEF8B2FFF796FE4A
:2092E000380AFFF793FE0120F7F772FF5DB1902D28BF90253446FFF797FE04F8010BA31BF3
:20930000DBB29D42F7D8012400F00EFC2046BDE8F883B8F1000F0DD0CC20FFF777FED9E7C1
:20932000044600F001FC2046BDE8F8833C20FFF76DFECFE74846FFF787FECBE74E250020AF
:20934000F8B506460F46144600F0EEFB18B3184B1B78DBB926BB3846FFF7F8FEF020FFF7E6
:2093600055FE8020FFF752FE0020FFF74FFE0120F7F72EFFE51DFFF757FE04F8010BAC42D2
:20938000F9D1012500F0D0FB2846F8BD66B1CC20FFF73CFEE2E7054600F0C6FB2846F8BDE4
:2093A0003C20FFF733FED9E73846FFF74DFED5E74E2500202DE9F04F83B08046019117461F
:2093C0001E4600F0B1FB002800F0C2825B4B1B78002B40F0B682B8F1000F40F0C0820198A2
:2093E000FFF7B4FE0120FFF757FF26F007050F20534CADB2FFF70AFE4FF6FF7305F0F80067
:209400002380FFF703FE238806F0F8065E407308F20744BF83F4204383F00103DE074FEA8F
:20942000530204D582F4204282F0010292B2D0074FEA520304D583F4204383F001039BB291
:20944000D9074FEA530204D582F4204282F0010292B25308D20704D583F4204383F00103D6
:209460009BB25A08DB0704D582F4204282F0010292B2D6074FEA520304D583F4204383F060
:2094800001039BB2D8074FEA530204D582F4204282F0010292B22D0A28462280FFF7B6FDB4
:2094A00023885D406A08E90744BF82F4204282F001025308D20704D583F4204383F0010354
:2094C0009BB25A08DB0704D582F4204282F0010292B2D6074FEA520304D583F4204383F000
:2094E00001039BB2DD074FEA530204D582F4204282F0010292B2D0074FEA520304D583F48A
:20950000204383F001039BB2D9074FEA530204D582F4204282F0010292B25308D20704D53F
:2095200083F4204383F001039BB2064D23800022013F2A704AF2010607E000BF4E2500201F
:20954000C8190020C6190020238817F8010F4340C3F34F01DB0748BF71404A08C90744BFF9
:20956000724092B25308D20744BF73409BB25A08D90744BF724092B25308D20744BF734099
:209580009BB25A08D90744BF724092B25308D20744BF73409BB25A08DB0748BF724022806D
:2095A000FFF734FD2B780133DBB2072B2B70CBD90120F7F70DFEFFF737FDC04F3880FFF7AE
:2095C00033FD3B8843EA0023DB433B8000F0ACFABB4B1B78002B40F0D781B8F1000F00F0E5
:2095E000E8813C20FFF712FD0120FFF755FEAA20FFF70CFD0120F7F7EBFD4FF6FF7323801D
:20960000B04EFFF711FD2B782288F35CAE49534008705908D80744BF81F4204181F001011E
:209620004A08C90704D582F4204282F0010292B25308D20704D583F4204383F001039BB2F3
:209640005A08DB0704D582F4204282F0010292B2D0074FEA520304D583F4204383F00103CD
:209660009BB2D9074FEA530204D582F4204282F0010292B25308D20704D583F4204383F06B
:2096800001039BB25A08DB0704D582F4204282F0010292B22280FFF7C7FC2B782288F35CD4
:2096A00053408A4A59081070D80744BF81F4204181F001014A08C90704D582F4204282F0F2
:2096C000010292B25308D20704D583F4204383F001039BB25A08DB0704D582F4204282F031
:2096E000010292B2D0074FEA520304D583F4204383F001039BB2D9074FEA530204D582F48A
:20970000204282F0010292B25308D20704D583F4204383F001039BB2D8074FEA530204D53D
:2097200082F4204282F0010292B22280FFF77CFC2B782288F35C5340654AD90710704FEA11
:20974000530244BF82F4204282F001025308D20704D583F4204383F001039BB25A08DB0775
:2097600004D582F4204282F0010292B2D0074FEA520304D583F4204383F001039BB2D907C3
:209780004FEA530204D582F4204282F0010292B25308D20704D583F4204383F001039BB226
:2097A0005A08DB0704D582F4204282F0010292B2D0074FEA520905D589F4204383F001035F
:2097C0001FFA83F90022A4F800902A7093464AF2010AFFF729FC89EA0009C9F34F0319F03E
:2097E000010F18BF83EA0A035A08D90744BF82EA0A0292B25308D20744BF83EA0A039BB209
:209800005A08DB0744BF82EA0A0292B2530806F80B00D00744BF83EA0A039BB25A08D907FE
:2098200044BF82EA0A0292B25308D20744BF83EA0A039BB24FEA5309DB0795F800B040F186
:2098400096800BF1010B5FFA8BFB89EA0A091FFA89F9BBF1070FA4F8009085F800B0B8D93E
:20986000FFF7E2FB3880FFF7DFFB3B8843EA0023DB433B8000F058F9114B1B78002B40F016
:209880009180B8F1000F00F0A4803C20FFF7BEFB0120FFF701FD5520FFF7B8FB0A4B0D4CFF
:2098A0001878FFF7B3FB094B1878FFF7AFFB084B1878FFF7ABFB01200EE000BFC4190020A6
:2098C0004E250020D0190020CC190020CD190020CA190020CB190020FFF7E6FC0A2000F0E8
:2098E000E1F90020FFF7E0FCFFF79EFBAA2804BF0123237000F018F93A4B1B78002B4AD162
:20990000B8F1000F5DD03C20FFF780FB0120FFF7C3FCAA20FFF77AFB0120F7F759FCFFF730
:2099200083FB314B1870FFF77FFB304B1870FFF77BFB2F4B187000F0F7F8207803B0BDE8F5
:20994000F08FB8F1000F0ED0CC20FFF75FFB4CE5284C00F0E9F8207803B0BDE8F08F3C2075
:20996000FFF754FB3EE50198FFF76EFB3DE50BF1010B5FFA8BFBBBF1070FA4F8009085F813
:2099800000B07FF626AF6BE7B8F1000F1DD0CC20FFF73CFB2BE6B8F1000F1ED0CC20FFF724
:2099A00035FBB6E7B8F1000F07D0CC20FFF72EFB71E70198FFF7CAFB16E60198FFF744FBCA
:2099C00069E70198FFF7C2FBA0E70198FFF73CFB0DE60198FFF7BAFB5AE70198FFF734FB68
:2099E00097E700BF4E250020CC190020CD190020CA190020CB1900207F2B07D810B41C46D6
:209A0000640705D000205DF8044B7047002070475DF8044BFFF7CEBC38B51D4C0020FFF724
:209A200043FC237803B172B600220221194800F0D5FC2378D3B90620F7F7CAFB01220221C3
:209A4000144800F0CBFC2378EBB90920F7F7C0FB0221104800F0BCFC2378051C18BF012506
:209A600043B93720F7F7B4FB284638BD0120F7F7AFFBE3E762B62378002BF2D00720F7F75B
:209A8000A7FB284638BD0120F7F7A2FBE0E700BF4C2500200000024038B5214C05460020F7
:209AA000FFF702FC237803B172B6002202211D4800F094FC2378C3B90620F7F789FBCDB9DC
:209AC00023782BB30920F7F783FB01220221154800F084FC237803B162B60220F7F778FB7B
:209AE0000120BDE83840FFF7DFBB0120F7F770FB002DE5D0012202210A4800F06FFC012028
:209B0000FFF7D2FB23783BB93A20F7F761FBDCE74020F7F75DFBD8E70720F7F759FBD4E703
:209B20004C250020000002402DE9F041324FDFF8D0803B78002288F80020002B55D100227B
:209B400002212E4800F04AFC3B78002B44D14FF42F70F7F73DFB2948012202210646002414
:209B600000F03CFC06E00A20F7F732FB40F291139C423ED00221304600F02AFCA5B2013495
:209B80000028F0D03B781BBB4620F7F721FB02211A4800F01DFCB5F5BE7F044605D25F2DC2
:209BA0008CBF0223012388F800303B78C3B12820F7F70EFB0120FFF777FB012000F072F8F7
:209BC0000020FFF771FBB4FA84F04009BDE8F0810920F7F7FDFADAE74620F7F7F9FABAE7CB
:209BE0004FF4D270F7F7F4FAE4E70220F7F7F0FAA5E72546C6E700BF4C2500200000024009
:209C00004D25002038B50E4A0E4B12781B6805464FF47A70B0FBF2F0B3FBF0F000F0D0F8BC
:209C200008B90F2D01D9012038BD0446024629464FF0FF3000F05AF8034B20461D6038BD60
:209C4000340400202C0000203804002008B50B4B1A6842F400721A601A6842F480621A6039
:209C60001A6842F480721A60032000F02DF80020FFF7C8FFFDF796FB002008BD003C0240C3
:209C8000034A044B11681B780B441360704700BF5025002034040020014B1868704700BFB5
:209CA0005025002038B50446FFF7F6FF631C054602D0044B1B781C44FFF7EEFF401BA042EF
:209CC000FAD338BD34040020074AD3684FF6FF010B40000243F0BF6300F4E06043F4003359
:209CE0000343D360704700BF00ED00E0184BDB68C3F3022330B4C3F10705042D03F1040456
:209D000028BF0425062C19D9033B4FF0FF349C4022EA04044FF0FF32AA4021EA020101FA0C
:209D200003F2224312010028D2B20ADB00F1604000F5614080F8002330BC70470024234633
:209D4000E8E7044B00F00F0003441A7630BC704700ED00E0FCEC00E0002807DB00F01F01BD
:209D600001234009024A8B4042F82030704700BF00E100E000280DDB43092033012206497D
:209D800000F01F0002FA00F041F82300BFF34F8FBFF36F8F704700BF00E100E0BFF34F8F65
:209DA0000549064BCA6802F4E0621343CB60BFF34F8F00BFFDE700BF00ED00E00400FA0557
:209DC0000138B0F1807F0ED2084B10B4084C5860F02084F823000022072110469A601960E5
:209DE0005DF8044B70470120704700BF10E000E000ED00E0F8B50446FFF74EFF002C54D04A
:209E00000222236884F835201A68002122F0010284F8341005461A6005E0FFF73DFF401B13
:209E200005283BD823681A68D107F6D4D4E90126D4E90351324360691F682A43D4E90665E4
:209E40000A430243216A354832432A430A43616A3840042942EA000229D01A605A6922F053
:209E600007021143DAB22E485961103AA0FB021212092C4923F47F73895CE16523F00303F3
:209E8000032A88BF04333F228A4001250021A36508469A60616584F83550F8BD0323202271
:209EA0006265184684F83530F8BD0120F8BDD4E90B0101430A43A56A1A605A6945F0040131
:209EC00022F0070211430028CCD07EB1B6F5005F16D0022D03D9032DC4D1C201C2D50123E2
:209EE00040226265184684F83530F8BD012D03D0F3D3022DB6D1F0E7B0F1C07FB2D1EEE7B9
:209F0000032DAFD801A252F825F000BFDF9E0008DB9E0008DF9E0008F99E00083F8010F0E0
:209F2000ABAAAAAA9C4F010890F83530022B03D080234365012070470268052380F8353005
:209F4000136823F00103136000207047F0B583B00023876D0193C36D3D68654908229A401B
:209F60002A4204460E6803D001680868400759D401229A402A4203D021684969080674D4C8
:209F800004229A402A4203D021680968890766D410229A402A4203D02168086800074BD454
:209FA00020229A402A4214D021680868C00610D5BA6094F83520052A63D00B6813F4802F0B
:209FC0000B687ED0190340F18980E36B0BB120469847636D23B3636DDA071AD50523226823
:209FE00084F835301368434923F00103A1FB06161360B60A02E01368DB0704D5019B01338F
:020000040800F2
:20A00000B3420193F7D90022012384F8342084F83530E36C23B1204603B0BDE8F040184780
:20A0200003B0F0BD086820F004000860BA60626D42F0010262659BE7BA600A6812F4802F2C
:20A040000A6818D1D20503D40A6822F008020A60226C002AA4D020469047E36DA0E7BA60A5
:20A06000626D42F00402626592E7BA60626D42F00202626584E71103EAD5A26C002AEAD182
:20A080008EE70A68206C22F016020A604A6922F080024A6138B30A6822F008020A603F2283
:20A0A000216D02FA03F300200122BB6084F8340084F835200029B3D0204603B0BDE8F040A7
:20A0C000084713F4807380D10A68012022F010020A6084F8343084F8350076E7636C002BDD
:20A0E0007FF475AF75E7A26C002AD4D1D7E700BF2C000020B5814E1B90F83500704700BFF5
:20A100002DE9F04F884683B0D1F800B0DFF898E100244FF0010902E00134102C77D009FA16
:20A1200004F20BEA02039A42F6D1D8E9012622F0100C65000CF1FF370321A940012F6FEA48
:20A14000010106FA05F665D9C7680F403E43C660076802F003060F4006FA05F53D43D70095
:20A160000560D9D54B4D00210191696C41F480416964696C24F0030606F1804601F4804184
:20A1800006F59C36019104F003050199B768AD000F21A94027EA01013F4FB84211D007F56D
:20A1A0008067B84268D03D4FB84269D03C4FB8426BD03C4FB8420CBF0427072707FA05F563
:20A1C0002943B160DEF80010DD43D60354BF29401943CEF80010DEF80410970354BF294075
:20A1E0001943CEF80410DEF80810D60254BF29401943CEF80810DEF80C10920204F101042D
:20A2000054BF29401943102CCEF80C1087D103B0BDE8F08F876807EA010AD8F80C70AF40F3
:20A2200047EA0A078760D0F804A0C2F300172AEA030AA74047EA0A074760C7680F403E43CD
:20A24000BCF1020FC66083D14FEAD40A00EB8A0A04F00706DAF82070B6004FF00F0C0CFAB7
:20A2600006FC27EA0C0CD8F8107007FA06F646EA0C06CAF820606BE709FA05F52943A0E7A0
:20A28000022707FA05F529439BE7032707FA05F5294396E700380240000002400008024098
:20A2A000000C024000100240003C01402DE9F04F002383B0DFF814914FF001084FF00F0ABA
:20A2C0004FF0030B02E00133102B66D008FA03F404EA0105AC42F6D123F0030606F180462F
:20A2E00006F59C3603F00302B76892000AFA02FC0CEA07070197314FB84251D007F58067CC
:20A30000B8424FD02E4FB8424FD02E4FB84251D02D4FB84214BF4FF0070E4FF0040E0EFA00
:20A3200002F2019F974218D1D9F80020ED432A40C9F80020D9F804202A40C9F80420D9F846
:20A3400008202A40C9F80820D9F80C201540C9F80C50B26822EA0C02B2605A0005680BFA01
:20A3600002F2D243DE08154000EB8606056003F00705376AAD000AFA05F527EA05053562C0
:20A38000C5681540C560456825EA04044460846801332240102B826098D103B0BDE8F08FCF
:20A3A0000022BEE708FA02F2BBE74FF0020E0EFA02F2B6E70BFA02F2B3E700BF00000240C2
:20A3C00000080240000C024000100240003C01400369194214BF01200020704702B90904BC
:20A3E00081617047436931EA030308BF09048161704700BF704700BF044A5169014200D139
:20A40000704708B55061FFF7F5FF08BD003C0140036D5BB9C36C0268012B836C0DD0C3F320
:20A4200007231361036D013303657047036D012B09D0036D022B0ED07047DBB21361036DA3
:20A44000023303657047836C0268DBB21361036D01330365704790F83D30222B0ED090F8E3
:20A460003D30212BE8D1426A036812F8011B1961438D4262013B9BB24385DDE70268136845
:20A4800043F48073136070472DE9F0420446006882B089460168089D41F4807116461F4678
:20A4A00001606A1C40D14369DB07FCD509F0FE0101616B1C14D043699B0714D443695A053F
:20A4C00056D4FFF7E9FB099BC01A8542C0F0A080002D00F09D802068EBE743695A0547D4A9
:20A4E00043699907F9D5002301934369019383690193019B6A1C03D06CE0436959054FD45D
:20A5000043691B06F9D5012F0AD0330A03616F1C03D06EE043695A0542D443691906F9D58F
:20A52000F6B2066100201CE04369D907BED4FFF7B3FB099BC01A8542206801D3002DB0D1DF
:20A5400000222023226384F83D3084F83E20236C84F83C2043F0200323640368D90503D4EA
:20A56000032002B0BDE8F0824FF400732364F7E7036800226FF4806543F4007320210360B1
:20A580004561226384F83D1084F83E20236C84F83C2043F004030120236402B0BDE8F082DB
:20A5A000002220236FF480614161226384F83D3084F83E20236C84F83C2043F004032364E0
:20A5C000236C042B04D12268136843F4007313600120C6E743691A0695D443695905DFD406
:20A5E000FFF75AFB099BC01A854220D3FDB1206880E743691B0693D443695B05D0D4FFF761
:20A600004BFB099BC01A854211D385B120687EE700222023226384F83D3084F83E20236C6C
:20A6200084F83C2043F020032364012099E700222023226384F83D3084F83E20236C84F80C
:20A640003C2043F020032364BAE700BF002800F09F80F8B590F83D30044603F0FF02002B1F
:20A6600000F08F802368242284F83D201A6822F001021A601A6842F400421A601A6822F414
:20A6800000421A6001F05CFB61684B4B99424BD84A4B98427AD92268494B5568A3FB0063BB
:20A6A0009B0C25F03F051D435560156A013325F03F052B431362D5694900431EB3FBF1F31C
:20A6C0000133C3F30B0325F44F45042B38BF042325F0FF052B43D361D4E9073510682169D2
:20A6E00020F0C0002B43034313609068E568636920F4034020F0FF00294301439160D16812
:20A70000A06921F0FF0103430B43D3601168002341F00101202511601846236484F83D50E5
:20A72000236384F83E30F8BD264B98422ED92268234B5668244FA3FB00539D0C26F03F0684
:20A740002E434FF49673566003FB05F3A7FB0353156AA6689B0925F03F0501332B431362F7
:20A76000D56925F44F45013825F0FF0596B901EB4101B0FBF1F00130C0F30B00C0B9012307
:20A78000A8E780F83C20FCF735FE6BE70120F8BD0120704701EB810101EB8101B0FBF1F0C8
:20A7A0000130C0F30B000028E9D040F4404391E740F400438EE700BFA08601007F841E00A7
:20A7C00083DE1B43FF083D00D34D62102DE9F04F044683B099460F469046BDF834A00E9ED3
:20A7E000FFF75AFA94F83D30202B04D00227384603B0BDE8F08F054605E0FFF74DFA401BB1
:20A80000192800F2A68022689369DB4313F0020BF3D094F83C30012BE8D013680121D80710
:20A8200084F83C1002D413680B43136013685E4823F400631360212384F83D30402200237E
:20A8400084F83E202364A4F82AA0B4F82AC00C9B63623946CDE900654B46E0624246A4F89E
:20A8600028C02046FFF710FE074600284FD12368228DF2B1721C03D04EE05A6951052ED46A
:20A880005A691006F9D5D4F824C0B4F828E060460EF1FF3210F8011B1961618D606201394F
:20A8A00089B26185596992B248072285E1D5002A40D1721C03D05AE05A6951050FD45A6930
:20A8C0005007F9D51A680021202042F400721A6084F83D0084F83C1084F83E1087E7002273
:20A8E0006FF4806020215861226384F83D1084F83E20236C84F83C2043F004032364236C3C
:20A90000042B04D12268136843F4007313600127384603B0BDE8F08F5A691206B3D45A696F
:20A920005105DCD4FFF7B8F9401B86422DD366B323689FE79CF801201A61608DAEF102025D
:20A94000013892B20CF1020180B22285616260858FE72023C4F830B084F83D3084F83EB051
:20A96000236C84F83CB043F0200323643EE75A695207A7D45A695105B1D4FFF78DF9401BD2
:20A98000864202D30EB1236893E700222023226384F83D3084F83E20236C84F83C2043F00F
:20A9A00020032364ABE700BF0000FFFF704700BF704700BF704700BF704700BF704700BF50
:20A9C000704700BF704700BF704700BF704700BF704700BF836BD3E90D0170B593F83D4044
:20A9E0001A68E6B240B30024C463F1B11568CC6325F4806515605C850465002008651168EE
:20AA000021F00101116093F83D10602929D006F02804282C18D02021002283F83D1083F854
:20AA20003E201846FFF7D2FF70BD146824F48064146059850165E2E7F1B11468C86324F40C
:20AA4000806414605885D8E7116841F0010111601168002041F480611160186383F83D4052
:20AA6000DFE70022202183F83D10184683F83E201A64FFF7ADFF70BD106820F48060106085
:20AA80005985BCE770B5036804465868E56A94F83E2094F83D10D2B2102A8CB020D0402A35
:20AAA0001ED0226CC9B2002A00F0BB805A690026C2F34005002D78D085057BD5226C02B1D7
:20AAC0009E6994F83D2002F02802282A00F01C826FF002010022596184F83C200CB070BD8B
:20AAE00099695A69D6073AD4B5F52A0FF6D0B5F12A4FF3D0160740F19A80850500F1F581C2
:20AB000011F0040F596800F0FF800905E6D41606C2F3800140F1A081450540F19D810029C3
:20AB200040F09D8194F83D20208D94F83E10E56AD2B2C9B2002840F07883212A00F01884DF
:20AB40004029CBD1222AC9D1628D92B2002A00F0098494F83E20402A40F0B6808DE185057E
:20AB600062D5E26AB2F52A0F00F0E981E26AB2F12A4F04BF0822E26294F83E20402A00F03B
:20AB8000D7812269B2F5804F00F09781226D002A00F0D881226D012AA0D1626CD21102F084
:20ABA000060242F0F1021A6198E7D60602D5860500F1D78001F0F7012129C2F380054ED05D
:20ABC000510640F18B80420540F18880002D40F0888094F83D10628D92B2C9B2002A3FF419
:20ABE0007DAF626A1B691370638D626A013B9BB26385638D01329BB26262002B7FF46EAF3A
:20AC00002A297FF46BAF22685368222523F48063282153602046256384F83D10FFF7CCFE5B
:20AC20005CE79E695A6943E715073FF569AF96077FF566AF85057FF563AF94F83E20E06A0B
:20AC4000256B94F83D102229D2B200F00B8200220A925A690A929B690A930A9B3EE712069F
:20AC600027D5460525D53DBB94F83D00628D92B2C0B2002A3FF432AF656A15F8012B1A616C
:20AC8000628D6562013A92B26285628D92B2002A7FF424AF29287FF421AF5A68282522F43C
:20ACA00080625A602046216384F83D50FFF782FE14E7002D3FF412AF80057FF50FAF628DCD
:20ACC00092B2002A3FF40AAF626A12F8011B1961638D6262013B9BB26385FFE6002D3FF444
:20ACE000FDAE86057FF5FAAE628D92B2002A3FF4F5AE626A1B691370638D626A013B9BB2B7
:20AD0000013263856262E9E60E053FF5E7AE5506C2F3800140F1B780420540F1B4800029DB
:20AD200040F0B48094F83D20222A7FF4D7AE628D92B2032A40F2E982626A1B691370638DC2
:20AD4000626A013B9BB26385638D9BB20132032B62627FF4C3AE2268536823F4806353607E
:20AD6000BCE694F83D105A6822F4E0625A600B955A690B921A6842F001021A600B9A1A682C
:20AD800022F480621A605A68CDB2110521D505F0F702222A00F04181606B0268526892B2D5
:20ADA0006285628D92B21AB1226C42F0040222645A6822F400625A60FFF79EF9012808D0E0
:20ADC000606BA64B0365FFF7AFF810B1606B036D9847638D9BB213B323685A6952070AD54E
:20ADE000626A1B691370628D616A2368013A92B20131628561625A69560609D5626A1B6993
:20AE00001370638D626A013B9BB2013263856262638D9BB21BB1236C43F004032364236CA3
:20AE2000002B40F09D802A2D00F04F8194F83D30282B00F0E080236B222B02D0222D7FF478
:20AE40004DAE002320222363204684F83D2084F83E30FFF7B1FD41E600293FF43FAE820548
:20AE60007FF53CAEE16A94F83D20212A00F06E8194F83E30402B7FF431AE20460CB0BDE898
:20AE80007040FFF7C5BA00293FF428AE86057FF525AEE06A628D616A92B2042A00F07B8127
:20AEA000628D92B2032A00F0B181628D92B2022A00F0D4811B690B701EE794F83D20212A34
:20AEC000626C16BF42F0010202F0FE02D2B21A61626B002A00F0E380D26B002A00F0DF80A9
:20AEE0005A6842F400625A60F8E5626C616BD2B21A61002900F08C80CA6B002AF0D1A26B76
:20AF0000D26B002AECD1E9E55A6822F480625A606FEA960133064FF0000301F0010154BF5A
:20AF2000A289228B84F83C302046FFF747FDD5E5226D7AB9626C02F0FE021A61CEE5012224
:20AF4000E26219E6626CD21102F0060242F0F0021A61C3E5626C42F00102D2B21A61BDE518
:20AF600094F83D2094F83E1023681029D2B200F0B98002F02801282900F0AF805968090543
:20AF800004D4602A02D0202284F83D200022226384F83E205A6812F4006200F085805A6800
:20AFA000606B22F400625A6090F83530012B00F00F812A4B0365FEF7B7FF50B12268606B1D
:20AFC0001368016D23F001032025136084F83D508847236C180704D02268536823F4E063C0
:20AFE000536094F83D30226C5107DBB27FF576AD282B7FF473AD1A4BE36220220023236320
:20B00000204684F83D2084F83E30FFF7D9FC65E5A26B002A7FF470AF60E5A06B02685268B5
:20B0200092B26285628D92B21AB1226C42F0040222645A6822F400625A60FFF75DF8012833
:20B040003FF4C7AEA06B054B0365FEF76DFF00283FF4BFAEA06B036D9847BAE6D5A90008DC
:20B060000000FFFF216D11B9402A00F0E280226D22B92169B1F5404F00F0E280628D92B210
:20B08000002A3BD103925A6903929A690392039A1A6842F400721A60002323651EE5A26BF9
:20B0A000002A7FF42DAF19E594F83D10602979D05A69550605D5626A1B691370636A0133A2
:20B0C00063622046FFF782FC83E728222363204684F83D20FFF770FCA8E60022226384F845
:20B0E0003D1057E7222A7FF444AF1A6822F400621A605A6810057FF546AF47E7628D92B2FE
:20B10000012A00F0E180628D92B2022A00F056811A6842F480621A605A6815050ED510F5B5
:20B12000803F07D001381F2808D8A14A22FA00F0C00703D55A6842F480525A600022099242
:20B140005A6909929B690993099BA5E7628D92B2002A7FF4B9AD082905D0202903D011F563
:20B16000803F40F07E815A6822F4E0625A6019680022202041F400711960226384F83D00CD
:20B1800094F83E3084F83E20402B204600F00B81FFF70CFCA2E45A6822F480625A601B6912
:20B1A0000B70A9E5202184F83D1022645A69560606D5626A1B691370626A236801326262DB
:20B1C0001A6822F001021A602046FFF701FC00E7A06B784B0365FEF7A7FE00283FF4F9AE4C
:20B1E00023685A69520606D5626A1B691370626A2368013262621A68A06B22F001022021CA
:20B200001A60036D84F83D109847E2E65A68042822F480625A603FF44DAE02283FF44AAEB1
:20B220001A6822F480621A6044E6212A3FF48CAC86E401915A6901929B690193019B4DE483
:20B2400002925A6902929A690292029A1A6842F480721A60236D013323653FE401281A6892
:20B260007CD010287AD0042800F00881022800F0058142F400721A601B690B70638D626ADE
:20B280002168013B9BB263850B69511C61625370638D2168626A013B9BB263854B680132B1
:20B2A00023F44073202062624B6084F83D0094F83E30402B49D00022122384F83E20204647
:20B2C0002363FFF775FB09E410F5803F00F0B580082800F0A280202800F09F80122D00F0E4
:20B2E0009980102805D8344A22FA00F0C00700F1D4801A6822F480621A60002206925A6919
:20B3000006929B690693069BC6E6E16A02293FF4E5AB012A3FF6E2AB1A68616A22F4806240
:20B320001A605A6822F4E0625A601B690B70638D626A013B9BB22021638584F83D1094F8FD
:20B340003E300132402B6262B5D1002384F83E3020462363FFF738FBFFF7C0BB22F480620C
:20B360001A6089E75A6822F480625A60FFF7B6BB082D3FF4F8AE202D3FF4F5AE15F5803F0E
:20B380003FF4F1AE5A68112622F4E062002520215A602046266384F83E5084F83D10FFF7B2
:20B3A00005FBFFF79BBBFFF70DFBFFF797BB00BF81800080D5A9000814000100102820D9EF
:20B3C0001A6822F480621A601A6842F400621A605A6812050DD510F5803F06D001381F2810
:20B3E00007D8304AC240D60703D55A6842F480525A60002208925A6908929B690893089B5E
:20B400004AE6294AC240D107DAD51A6842F480621A60DDE701283FF46CAF1A68002122F4F8
:20B4200080621A6007915A6907929A690792079A1A6842F400721A602EE61A6822F480624D
:20B440001A605A6812F400621CD01A68002122F480621A6004915A6904929B690493049B1F
:20B460001AE65968112621F4E061202559602046266384F83E2084F83D5089E642F4806227
:20B480001A60F9E605925A6905929A690592059A1A6842F400721A60FEE51A6842F4806208
:20B4A0001A602AE78180008014000100F8B503685D695A6890F83E10CEB2E90504469C465B
:20B4C000C5F3402078D5110ACF0775D56FF480725A6100287FD1690540F1D5800127628D39
:20B4E00094F83D10206B202E92B2C9B200F0AA806FF48062102E47F004075A6101D0402E02
:20B5000003D11A6842F400721A602D059C4605D56FF4006347F00807CCF81430236C1F43C0
:20B52000276494F83D3094F83E20102ADBB27CD003F02802282A73D0DCF80420100504D4F3
:20B54000602B02D0202384F83D300023236384F83E30DCF8043013F400634ED0DCF8043037
:20B56000606B23F40063CCF8043090F83530012B00F0AB80824B0365FEF7D6FC50B12268D3
:20B58000606B1368016D23F001032025136084F83D508847236C1F0704D02268536823F46B
:20B5A000E063536094F83D30226C5607DBB202D5282B00F0A880F8BD10B1110ACF071AD48D
:20B5C000C5F380271FB1D105F5D5002787E72B05F1D5110A08E003276FF4007268055A61E7
:20B5E0003FF57DAF2A0504D5CE0791D4002FE2D023689C4692E70227EEE794F83D20602A71
:20B6000048D0DCF814305B0606D5636ADCF810201A70636A013363622046FFF7D7F9B9E7D1
:20B620000023236384F83D2093E7222B80D1DCF8003023F40063CCF80030DCF804301D05D4
:20B6400080D582E7CAB901F0F702212A03D0282913D1212811D194F83D20E16A0829D2B258
:20B660005ED020295CD0212A73D06FF480625A612805BBD5D4F800C04AE76FF4806247F0A3
:20B6800004075A6141E72A054FF001073FF540AF9C4643E7202284F83D202364DCF814305D
:20B6A0005A0608D5636ADCF810201A70636AD4F800C001336362DCF8003023F00103CCF8C1
:20B6C00000302046FFF784F964E7A06B2C4B0365FEF72AFC00283FF45DAF23685A69510605
:20B6E00006D5626A1B691370626A2368013262621A68A06B22F0010220211A60036D84F805
:20B700003D10984746E71F4BE362202200232363204684F83D2084F83E30FFF751F9F8BD18
:20B72000282AA0D1174AE2625A686FF4806122F4E0625A6059611A680A401A600021202325
:20B740002163204684F83D3084F83E10FFF738F98EE70C49E16220200021226384F83D0079
:20B7600084F83E105A686FF4806122F4E0625A6059611A680A401A602046FFF71BF977E719
:20B78000D5A900080000FFFFE8B138B5D0E9003182684CF6CC45044645F255501D6018605D
:20B7A00059609A60FEF778FA054604E0FEF774FA401B302809D82368D8680028F6D14AF64F
:20B7C000AA221A6038BD01207047032038BD00BF03684AF6AA221A6000207047002800F09F
:20B7E00032812DE9F0410368DD0782B004462FD5AC498A6802F00C02042A00F0EA808A681F
:20B8000002F00C02082A00F0E0806368B3F5803F00F0E980B3F5A02F00F07881A14D2A683B
:20B8200022F480322A602A6822F480222A60002B40F0DE80FEF730FA064605E0FEF72CFABE
:20B84000801B642800F2F2802B689B03F6D423689F0775D41A0715D56369002B00F0A580D1
:20B86000914B904D01221A60FEF716FA064605E0FEF712FA801B022800F2D8806B6F9B07B0
:20B88000F6D5236858073BD5864A136C13F0805340F0DB800193136C43F080531364136C24
:20B8A00003F080530193019B0126804D2A68D10540F1AC80A368012B00F0C980052B00F049
:20B8C0002F81784D2A6F22F001022A672A6F22F004022A67002B40F0BF80FEF7DDF941F2DA
:20B8E0008837804606E0FEF7D7F9A0EB0800B84200F29C802B6F9807F5D4002E40F0DC80C1
:20B90000A069C8B1674DAA6802F00C02082A00F0D980674A00210228116000F00B81FEF786
:20B92000BBF92C46054604E0FEF7B6F9401B02287CD823689B01F7D4002002B0BDE8F0815B
:20B94000584A916811F00C0F24D0916801F00C0108291CD0E368002B00F09280554B514D72
:20B9600001221A60FEF798F9064604E0FEF794F9801B02285AD82B689807F7D52B682269DF
:20B9800023F0F80343EAC2032B60236862E752685602DFD4434A126895074BD5E268012A4B
:20B9A00048D0012002B0BDE8F0813F4A3D4D1360FEF772F9064604E0FEF76EF9801B02284F
:20B9C00034D86B6F9F07F7D45BE74A6850027FF51CAF344A126891037FF53AAF6268002AAE
:20B9E0007FF436AFDDE72F4A136843F480331360FEF752F92B4D064604E0FEF74DF9801B1C
:20BA0000642813D82B689A03F7D520E72A6842F480722A60FEF740F907462B68DA053FF547
:20BA200049AFFEF739F9C01B0228F6D9032002B0BDE8F0811B4920690A6822F0F80242EA91
:20BA4000C0020A6006E70120704700262DE7154A136F43F001031367FEF71EF9114D8046F9
:20BA600041F2883705E0FEF717F9A0EB0800B842DCD82B6F9B07F6D5002E3FF441AF1BE056
:20BA80000C4A084D1360FEF707F9064604E0FEF703F9801B0228C9D82B689907F7D4236883
:20BAA000D8E600BF00380240800E4742007000406000474200004742354A136C23F0805372
:20BAC00013641DE701283FF46DAFAB68E26903F4800191427FF465AF226A03F03F019142B1
:20BAE0007FF45FAF47F6C072616A1A408A427FF458AFA26A03F4403191427FF452AFE06AE6
:20BB000003F07063181A18BF01204BE7204B1A6842F480221A601A6842F480321A6067E792
:20BB20001B4B1A6F42F004021A671A6F42F001021A6791E7FEF7B0F8064605E0FEF7ACF83F
:20BB4000801B02283FF672AF2B689901F6D4D4E90736D4E90902E16A0D4C334343EA801337
:20BB6000520843EA0163013A0A4943EA024301226B600A60FEF790F8054605E0FEF78CF85C
:20BB8000401B02283FF652AF23689A01F6D5D3E60038024060004742174908B58B6803F0DA
:20BBA0000C03042B1BD0082B17D14A684B6813F4800302F03F0214D149681048C1F38811E4
:20BBC000A1FB0001F5F768F80B4B5B68C3F3014301335B00B0FBF3F008BD084808BD084822
:20BBE00008BD4B680648C3F38813A3FB00010023F5F752F8E8E700BF003802400024F40016
:20BC000000127A0060B1494A136803F00F038B4208D2CBB21370136803F00F038B4201D0AF
:20BC20000120704703682DE9F0419D0714D55C0704D53F4CA26842F4E052A2601A0704D5B8
:20BC40003B4CA26842F46042A260394C8568A26822F0F0022A43A260DF0704460D4622D510
:20BC60004268012A57D0931E012B314B1B6859D9990725D52E4EB36823F003031343B36007
:20BC8000FEF70AF841F28837804605E0FEF704F8A0EB0800B84243D8B368626803F00C0390
:20BCA000B3EB820FF2D1214A136803F00F03AB4209D9EBB21370136803F00F03AB4202D079
:20BCC0000120BDE8F08123685A0706D51849E0688A6822F4E05202438A601B0712D4FFF756
:20BCE0005BFF134B134C9B681349144AC3F30313E35C20FA03F308681360FDF783FF0020DC
:20BD0000BDE8F0810A4A2169936823F4604343EAC1039360E3E7064B1B689E03AAD4CFE723
:20BD20000320EDE79801A5D4CAE700BF003C02400038024038FB0008380400202C000020AF
:20BD4000044B054A9B680549C3F382230868D35CD84070470038024048FB00082C0000201A
:20BD6000044B054A9B680549C3F342330868D35CD84070470038024048FB00082C0000202A
:20BD8000F0B50446006810F0050F83B00AD1850742D410F0080003D0484B227C1A600020E2
:20BDA00003B0F0BD464B474D00221A60FDF774FF064604E0FDF770FF801B022829D82B680F
:20BDC0001B01F7D4D4E901133D4A3E4E1B0743EA81130121C5F884301160FDF75DFF054616
:20BDE00004E0FDF759FF401B022812D833681F01F7D52068CBE70D46FDF74EFF41F288365E
:20BE000007462B6F9B073AD4FDF746FFC01BB042F7D9032003B0F0BD2A4B2B4D0022019290
:20BE20001A6C42F080521A641B6C03F080530193019B2B6843F480732B60FDF72DFF0646C9
:20BE400004E0FDF729FF801B0228E2D82B68D905F7D51C49E3680A6F12F4407203F440709E
:20BE600010D082420ED00B6F184A23F4407301250020156010600B670B6FDA07BBD4E368C8
:20BE800003F44070B0F5407F0CD00E498A6822F4F8128A600B4A116FC3F30B030B43136707
:20BEA000206876E70748826823F0704122F4F81221F440710A438260ECE700BFE01147427F
:20BEC000680047420038024000700040400E4742002846D0F8B590F83D30044603F0FF0252
:20BEE00033B32268284DA669E0686168022384F83D30AA42136836D0B2F1804F1DD0A5F5C9
:20BF00007C45AA4219D005F58065AA4215D005F58065AA4211D005F59A35AA4211D005F59F
:20BF20008065AA420DD005F58065AA420DD108E080F83C20FBF7C8FAD3E7A56823F07003ED
:20BF40002B43256923F440732B4323F0800333431360D062916201235361002084F83D3028
:20BF6000F8BD01207047A768256923F070033B4323F440732B4323F0800333431360D062AA
:20BF8000916263691363E6E7000001400222036810B580F83D20196A41F2111211420446BF
:20BFA00008D1196A40F24442114203D11A6822F001021A602046FBF715FC002084F83D00F3
:20BFC00084F83C0010BD00BF0223026880F83D30936803F00703062B03D0136843F00103FB
:20BFE0001360012380F83D30002070470368DA6842F00102DA609A6802F00702062A03D0D2
:020000040800F2
:20C000001A6842F001021A6000207047704700BF002846D0F8B590F83D30044603F0FF0284
:20C0200033B32268284DA669E0686168022384F83D30AA42136836D0B2F1804F1DD0A5F587
:20C040007C45AA4219D005F58065AA4215D005F58065AA4211D005F59A35AA4211D005F55E
:20C060008065AA420DD005F58065AA420DD108E080F83C20FFF7CAFFD3E7A56823F07003A1
:20C080002B43256923F440732B4323F0800333431360D062916201235361002084F83D30E7
:20C0A000F8BD01207047A768256923F070033B4323F440732B4323F0800333431360D06269
:20C0C000916263691363E6E70000014003680122186A01F01F0102FA01F120EA010010B43F
:20C0E00018621A6A0B4C1143A34219620CD09A6802F00702062A03D01A6842F001021A602A
:20C1000000205DF8044B70475A6C42F400425A64EDE700BF00000140002846D0F8B590F861
:20C120003D30044603F0FF0233B32268284DA669E0686168022384F83D30AA42136836D0D4
:20C14000B2F1804F1DD0A5F57C45AA4219D005F58065AA4215D005F58065AA4211D005F5FA
:20C160009A35AA4211D005F58065AA420DD005F58065AA420DD108E080F83C20FBF7B6FA74
:20C18000D3E7A56823F070032B43256923F440732B4323F0800333431360D0629162012356
:20C1A0005361002084F83D30F8BD01207047A768256923F070033B4323F440732B4323F049
:20C1C000800333431360D062916263691363E6E70000014090F83C30012B00F09580F0B4B5
:20C1E0000223012480F83C4080F83D30D1E900570368D1E9026472B3042A63D0082A1A6A44
:20C2000000F0848022F480521A62D969D3F820C021F4407124032A0341EA0721A4B202F420
:20C22000204221F470412CF4204C42EA0C020C43DC611A62DA6922F44062DA61DA6942EA63
:20C240000626DE610023012280F83D2080F83C30F0BC184670471A6ADFF8F0C022F0010293
:20C260001A62634599691A6A15D0B3F1804F12D0ACF57C4C63450ED00CF5806C63450AD07C
:20C280000CF5806C634506D00CF59A3C634502D041F0010102E021F003013943240122F005
:20C2A0000A07E4B221F0F00105F00A023A43214399611A629A6922F00C029A619A69164303
:20C2C0009E61BFE71A6A22F010021A629969D3F820C021F4407124032A0141EA0721A4B227
:20C2E00002F0A00221F470412CF0A00C42EA0C02214399611A629A6922F440629A619A694F
:20C3000042EA06269E619DE70220704722F480721A62D969D3F820C021F0030124012A0292
:20C320003943E4B202F4206221F0F0012CF4206C42EA0C022143D9611A62DA6922F00C020E
:20C34000DA61DA691643DE617CE700BF0000014090F83C30012B00F0C880F0B5022301241D
:20C3600080F83C4080F83D300C2A37D8DFE802F03E36363668363636933636360700036855
:20C380008F681D6A0E68DFF8C0C125F480551D621A6AD3F804E0DC6922F4005224F4E644C2
:20C3A000634542EA073244EA062404D14D692EF4804E4EEA851E4D68C3F804E0DC611D64B0
:20C3C0001A62DC690D6944F40064DC61D96921F48061D961DA6942EA0522DA6100230122C4
:20C3E00080F83D2080F83C301846F0BD0368D1F808E01D6A0F68544E25F001051D621A6A9F
:20C40000D3F804C09C6922F0020224F07304B34242EA0E0244EA070478D04D68C3F804C001
:20C420009C615D631A629C690D6944F008049C61996921F0040199619A692A439A61CDE7DA
:20C4400003688F681D6A0E68DFF8FCE025F010051D621A6AD3F804C09C6922F0200224F4BD
:20C46000E644734542EA071244EA06245CD04D68C3F804C09C619D631A629C690D6944F4B1
:20C4800000649C61996921F4806199619A6942EA05229A61A2E703688F681D6A0E68DFF839
:20C4A000A8E025F480751D621A6AD3F804C0DC6922F4007224F07304734542EA072244EAC1
:20C4C000060414D04D68C3F804C0DC61DD631A62DC690D6944F00804DC61D96921F00401B1
:20C4E000D961DA692A43DA6178E702207047D1E90575CE6822F400622CF4405C42EA0622ED
:20C500003D4322F480624CEA051CDBE7D1E90556CF6822F008022CF4407C3A43354322F03F
:20C52000040245EA0C0C78E7D1E90575CE6822F080022CF4406C42EA06123D4322F040026D
:20C540004CEA850C93E700BF0000014090F83C30012B5AD002220368F0B480F83D209A6846
:20C560000C6822F47F4222F077020125402C80F83C509A6074D04AD9602C2DD056D9702C9A
:20C580001AD0B4F5005F0ED1D1E90152CC6899682A4342EA042221F47F410A439A609A68AB
:20C5A00042F480429A600023012280F83D2080F83C30F0BC18467047D1E90152CC68996887
:20C5C0002A4342EA042221F47F410A439A609A6842F077029A60E6E71C6A4D68CE6824F087
:20C5E00010041C6299691A6A21F4704122F0A00242EA051241EA063199611A629A6822F07A
:20C60000700242F067029A60CDE702207047102C04D03DD9202C01D0302CC4D19A6844F01C
:20C62000070422F0700214439C60BCE7502CBAD11D6A1E6A4C68CF6826F001061E629A69D4
:20C6400025F00A0122F0F00242EA071221439A6119629A6822F0700242F057029A60A2E703
:20C660001D6A1E6A4C68CF6826F001061E629A6925F00A0122F0F00242EA071221439A6158
:20C6800019629A6822F0700242F047029A608AE7002CC3D087E700BF90F83C30012B47D090
:20C6A00002680223F0B480F83D30D1E90065936823F070032B43044623F007033343012056
:20C6C000502D84F83C0093604ED01FD9602D38D0702D0AD1D1E90253086991682B4343EAFB
:20C6E000002321F47F410B439360D36823F04003D360D3680125002123F48043D360084660
:20C7000084F83D5084F83C10F0BC7047402DECD1052E0FD0156A106A0E6920F001001062B6
:20C72000936923F0F00343EA061393611562DCE702207047002384F83D0084F83C30F0BC3A
:20C740007047106A8D680E6920F0100010629169136A21F4704123F0A00341EA063143EA28
:20C76000051391611362C0E7156A166A88680F6926F001061662936925F00A0123F0F00375
:20C78000014343EA071393611162AEE7704700BF704700BF704700BF704700BF704700BFC4
:20C7A00003681A69910710B5044602D5DA6892075FD41A69500702D5DA68510746D41A6917
:20C7C000120702D5DA6810072ED41A69D20602D5DA68D00618D41A69D10702D5DA68D2078B
:20C7E0005DD41A69100602D5DA6811065FD41A69520602D5DA68500661D41A69910602D59C
:20C80000DA68920643D410BD6FF010021A61DB69082213F4407F2277204664D0FFF7BAFF58
:20C82000002223682277D6E76FF008021A61DB69042299072277204652D1FFF7A9FF2046E1
:20C84000FFF7AAFF002223682277BEE76FF004021A619B69022213F4407F227720463CD174
:20C86000FFF796FF2046FFF797FF002223682277A5E76FF002021A619B6901229B07027749
:20C8800025D0FFF787FF00222368227791E76FF0200220461A61BDE8104000F069B86FF0A2
:20C8A00001021A612046FFF771FF236899E76FF080021A61204600F05DF8236897E76FF0B4
:20C8C00040021A612046FFF769FF236895E7FFF75FFF2046FFF760FFD5E7FFF75BFFC4E70A
:20C8E000FFF758FFAEE7FFF753FF2046FFF754FF96E700BF90F83C30012B32D00368022272
:20C9000070B480F83D205A680E68174D9C6822F070023243AB424FF0010680F83C605A6084
:20C9200011D0B3F1804F0ED0104A93420BD002F58062934207D002F58062934203D002F5BE
:20C940009A32934204D14A6824F0800414439C600023012280F83D2080F83C3070BC18463B
:20C9600070470220704700BF0000014000040040704700BF704700BF002800F0938090F844
:20C98000393070B503F0FF020446002B00F0858023682669242284F83920D86820F40050D2
:20C9A000D4E90225D8601969E06921F4405129431961D9686569324321F416412A4321F096
:20C9C0000C0102430A43DA605A69A16922F440720A43B0F5004F5A61364A34D0934263D061
:20C9E00002F5806293425FD0FFF7AAF96368324D1922A0FB02019A009B0FF4F74DF9A5FB89
:20CA000000214909642202FB1102120132322368A5FB0202090101EB52129A601A6922F47A
:20CA200090421A615A6922F02A025A61DA680025202142F40052DA602846E56384F8391008
:20CA400084F83A1070BD934231D002F5806293422DD0FFF775F96268002692184FF019010B
:20CA600046EB0603A0FB0101F4F716F9124E2368A6FB00214D09642202FB1502D200323212
:20CA8000A6FB0212520902F00701520001EB051102F4F8720A449A60C0E780F83820FAF728
:20CAA00015FF75E701207047FFF75AF99EE7FFF757F9D0E7001001401F85EB512DE9F041EB
:20CAC0000E4690F83910202982B032D1002E34D00192002A31D01F4690F83830012B0446F8
:20CAE00027D04FF0000801212123C0F83C8080F8381080F83930FDF7CFF8019AA284E2849B
:20CB0000226884F838800546E38C9BB2002B3BD0E08CA168013880B2B1F5805FE0841BD066
:20CB2000781C3BD110680106FCD5337853600136EAE7022002B0BDE8F081012002B0BDE83D
:20CB4000F08113681B060CD4002F31D0FDF7A4F8401B874222682BD3781CF2D110680106A6
:20CB6000FCD533882169C3F3080353600029DED10236C9E713685B060BD4CFB1FDF78CF8B8
:20CB8000401B8742226813D3781CF3D113685906FCD5202384F839300020CBE713681B0668
:20CBA000C3D42FB1FDF778F8401B87422268B7D2D36823F4D073D3605369202123F0010387
:20CBC00000250320536184F8391084F8385084F83A1002B0BDE8F08190F83930202B18D1DD
:20CBE000C9B1C2B190F83830012B12D030B400230568C2842124C36380F83940EC6801627D
:20CC000044F08004828480F838301846EC6030BC7047022070470120704700BF90F83A30C7
:20CC2000202B20D109B302B390F83830012B1AD030B400230468C2852225C36380F83A5018
:20CC4000E568828545F48075816280F83830E560626942F001026261E26842F0200218468B
:20CC6000E26030BC7047022070470120704700BF704700BF10B584680169836A0268B4F5CE
:20CC8000805F20D05C1C52688462C9B91A70C38D013B9BB2C3858BB90268D16821F0200167
:20CCA000D160D16821F48071D1605169202421F00101516180F83A40F4F7B2FF002010BD95
:20CCC00002F07F02E2E7526829B9C2F3080223F8022B8362DBE7D2B223F8012B8362D6E761
:20CCE000704700BF03681A6870B51607DD685969044646D011F001014CD0D00705D5EE0565
:20CD000003D5E06B40F00100E063500774D529B1E06B960740F00200E06371D4160703D56B
:20CD2000A80672D4002970D1E16B002931D0960601D5A80672D45D69E16B090702D415F0BC
:20CD4000400578D0DA6822F49072DA605A69202122F001025A6184F83A105A69520659D5CF
:20CD60005A69606B22F040025A61002852D03A4B0365FDF7D9F860B1606BBDE87040036D79
:20CD80001847910609D5AE0607D590F83A30222B4DD070BD15F4907FAFD116060ED45106B9
:20CDA000F7D56A06F5D5DA68202122F04002DA60204684F83910FFF75BFF70BD2806EED5C3
:20CDC00094F83920212AE4D1A168226AB1F5805F36D0511C216212785A60E28C013A92B22D
:20CDE000E284002AD5D1DA6822F08002DA60DA6842F04002DA6070BD90078FD500298DD04F
:20CE0000E06B40F00400E06388E7E16B41F00801E16389E72046FFF763FF70BD94F83A20D6
:20CE2000222A88D12046FFF725FF236883E7BDE87040FFF71FBF2046FFF752FFE56370BD8D
:20CE400011882069C1F30801596010B902322262C3E701322262C0E75DCE000808B5836BD3
:20CE60000022DA851846DA84FFF73AFF08BD00BF014B1868704700BF3C04002070B50D4EA0
:20CE80000D4CA41BA4100025A54209D10B4E0C4C02F0F6F8A41BA4100025A54205D170BDCD
:20CEA00056F8253098470135EEE756F8253098470135F2E70852010808520108085201082B
:20CEC0000C52010802440346934200D1704703F8011BF9E72DE9FF4755EC104B0D9FDDF88F
:20CEE00030A0002D0E4691461946B8BF22462B4627F02007BBBF05F100431D4600232D2394
:20CF0000B8BF1446462F0B7004D0452F00D10136022100E0032103AB019302AB00933246DF
:20CF2000534645EC104B00F077FD472F804602D119F0010F26D0462F08EB060911D198F861
:20CF40000030302B0AD10022002320462946F3F7C3FD18B9C6F10106CAF80060DAF80030F4
:20CF600099440022002320462946F3F7B5FD38B93022039B4B4505D2591C03911A70F8E764
:20CF8000CDF80C90039B0E9AA3EB08034046136004B0BDE8F087F7B500290446BABF494265
:20CFA0002D232B23092904F8022B437020DD0DF107031F460A2691FBF6F506FB151130312C
:20CFC000092D03F8011C03F1FF32294609DC3031023B02F8011CBB42224604D3101A03B0BC
:20CFE000F0BD1346E7E713F8012B04F8012BF2E7302319448370021DC170EFE72DE9F04F07
:20D000008DB00C46DDF8588016461F46054601F0BBFA036804931846F3F7E2F800230A933E
:20D02000D8F800300590073323F0070303F1080294F818A0D4F800B0C8F80020D3E9002387
:20D04000C4E91223D4E9128929F000430793CDF818804FF0FF32A74BDDE90601F3F76EFDBF
:20D0600070BB4FF0FF32A34BDDE90601F3F748FD30BB0022002340464946F3F737FD10B107
:20D080002D2384F843309C4A9C4BBAF1470F8CBF9046984603232BF00402236122604FF0F8
:20D0A0000009009733460BAA2146284600F0E6F9013040F08D804FF0FF300DB0BDE8F08F41
:20D0C00042464B4640464946F3F738FD10B18C4A8C4BDAE761684B1C4BF480620AA83ED1C2
:20D0E000062363600023CDE9020309AB009349EC108B0DF123032260CDF804A06168284609
:20D10000FFF7E8FE0AF0DF03472B804609D1099BD81C02DB6268934247DDAAF1020A5FFA0D
:20D120008AFABAF1650F099924D80139524604F150000991FFF72FFF0A9A1318012A814618
:20D14000236102DC2268D10701D5013323619DF82330002BA5D02D2384F84330A1E7BAF183
:20D16000670F00F07781BAF1470FBBD10029B9D10123B6E7BAF1660F19D1002963680CDD69
:20D18000216113B92268D20702D501330B442361099BA3654FF00009D9E713B92268D0071F
:20D1A00001D50233F3E70123F1E74FF0670ADDE90932934205DB22682361D107E8D5013351
:20D1C000E5E7002BD4BFC3F1020301231344DEE723685A0507D42369424631462846B8470F
:20D1E00001302BD167E7BAF1650F40F2DC8000220023D4E91201F3F76FFC002833D001234E
:20D20000414A31462846B84701303FF454AFDDE909239A4202DB2368D8070FD5DDE9042352
:20D2200031462846B84701303FF445AF4FF0000804F11A090A9B013B434509DC23689B07D8
:20D2400000F10381E0680B9B9842B8BF184634E701234A4631462846B84701303FF42BAFCB
:20D2600008F10108E6E7099B002B2BDC0123264A31462846B84701303FF41DAF099B23B9E1
:20D280000A9B13B92368D907D8D5DDE9042331462846B84701303FF40EAF4FF0000904F1D6
:20D2A0001A0A099B5B424B4501DC0A9B94E70123524631462846B84701303FF4FCAE09F1D4
:20D2C0000109EEE70A9AA36D9A42A8BF1A46002A914607DD1346314642462846B84701303D
:20D2E0003FF4E9AE04F11A034FF0000B29EAE979069315E0FFFFEF7FA84F0108A44F01089D
:20D30000B04F0108AC4F0108B44F01080123069A31462846B84701303FF4CDAE0BF1010B66
:20D32000D4F858A0AAEB09035B45EFDCDDE909239A42D04415DB2368DA0712D40A9B0999B2
:20D34000A3EB0A02A3EB010A9245A8BF9246BAF1000F0EDC4FF000082AEAEA7A04F11A0909
:20D3600019E0DDE9042331462846B8470130E5D1A1E65346424631462846B8470130E9D185
:20D3800099E601234A4631462846B84701303FF492AE08F10108DDE909239B1AA3EB0A038E
:20D3A0004345EEDC4AE70A9A012A01DCDB073AD50123424631462846B84701303FF47BAE30
:20D3C000DDE9042331462846B847013008F101083FF471AE0A9B002203F1FF3AD4E9120133
:20D3E0000023F3F779FBC8B95346424631462846B84701300ED15EE6012352463146284631
:20D40000B84701303FF457AE08F101080A9B013B4345F1DC4B4604F15002DEE64FF0000889
:20D4200004F11A0AF2E70123DFE701234A4631462846B84701303FF43EAE08F10108E368DB
:20D440000B9A9B1A4345F0DCFCE64FF0000804F11909F4E700293FF48BAE0023CDE9020390
:20D4600009AB009349EC108B2260CDF804A00DF123032846FFF72EFD804648E62DE9F047B6
:20D4800091461F468A680B69DDF820809342B8BF1346C9F8003091F8432006460C4612B192
:20D4A0000133C9F800302368990642BFD9F800300233C9F80030256815F0060507D104F18B
:20D4C000190AE368D9F800209B1AAB4228DC94F843302268003318BF012392062DD404F102
:20D4E000430239463046C047013020D02368E568D9F8002003F00603042B08BFAD1AA3683D
:20D5000022690CBF25EAE57500259342C4BF9B1AED184FF000091A344D451AD1002008E0FA
:20D520000123524639463046C047013003D14FF0FF30BDE8F0870135C3E7E1185A1C302005
:20D5400081F84300224494F8451082F843100233C5E70123224639463046C0470130E6D0AB
:20D5600009F10109D8E700002DE9F04301F1430C0C46097E85B06E291746064698460C9A8C
:20D5800000F0B38022D8632936D00AD8002900F0B980582900F0838004F1420584F842102A
:20D5A00032E0642901D06929F6D120681368050603F104012AD51B681160002B03DA2D2251
:20D5C0005B4284F843206F480A2239E0732900F09D8008D86F2920D07029DDD1236843F0BD
:20D5E0002003236003E0752917D07829D4D1782384F84530644855E01368191D1B681160C5
:20D6000004F1420584F8423001238CE01B68116010F0400F18BF1BB2CFE713682568181D76
:20D620001060280601D51B6802E06806FBD51B8854486F2914BF0A220822002184F84310E3
:20D640006568A560002DC0F29580216821F004012160002B3DD1002D40F08E806546082A63
:20D660000BD12368DB0708D5236962689A42DEBF302305F8013C05F1FF35ACEB05032361DB
:20D68000CDF800803B4603AA21463046FFF7F6FE01304DD14FF0FF3005B0BDE8F083394845
:20D6A00084F84510136821681D1D1B6815600A060BD5CA0744BF41F0200121601BB922686E
:20D6C00022F0200222601022B7E74D0648BF9BB2EFE76546B3FBF2F102FB1133C35C05F8AE
:20D6E000013D0B460029F5D1B9E7136825686169181D106028061B6801D5196002E06A0643
:20D70000FBD51980002323616546B9E71368191D11601D68626800212846F2F769FD08B1A6
:20D72000401B606063682361002384F84330A7E723692A4639463046C0470130AAD02368B1
:20D740009B0713D4E068039B9842B8BF1846A3E701234A4639463046C04701309AD00135A0
:20D76000E368039A9B1AAB42F2DCEBE7002504F11909F5E7002BACD1037884F8423004F161
:20D7800042056CE7B64F0108C74F010838B50D4B1C68A36B05467BB9182000F003FF0A4AEE
:20D7A0000A4BA063C0E90023094B83600B23838101220023C0E90423A36B00221D615A615D
:20D7C00038BD00BF3C0400200E33CDAB34126DE6ECDE050038B5134B1C68A36B7BB91820CB
:20D7E00000F0E0FE104A114BA063C0E90023104B83600B23838101220023C0E90423A16B44
:20D800000C480A694B690C4C504304FB0300A2FB04230344541C43F10005C1E9044525F0E4
:20D82000004038BD3C0400200E33CDAB34126DE6ECDE05002DF451582D7F954C0EB400B564
:20D840009CB01DAB029006906FF00041094807910491094953F8042B05910068019302A965
:20D8600001F09EFA029B00221A701CB05DF804EB03B070473C0400200802FFFF034611F8A2
:20D88000012B184603F8012B002AF8D1704710B503461A785C1C3AB9013B11F8012B03F8B6
:20D8A000012F002AF9D110BD2346F2E710B56AB10139841810F8013B11F8012F934203D159
:20D8C000A04201D0002BF5D1981A10BD1046FCE770B50139044602B970BD234611F8015F89
:20D8E00003F8015B561E2DB91444A342F4D003F8015BFAE71C463246EDE72DE9F74F0369C8
:20D900000C69A3428046C0F28280013C01F114074FEA840C00F1140657F8245056F82400E0
:20D9200006EB0C03013507EB0C090193B0FBF5F595B34FF0000A3846B646D34650F8042BE6
:20D9400093B205FB03A34FEA134A9BB2ABEB0303120CDEF800B005FB02A213FA8BF34FEA51
:20D96000124A1FFA82FBDEF80020CBEB124202EB23429BB243EA024381454FEA224B4EF8F2
:20D98000043BDBD256F80C3033B9019B043B9E421A4630D3C8F81040404601F02BF8002835
:20D9A00025DB013530464FF0000C57F8042BD0F800E093B2ACEB0303120C13FA8EF3C2EB0F
:20D9C0001E4202EB23429BB243EA0243B9454FEA224C40F8043BE8D256F8242006EB8403F6
:20D9E0002AB9043B9E421A460BD3C8F81040284603B0BDE8F08F1268043B002ACAD1013CD7
:20DA0000C5E71268043B002AEFD1013CEAE70020EEE70000000000002DE9F04F57EC106BA1
:20DA200097B0456A069104460B921293DDF88080CDE900673DB9102000F0B4FD6062C0E9A9
:20DA400001550560C560636A196851B15A684A60012393408B60204600F0EBFD636A00221B
:20DA60001A603B1EBBBF23F00043019300230122ACBFC8F80030C8F80020AF4BDDF804809B
:20DA800033EA080314D1129A42F20F731360009B23B9C8F31300002800F04285219BDFF8ED
:20DAA000ACB2002B00F044850BF1030300F03EBDDDE900670022002330463946F3F70CF8E2
:20DAC000814668B1129A01231360219B002B00F024859A4B219A03F1FF3B136000F028BD8D
:20DAE00014AA15A947EC106B204600F0FAFFC8F30A550490002D7CD0C7F3130343F07F5BA9
:20DB0000B2464BF4401BA5F2FF35CDF84C9000228B4B50465946F2F7BFFB81A3D3E9002334
:20DB2000F2F772FD80A3D3E90023F2F7B7FB064628460F46F2F7FEFC7DA3D3E90023F2F716
:20DB400063FD02460B4630463946F2F7A7FB06460F46F3F709F800228246002330463946BE
:20DB6000F2F7C4FF48B15046F2F7E4FC32463B46F2F7B2FF08B90AF1FF3ABAF1160F59D818
:20DB8000704901EBCA01DDE90023D1E90001F2F7CBFF002850D00AF1FF3A00230F93149BCE
:20DBA0005D1BB5F1010849BFC5F10103002305934FF0000858BF0593BAF1000F3EDB0023D5
:20DBC000D044CDF838A00793069B092B00F29080052BC4BF043B0693069BA3F10203CCBFD3
:20DBE00000250125032B00F28F80DFE803F07D7F3171DDE914531D4405F23240202813DD24
:20DC0000C0F14000009B08FA00F805F2124023FA00F048EA0000F2F77DFC01238246A1F116
:20DC2000F87B013D139372E7009BC0F1200003FA00F0F0E70123B1E70F90B0E7059BA3EBE4
:20DC40000A030593CAF10003079300230E93BBE701230A930B9B002B59DD02939946666A55
:20DC600000227260042202F114009842716853D9204600F0AAFC636A3060B9F10E0FD3F8B9
:20DC800000B000F2E680002D00F0E3809DED007BBAF1000F8DED107B74DD2A4A0AF00F0367
:20DCA00002EBC30393ED007B4FEA2A16F0068DED087B65D5244BDDE91001D3E90823F2F7FA
:20DCC000CDFDCDE9000106F00F0603251E4F4CE001230A930B9B534403F1010902934B46D5
:20DCE000012BB8BF0123BAE70023B2E70023F0E70125002306930A954FF0FF3302939946A0
:20DD0000002212230B92AAE701230A93F4E70123029399461A46F5E7013171605200A2E730
:20DD200061436F63A787D23FB3C8608B288AC63FFB799F501344D33F0000F07FB54F0108C9
:20DD40000000F83F10500108E84F0108E14F0108F10708D5DDE90801D7E90023F2F754FCEA
:20DD6000CDE90801013576100837002EF0D1DDE90823DDE90001F2F771FDCDE900011AE03A
:20DD80000225A3E700F0A080CAF100069F4BA04F06F00F0203EBC203D3E90023DDE91001B8
:20DDA000F2F732FCCDE90001361100230225002E7FD1002BE1D10F9B002B00F08780DDE917
:20DDC00000670022934B30463946F2F78FFE00287CD0B9F1000F79D0029B002B35DD0AF126
:20DDE000FF330893394600228B4B3046F2F70CFCCDE90001029F01352846F2F79BFBDDE937
:20DE00000023F2F701FC0022844BF2F747FA0546A1F15076002F5DD10022814BDDE9000129
:20DE2000F2F73AFA2A463346CDE90001F2F77CFE002840F088822A4606F10043DDE90001EF
:20DE4000F2F754FE002840F07C82DDE91023CDE90023159B002BC0F25081BAF10E0F00F346
:20DE60004C816A4B03EBCA0393ED007B0B9B002B8DED027B80F2D880B9F1000F00F3D480D8
:20DE800040F05E820022664B51EC170BF2F7BCFBDDE90023F2F73EFE4F464E46002840F011
:20DEA000348231230BF101058BF800300AF1010A2FE2F20705D5D7E90023F2F7A5FB013517
:20DEC00001237610083772E7022574E7CDF820A04F4691E74D4B03EBC70353E902010A9BB8
:20DEE000002B47D002460B4600204E49F2F7B6FC2A463346F2F7D0F9CDE90C015D46DDE92E
:20DF00000001F2F731FE0646F2F714FB02460B46DDE90001F2F7C0F9303605F8016BDDE90D
:20DF20000C23CDE90001F2F7E1FD002863D1DDE9002300203749F2F7AFF9DDE90C23F2F7E0
:20DF4000D5FD002840F0B780A5EB0B039F427FF77CAF0022304BDDE90C01F2F755FB002275
:20DF6000CDE90C012C4BDDE90001F2F74DFBCDE90001C4E72A463346F2F746FBCDE90C0137
:20DF80000BEB07055E46DDE90001F2F7EDFD0746F2F7D0FA303702460B46DDE90001F2F791
:20DFA0007BF906F8017BAE42CDE900014FF0000226D11C4BDDE90C01F2F770F902460B466F
:20DFC000DDE90001F2F7B0FD002874D1DDE90C2300201449F2F760F902460B46DDE9000163
:20DFE000F2F784FD00283FF430AF15F8013C302B05F1FF3202D0DDF820A04AE01546F4E7EA
:020000040800F2
:20E00000054BF2F701FBCDE90001BCE710500108E84F01080000F03F0000244000001C40D9
:20E02000000014400000E03FDDE900675D46DDE9022330463946F2F711FCF2F795FD804686
:20E04000F2F778FADDE90223F2F7DEFA02460B463046394608F13006F2F71EF905F8016B93
:20E06000A5EB0B06B14502460B4639D1F2F716F9DDE9022306460F46F2F756FDC8B9DDE95F
:20E08000022330463946F2F727FD10B118F0010F0FD10499204600F0CCFA0023129A2B707D
:20E0A0000AF101031360219B002B00F041821D603EE2CDF820A015F8012C392A05F1FF336D
:20E0C00008D19B450AD1089B0133089330238BF800305B461A7801321A708CE71D46EAE79D
:20E0E00000229B4BF2F790FA0022002306460F46F2F7F2FC00289AD0CBE70A9A002A00F0E6
:20E100008B80069A012A6EDC139A002A67D003F23343079F059D059A01211A442046059202
:20E12000984400F026FB0646002D0CDDB8F1000F09DD4545059A2B46A8BF4346D21A0592E5
:20E14000ED1AA8EB0308079BEBB10A9B002B67D08FB131463A46204600F0AAFB049A0146BE
:20E160000646204600F00EFB04990890204600F060FA089B0493079BDA1B04D00499204667
:20E1800000F096FB04900121204600F0F2FA0E9B0746002B00F0D0811A460146204600F0A7
:20E1A00087FB069B012B074640DC009B002B39D1019BC3F31303002B36D1019B23F000434B
:20E1C0001B0D1B052BB1059B0133059308F10108012307930E9B002B2AD1012030E0149B40
:20E1E000C3F1360395E7079B09F1FF37BB42BFBF079B0797FA1A0E9BBBBF9B180E93DF1BA4
:20E200000027B9F1000FB5BF059B059DA3EB09054B46B8BF00237EE7079F059D0A9E83E7E2
:20E22000079AABE70023D4E7009BD2E7002307933B6907EB8303186900F04DFAC0F1200017
:20E24000404410F01F0047D0C0F12003042B3BDD059BC0F11C000344059305448044059BF0
:20E26000002B05DD1A460499204600F06FFB0490B8F1000F05DD39464246204600F066FBE8
:20E2800007460F9B53B33946049800F0B3FB002824DA00230A220499204600F0E1F90A9BE1
:20E2A00004900AF1FF3A002B00F04D81002331460A22204600F0D4F9029B002B06464FDC85
:20E2C000069B022B4CDD11E0C9D0059A1C331A4405921D449844C2E70346F6E7B9F1000F15
:20E2E00038DC069B022B35DDCDF80890029B63B939460522204600F0B3F90146074604983C
:20E3000000F078FB00283FF7CCAD0B9B5D466FEA030A4FF000093946204600F08AF9002E46
:20E320003FF4B7AEB9F1000F05D0B14503D04946204600F07EF93146204600F07AF9A8E6C4
:20E3400000273E46E1E7DDF820A03E46A9E500BF000024400A9BCDF80890002B00F0FA80E9
:20E36000002D05DD31462A46204600F0EFFA0646079B002B4CD07168204600F026F932694A
:20E3800002320546920006F10C010C3000F012F901222946204600F0D9FA009BCDF814B052
:20E3A00003F00103B1460793064639460498FFF7A4FA4946054600F13008049800F01AFB36
:20E3C000324600903946204600F02EFBC368024603BB01460890049800F00CFB089A0346A9
:20E3E00011462046089300F024F9089BA3B9069A92B9079A82B9B8F1390F29D0009B002B42
:20E4000001DD05F13108059B5D1C83F8008082E73046C2E70123E3E7009A002A04DB25D1CC
:20E42000069A1ABB079A0ABB002BECDD01220499204600F08BFA3946049000F0DBFA002872
:20E4400003DCE0D118F0010FDDD0B8F1390FD8D1059B059A5D1C3923137015F8013C392B88
:20E4600005F1FF324FD00133137054E7059A002B02F1010506DDB8F1390FE9D008F1010812
:20E48000059BC2E7029A05F8018CA5EB0B03934221D000230A220499204600F0E1F8B14598
:20E4A00004904FF000034FF00A024946204605D100F0D6F881460646059576E700F0D0F8F0
:20E4C0003146814600230A22204600F0C9F80646F2E74FF0000901220499204600F036FAE5
:20E4E0003946049000F086FA0028B6DC02D118F0010FB2D115F8013C302B05F1FF327FF432
:20E500000AAF1546F6E7934505D131230AF1010A8BF80030FFE615469FE7DFF864B007E0B7
:20E52000219BDFF860B01BB10BF10803219A1360584617B0BDE8F08F069B012B7FF735AE88
:20E540000E9B079349E6029B002B03DC069B022B3FF7CCAE5D4639460498FFF7CEF900F1B8
:20E56000300805F8018B029AA5EB0B039A42B0DD00230A220499204600F072F80490EAE726
:20E58000B44F0108D84F0108044B1B68186A044B002808BF1846F030704700BF3C04002059
:20E5A000A0040020024B0146186800F045BB00BF3C04002010B5431E0A44914200D110BD8F
:20E5C00011F8014B03F8014FF7E770B5456A04460E463DB91020FFF7E5FF6062C0E901558A
:20E5E0000560C560656AEB6883B1636ADB6853F82600B8B9012101FA06F56A1D92002046B2
:20E6000000F0BEFA60B1C0E901650EE021220421204600F0B5FA636AE860DB68002BE4D19F
:20E62000002070BD026843F826200023C0E90333F7E770B5446A06460D463CB91020FFF735
:20E64000B1FF7062C0E901440460C4603DB1736A6A68DB6853F82210296043F8225070BD02
:20E660002DE9F0410D691F4606460C4601F1140C0023DCF8000081B202FB01710F0C000C08
:20E6800002FB007089B2013301EB00419D424FEA10474CF8041BECDCD7B1A368AB4212DC69
:20E6A000616830460131FFF790FF2269023204F10C01804692000C30FFF77CFF21463046C1
:20E6C000FFF7B7FF444604EB850301355F6125612046BDE8F081020C12040346B2B90304B6
:20E6E000102013F07F4F04BF1B02083013F0704F04BF1B01043013F0404F04BF9B0002300A
:20E70000002B06DB5B0003D5013070470020E8E720207047036813F0070201460BD0DA0772
:20E7200023D4980749BF5B089B0801200B605CBF0B600220704798B2A8B91B0C102013F045
:20E74000FF0F04BF1B0A08301A0704BF1B0904309A0704BF9B080230DA0702D45B0806D026
:20E7600001300B6070471046E9E7002070472020704710B50C460121FFF727FF0122446135
:20E78000026110BD2DE9F74F14460A6923699A42B8BF0B468846BCBFA0461C46D8F810700F
:20E7A000D4F81090D8F80830D8F8041007EB0906B342B8BF0131FFF708FF00F1140505EB6B
:20E7C000860E2B460022734516D304F1140208F1140102EB890301EB87070093009B0192A4
:20E7E00093420CD8002E03DD5EF8043D002B5DD0066103B0BDE8F08F43F8042BE3E7B2F847
:20E8000000B0BBF1000F23D08946AC464FF0000859F8044BDCF800A0A3B21FFA8AFA0BFB86
:20E8200003A34FEA144ADCF8004043444FEA14480BFB0A8404EB1344E2469BB243EA0443A8
:20E840004F454FEA14484AF8043B2BD8CCF80480019BB3F802A00432BAF1000F20D02B6867
:20E860008946A8464FF0000BB9F800C0B8F802400AFB0C445C44C4469BB243EA04434CF82A
:20E88000043B59F8043BB8F804B01B0C0AFB03B303EB14434F454FEA134B05D8C8F8043022
:20E8A00004359BE7D446B3E7E046DDE7013E99E72DE9F843154612F0030206460F4607D015
:20E8C000013A214C002354F82220FFF7C9FE0746AD1035D0746A3CB91020FFF763FE7062E7
:20E8E000C0E901440460C460D6F82480D8F808404CB940F271213046FFF73BFF0023C8F8C6
:20E900000800044603604FF00008EB070AD5394622463046FFF736FF394681463046FFF7F0
:20E9200088FE4F466D100BD0206838B9224621463046FFF727FF2060C0F800800446E4E7BD
:20E940003846BDE8F88300BFD85001082DE9F0470C464FEA621A236949680AEB0309A3688C
:20E960000746164609F10105AB4232DB3846FFF72CFE0023804600F114011A4653452BDB69
:20E9800020692AEAEA7A04F1140316F01F0201EB8A0103EB800C25D0C2F1200E00201E68D6
:20E9A0008A46964030434AF8040B53F8040B9C4520FA0EF014D8486008B109F10205013D0E
:20E9C0003846C8F810502146FFF733FE4046BDE8F08701315B00C7E741F823200133CDE7CA
:20E9E0005146DCE7043953F8042B41F8042F9C45F9D8E4E703690A699B1A30B50CD1920035
:20EA0000143014318418114454F8045D51F8042D954203D005D30123184630BDA042F3D3BC
:20EA2000FAE74FF0FF33F7E72DE9F0470D460746114628461446FFF7DDFF061E08D1314654
:20EA40003846FFF7C2FD0123C0E90436BDE8F087A4BF23462C4638466168A6BF1D460026ED
:20EA60000126FFF7B2FD2B69C660266905F1140904F1140202EB860709EB830800F1140560
:20EA80004FF0000E52F804AB59F8044B1EFA8AF1A3B2C91A230CC3EB1A4303EB214389B2FE
:20EAA0004FEA234EC84541EA0343944645F8043BE8D8BC4504D355F8043D83B10661C5E76B
:20EAC0005CF8041B1EFA81F31A1402EB11429BB243EA02434FEA224E45F8043BE9E7013ED6
:20EAE000E9E72DE9F7430E46012159EC108B1546FFF76BFDC9F30A540746C9F3130334BBBF
:20EB00000193B8F1000327D002A840F8083DFFF701FE0099F0B1019AC0F1200302FA03F307
:20EB20000B43C2407B610192019BBB61002B14BF022101213961C4B1A4F233440444346023
:20EB4000C0F135002860384603B0BDE8F08343F48013D5E77961E7E701A8FFF7DBFD019BBD
:20EB60007B61012139612030E5E707EB8103A0F2324030601869FFF7AEFDC0EB4110E1E7F1
:20EB800038B502FB01F4214600F056F8054618B122460021FEF796F9284638BD38B5054635
:20EBA000002945D051F8043C0C1F002BB8BFE41800F029FA1F4A1368104633B96360146055
:20EBC0002846BDE8384000F01FBAA3420CD921686218934204BF1A685B68636004BF521847
:20EBE00022600460ECE713465A680AB1A242FAD919685818A0420BD120680144581882421F
:20EC00001960DDD1106852685A6001441960D7E702D90C232B60D3E7206821188A4204BFC6
:20EC200011685268626004BF091821605C60C7E738BD00BFD819002070B5CD1C25F0030520
:20EC400008350C2D38BF0C25002D064601DBA94203D90C233360002070BD00F0D4F9214AC3
:20EC60001468214691B9204C23681BB9304600F08FF920602946304600F08AF9431C24D182
:20EC80000C233360304600F0BFF9E4E70B685B1B18D40B2B0FD90B60CD50CC18304600F004
:20ECA000B3F904F10B00231D20F00700C31AD3D05A42E250D0E78C424B6816BF63601360C0
:20ECC0000C46EBE70C464968CCE7C41C24F00304A04205D0211A304600F05AF90130CFD0E4
:20ECE0002560DBE7D8190020DC1900202DE9F0478E689E4282460C469046994637D88A8993
:20ED000012F4906F31D0256809696F1A6569022305EB450595FBF3F509F101033B449D4264
:20ED200038BF1D46530530D52946FFF785FF064650B90C23CAF80030A38943F04003A381F7
:20ED40004FF0FF30BDE8F0873A462169FFF732FCA38923F4906343F08003A381266165619E
:20ED60003E44ED1B2660A5604E464E4500D94E4632464146206800F02DF9A3689B1BA36089
:20ED800023681E4426600020DCE72A4600F03DF906460028E2D121695046FFF7FFFEC8E79E
:20EDA0002DE9F04F1D468B891F069DB080460C4616460FD50B696BB94021FFF73DFF206012
:20EDC000206128B90C23C8F800304FF0FF30C8E0402363610023099320238DF82930302342
:20EDE0008DF82A3003954FF0010B37463D4615F8013B0BB1252B3ED1B7EB060A0BD05346C7
:20EE0000324621464046FFF771FF013000F0A480099B534409933B78002B00F09D800023FD
:20EE20004FF0FF32CDE90523049307938DF853301A932F46052217F8011B5048F1F7D8F986
:20EE4000049BD0B9D90644BF20228DF853201A0744BF2B228DF853202A782A2A15D0079A89
:20EE60002F4600200A25394611F8013B303B092B4DD9B8B10FE02F46B8E7404A801A0BFAB0
:20EE800000F0184304903D46D3E7039A111D12680391002A01DB079204E0524243F002032E
:20EEA000079204933B782E2B0CD17B782A2B33D1039B1A1D1B680392002BB8BF4FF0FF33ED
:20EEC000023705932E4D397803222846F1F790F938B14023401B03FA00F0049B0343013780
:20EEE0000493397827488DF8281006227E1CF1F77FF9002838D0244B13BB039B073323F024
:20EF0000070308330393099B4B4409936DE705FB023201200F46A6E700230137059319466A
:20EF20000A25384610F8012B303A092A03D9002BC8D00591C6E705FB012101230746F0E707
:20EF400003AB00932246114B04A94046FEF756F8B0F1FF3F8146D6D1A3895B063FF535AF44
:20EF600009981DB0BDE8F08F03AB00932246074B04A94046FEF7F8FAEAE700BFE45001081D
:20EF8000EA500108EE500108FDCF0008EDEC000838B5064C0023054608462360F8F706FEC1
:20EFA000431C02D1236803B12B6038BD5425002082B001B901A942B14BB113780B601278C2
:20EFC000101C18BF012002B070471046FBE76FF00100F8E7884210B501EB020307D8421E6E
:20EFE00099420AD011F8014B02F8014FF8E78342F5D98118D21AD34200D110BD13F8014DBA
:20F0000001F8014DF7E770477047F8B5074614460E4621B91146BDE8F840FFF70DBE22B90B
:20F02000FFF7BCFD25462846F8BD00F021F8A0420FD221463846FFF7FFFD05460028F2D0BB
:20F0400031462246FFF7B6FA31463846FFF7A6FDE9E73546E7E749B1FF2A85BF8A2303600D
:20F060000A704FF0FF3098BF012070470846704751F8043C181F002BBCBF0B58C01870471C
:20F08000F8B500BFF8BC08BC9E467047F8B500BFF8BC08BC9E4670471B5B33336D00000029
:20F0A000000000001B5B33376D000000000000004000003F065B4F666D7D077F6F0000008F
:20F0C00000000000777C395E79717D763000003800373F7300506D313E3E00006E000000A0
:20F0E00000000800777C585E79717D741000003800545C7300506D311C1C00006E00003055
:20F10000244750474741000024475056544700002447504753560000244750524D43000071
:20F12000244750475341000024504D544B0000002538640025346400696D70004F564552D9
:20F140000000000020202020202020300000000025382E366600000025312E34660000005A
:20F1600025312E3366000000252032642E25303664000000252035642E2530336400000082
:20F180002520386400000000487A000025642E253032640025642E253033640025642E25AB
:20F1A00064000000252034640000000025642E25303664204D487A0025642E253033642076
:20F1C0006B487A0025302E3666204D487A00000025302E3666206B487A00000025302E3392
:20F1E0006620487A000000004761746520256473202F2025642E25640000000047617465FA
:20F2000020256473202F202564000000476174652025646D7300000025382E3766000000A8
:20F2200025382E35660000006D73000025382E346600000025382E33660000007573000097
:20F2400025382E326600000025382E316600000025322E336600000025342E33660000002B
:20F2600025302E366620730025302E3666206D730000000025302E33662075730000000099
:20F2800025302E3066206E73000000001B5B33316D2A2A2A2A2A20494E495420454550529B
:20F2A0004F4D202A2A2A2A2A0D0A00001B5B481B5B324A1B5B33306D1B5B34336D2A2A2AEB
:20F2C0002A2A2053544152542050524F4752414D55202A2A2A2A2A1B5B306D0D0A00000083
:20F2E00030393A34373A3436000000004665622032382032303230001B5B33326D466D6581
:20F300007465722054696E7946343031204156542D33323735200D0A1B5B33366D76312EA2
:20F32000312025732025730D0A0000001B5B33326D466D657465722054696E7946343031CB
:20F34000204156542D35373535200D0A1B5B33366D76312E312025732025730D0A0000008F
:20F360001B5B33316D48617264566563203D20253038780D0A0000001B5B33326D486172AD
:20F3800064566563204F4B0D0A0000001B5B33376D636E7452657365743D25642C20636EA2
:20F3A000745764743D25642C20497764673D25642C20426F643D25640D0A0000486172648A
:20F3C000776172653A2000001B5B33326D54696E7920380D0A0000001B5B33336D54696E55
:20F3E0007920340D0A0000001B5B33316D556E6B6F77730D0A0000001B5B33376D726573AD
:20F40000756C742072656164454570726F6D28293D25642C207273743D25642C2077647476
:20F420003D25640D0A0000001B5B33336D2A2A2A2A2A204E69652077796B7279746F2045EA
:20F440004570726F6D204453323433310D0A00004156542D3332373500000000415654003D
:20F46000436667204572726F72000000496E697420454570726F6D004156542D3537353568
:20F48000000000001B5B33316D486172644661756C7420253038780D0A000000302E305F81
:20F4A0005F5F5F5F000000005F5F5F5F5F302E3000000000302E30303030303000000000E9
:20F4C00057796761737A616E6965205A65720000312073656B2E00003130306D7300000086
:20F4E0003130302073656B2E0000000031302073656B2E00474154450000000020484F4CD4
:20F50000442000001B5B481B5B324A001B5B481B5B33326D466D657465722054696E794664
:20F52000343031204156542D33323735200D0A1B5B33366D76312E312025732025730D0A1D
:20F54000000000001B5B481B5B33326D466D657465722054696E7946343031204156542D6B
:20F5600035373535200D0A1B5B33366D76312E312025732025730D0A000000001B5B3335C7
:20F580006D417574686F723A205361530D0A652D6D61696C3A2073617340656C706F727467
:20F5A000616C2E706C0D0A0D0A0000001B5B33376D72656164436E744672657141282920F8
:20F5C0003D2025642E2530326420487A2028307825783A2530347829202020200D0A0000C2
:20F5E00072656164436E74422829203D2025642E2530326420487A0D0A0000001B5B3337BF
:20F600006D72656164436E7446726571412829203D2025642E256420487A20283078257870
:20F620003A2530347829202020200D0A0000000072656164436E74422829203D2025642E47
:20F64000256420487A0D0A001B5B33376D72656164436E7446726571412829203D202564F4
:20F6600020487A2028307825783A2530347829202020200D0A00000072656164436E74421D
:20F680002829203D20256420487A20202020200D0A0000004761746520256473202F202549
:20F6A000642E256420202020200D0A004761746520256473202F20256420202020200D0A2C
:20F6C00000000000476174652025646D7320202020200D0A00000000706572696F64203D89
:20F6E00020256620757320202020200D0A0000001B5B33336D6678203D20256620487A206F
:20F70000202020200D0A0000506572696F6458203D20256620757320202020200D0A0000D0
:20F720001B5B33366D7448203D20256620757320202020200D0A0000744C203D2025662012
:20F74000757320202020200D0A00000064757479203D20256620252520202020200D0A001B
:20F760001B5B33346D6D6E6F7A6E696B46203D2025642C20647A69656C6E696B46203D2084
:20F7800025642C206D6E6F7A6E696B54203D2025642C20506F6D6961722023256420202054
:20F7A00020200D0A000000001B5B33326D0000001B5B33356D636E74203D20256420696D1E
:20F7C000702C204C61746368203D20256420696D702C20636867496E203D2025642020207A
:20F7E00020200D0A000000001B5B33366D0000001B5B33316D00000054696D317070735F12
:20F80000434352315F3332203D2025642074203D2025662073656B0D0A257364656C74615D
:20F82000203D2025662070706D2C2573207070732E5F31707073203D202564202020202065
:20F840000D0A00001B5B33376D74696D31707073203D202573253034641B5B33376D2063A4
:20F8600066672E76636F203D20256420283078257829202020200D0A000000000D0A257343
:20F880005A61706973454570726F6D203D2025642C1B5B33376D20656E6B2E76616C203D6E
:20F8A0002025642C206366672E656B72616E203D2025642027257327202020200D0A000041
:20F8C0000D0A257347505320282564291B5B33366D205554433A2025733A25733A25730D9A
:20F8E0000A0000001B5B3542000000001B5B750028636E7429000000286D61746829000095
:20F9000074482000744C2000706572696F64200064757479202025252025302E32660000FD
:20F92000496E707574204100706572696F64000048696768000000004C6F77002520647503
:20F940007479000025342E3266000000462025642E25303364206B487A0000004C617463C1
:20F960006820256400000000496E707574204200496E7075742042200000000044656C74E9
:20F98000610000002D2D2D2D2D2D2D2D000000004F4B000044656C746120202025302E3403
:20F9A000662070706D0000004E6F207369676E616C000000522065206C202B005220652074
:20F9C0006C202D002564000073255800466D6574000000001B5B33316D2A2A2A2A204572A3
:20F9E000726F722043666720454570726F6D2049440D0A001B5B33336D2A2A2A2A20457290
:20FA0000726F722043666731204352430D0A00001B5B33316D2A2A2A2A204572726F7220EA
:20FA200043666732286261636B757029204352430D0A00001B5B33326D2A2A2A2A20434615
:20FA400047204F4B0D0A00001B5B33366D2E00001B5B33326D454E44205772204545707280
:20FA60006F6D20200D0A00001B5B33376D536B616E6F77616E696520312D576972653A0D9A
:20FA80000A0000001B5B33356D25303278201B5B33366D2530327825303278253032782584
:20FAA0003032782530327825303278201B5B33346D25303278201B5B33326D772025646D10
:20FAC000730D0A001B5B33346D5A6E616C657A696F6E6F201B5B33366D256420737A742E85
:20FAE0001B5B33346D2075727A61647A656E20312D5769726520772074796D2044533234E6
:20FB00003331201B5B33366D256420737A742E0D0A000000456E645F4366675F00000000E1
:20FB20001B5B33336D537461727420577220454570726F6D0000000000000000000000001D
:20FB40000102030406070809000000000102030400000000B71DC1046E3B8209D926430D57
:20FB6000DC7604136B6BC517B24D861A0550471EB8ED08260FF0C922D6D68A2F61CB4B2B4D
:20FB8000649B0C35D386CD310AA08E3CBDBD4F3870DB114CC7C6D0481EE09345A9FD5241FD
:20FBA000ACAD155F1BB0D45BC2969756758B5652C836196A7F2BD86EA60D9B6311105A678D
:20FBC00014401D79A35DDC7D7A7B9F70CD665E74E0B6239857ABE29C8E8DA19139906095FD
:20FBE0003CC0278B8BDDE68F52FBA582E5E66486585B2BBEEF46EABA3660A9B7817D68B3CD
:20FC0000842D2FAD3330EEA9EA16ADA45D0B6CA0906D32D42770F3D0FE56B0DD494B71D97C
:20FC20004C1B36C7FB06F7C32220B4CE953D75CA28803AF29F9DFBF646BBB8FBF1A679FF0C
:20FC4000F4F63EE143EBFFE59ACDBCE82DD07DEC77708634C06D4730194B043DAE56C5392C
:20FC6000AB0682271C1B4323C53D002E7220C12ACF9D8E1278804F16A1A60C1B16BBCD1F4C
:20FC800013EB8A01A4F64B057DD00808CACDC90C07AB9778B0B6567C69901571DE8DD475FC
:20FCA000DBDD936B6CC0526FB5E6116202FBD066BF469F5E085B5E5AD17D1D576660DC538C
:20FCC00063309B4DD42D5A490D0B1944BA16D84097C6A5AC20DB64A8F9FD27A54EE0E6A17C
:20FCE0004BB0A1BFFCAD60BB258B23B69296E2B22F2BAD8A98366C8E41102F83F60DEE87CC
:20FD0000F35DA9994440689D9D662B902A7BEA94E71DB4E0500075E4892636E93E3BF7ED7B
:20FD20003B6BB0F38C7671F7555032FAE24DF3FE5FF0BCC6E8ED7DC231CB3ECF86D6FFCB0B
:20FD40008386B8D5349B79D1EDBD3ADC5AA0FBD8EEE00C6959FDCD6D80DB8E6037C64F649B
:20FD60003296087A858BC97E5CAD8A73EBB04B77560D044FE110C54B383686468F2B47424B
:20FD80008A7B005C3D66C158E4408255535D43519E3B1D252926DC21F0009F2C471D5E28FB
:20FDA000424D1936F550D8322C769B3F9B6B5A3B26D6150391CBD40748ED970AFFF0560E8B
:20FDC000FAA011104DBDD014949B93192386521D0E562FF1B94BEEF5606DADF8D7706CFCFB
:20FDE000D2202BE2653DEAE6BC1BA9EB0B0668EFB6BB27D701A6E6D3D880A5DE6F9D64DACB
:20FE00006ACD23C4DDD0E2C004F6A1CDB3EB60C97E8D3EBDC990FFB910B6BCB4A7AB7DB07A
:20FE2000A2FB3AAE15E6FBAACCC0B8A77BDD79A3C660369B717DF79FA85BB4921F4675960A
:20FE40001A163288AD0BF38C742DB081C330718599908A5D2E8D4B59F7AB085440B6C9504A
:20FE600045E68E4EF2FB4F4A2BDD0C479CC0CD43217D827B9660437F4F460072F85BC1764A
:20FE8000FD0B86684A16476C93300461242DC565E94B9B115E565A1587701918306DD81CFA
:20FEA000353D9F0282205E065B061D0BEC1BDC0F51A69337E6BB52333F9D113E8880D03A8A
:20FEC0008DD097243ACD5620E3EB152D54F6D4297926A9C5CE3B68C1171D2BCCA000EAC87A
:20FEE000A550ADD6124D6CD2CB6B2FDF7C76EEDBC1CBA1E376D660E7AFF023EA18EDE2EECA
:20FF00001DBDA5F0AAA064F4738627F9C49BE6FD09FDB889BEE0798D67C63A80D0DBFB8479
:20FF2000D58BBC9A62967D9EBBB03E930CADFF97B110B0AF060D71ABDF2B32A66836F3A209
:20FF40006D66B4BCDA7B75B8035D36B5B440F7B100000000000000000000000000000000F5
:20FF6000000000000000000000000000000000000000000007000F800F800F800F800F80AF
:20FF80000700070000000000070007000700000000000E380E380E380E38063000000000F0
:20FFA0000000000000000000000000000000000000000C300C300C307FFE7FFE0C300C301B
:20FFC0000C300C307FFE7FFE0C300C300C3000000000024002400FF81FF81A401A401FF096
:20FFE0000FF8025802581FF81FF00240024000000000000000000E100E300E7000E001C021
:020000040801F1
:20000000038007000E700C700870000000000000000000000F001980198019800F000F08E4
:200020000F9819F818F018E019F00F9800000000000000000700070007000E000000000035
:20004000000000000000000000000000000000000000000000F001C0038007000E000E0049
:200060000E000E000700038001C000F000000000000000000F00038001C000E00070007016
:200080000070007000E001C003800F00000000000000000001801188099007E007E03FFC91
:2000A0003FFC07E007E00990118801800000000000000000000000000180018001800FF002
:2000C0000FF00180018001800000000000000000000000000000000000000000000000009E
:2000E0000000000000000700070007000E00000000000000000000000000000000001FF8C6
:200100001FF8000000000000000000000000000000000000000000000000000000000000C8
:20012000000000000000070007000700000000000000000000020006000E001C00380070D0
:2001400000E001C0038007000E001C0000000000000000000FF01C381C781CF81CF81DB866
:200160001DB81F381F381E381C380FF000000000000000000180018003801F801F8003800D
:20018000038003800380038003801FF000000000000000000FE01C701C380038007000E06A
:2001A00001C0038007000E381C381FF800000000000000000FE01C701C380038007003C009
:2001C00003C0007000381C381C700FE0000000000000000000E001E003E006E00CE018E077
:2001E0001FF81FF800E000E000E003F800000000000000001FF81C001C001C001C001FE0B0
:200200001FF0007800381C381C700FE0000000000000000003E007000E001C001C001FF011
:200220001FF81C381C381C381C380FF000000000000000001FFC1C1C1C1C1C1C001C003841
:20024000007000E001C003800380038000000000000000000FF01C381C381C381F3807E0CB
:2002600007E01CF81C381C381C380FF000000000000000000FF01C381C381C381C381FF822
:200280000FF800380038007000E007C0000000000000000000000000038003800380000047
:2002A00000000380038003800000000000000000000000000000000003800380038000002C
:2002C000000003800380038007000000000000000000007000E001C0038007000E001C00C9
:2002E0001C000E000700038001C000E000700000000000000000000000003FFC3FFC0000C3
:2003000000003FFC3FFC0000000000000000000000001C000E000700038001C000E00070A2
:20032000007000E001C0038007000E001C000000000003C00FF01E7818380038007000E0C8
:2003400001C001C00000000001C001C001C0000000000FF81C1C1C1C1C1C1C1C1CFC1CFCC1
:200360001CFC1CFC1C001C001C001FF007F800000000000003C007E00E701C381C381C38C7
:200380001C381FF81C381C381C381C3800000000000000001FF00E380E380E380E380FF07C
:2003A0000FF00E380E380E380E381FF0000000000000000007F00E381C381C001C001C0032
:2003C0001C001C001C001C380E3807F000000000000000001FE00E700E380E380E380E38A3
:2003E0000E380E380E380E380E701FE000000000000000001FF80E180E080E000E300FF0CA
:200400000FF00E300E000E080E181FF800000000000000001FF80E180E080E000E300FF0A0
:200420000FF00E300E000E000E001F00000000000000000007F00E381C381C381C001C0019
:200440001C001CF81C381C380E3807F800000000000000001C701C701C701C701C701FF0B4
:200460001FF01C701C701C701C701C7000000000000000000FE00380038003800380038033
:20048000038003800380038003800FE0000000000000000001FC00700070007000700070B1
:2004A000007038703870387038700FE000000000000000001E380E380E700EE00FC00F80D7
:2004C0000F800FC00EE00E700E381E3800000000000000001F000E000E000E000E000E0051
:2004E0000E000E000E080E180E381FF800000000000000001C1C1E3C1F7C1FFC1FFC1DDCEB
:200500001C9C1C1C1C1C1C1C1C1C1C1C00000000000000001C1C1C1C1E1C1F1C1F9C1DDC72
:200520001CFC1C7C1C3C1C1C1C1C1C1C000000000000000003E007F00E381C1C1C1C1C1C43
:200540001C1C1C1C1C1C0E3807F003E000000000000000001FF00E380E380E380E380FF0AD
:200560000FF00E000E000E000E001F00000000000000000003E00F780E381C1C1C1C1C1CCD
:200580001C1C1C7C1CFC0FF80FF8003800FC0000000000001FF00E380E380E380E380FF00B
:2005A0000FF00E700E380E380E381E3800000000000000000FF01C381C381C381C000FE090
:2005C00007F000381C381C381C380FF000000000000000001FFC19CC11C401C001C001C0D9
:2005E00001C001C001C001C001C007F000000000000000001C701C701C701C701C701C70F7
:200600001C701C701C701C701C700FE000000000000000001C701C701C701C701C701C70E7
:200620001C701C701C700EE007C0038000000000000000001C1C1C1C1C1C1C1C1C1C1C9C0E
:200640001C9C1C9C0FF80FF80770077000000000000000001C701C701C700EE007C0038052
:20066000038007C00EE01C701C701C7000000000000000001C701C701C701C701C700EE0F4
:2006800007C003800380038003800FE000000000000000001FF81C381838107000E001C0BC
:2006A000038007000E081C181C381FF8000000000000000007F007000700070007000700E1
:2006C0000700070007000700070007F00000000000000000100018001C000E000700038024
:2006E00001C000E000700038001C0007000000000000000007F00070007000700070007067
:200700000070007000700070007007F0000000000000018003C007E00E701C3800000000B5
:200720000000000000000000000000000000000000000000000000000000000000000000B9
:200740000000000000000000000000007FFF7FFF000000001C001C00070007000000000057
:20076000000000000000000000000000000000000000000000000000000000000FE000701A
:2007800000700FF01C701C701C700FD800000000000000001E000E000E000E000FF00E38D2
:2007A0000E380E380E380E380E381BF0000000000000000000000000000000000FE01C7055
:2007C0001C701C001C001C701C700FE0000000000000000000F80070007000700FF01C707B
:2007E0001C701C701C701C701C700FD8000000000000000000000000000000000FE01C70DB
:200800001C701FF01C001C701C700FE0000000000000000003E007700770070007001FE03C
:200820001FE007000700070007001FC0000000000000000000000000000000000FD81C704B
:200840001C701C701C700FF007F000701C700FE0000000001E000E000E000E000EF00F3886
:200860000F380E380E380E380E381E38000000000000000001C001C001C000000FC001C0F0
:2008800001C001C001C001C001C00FF80000000000000000007000700070000003F00070D9
:2008A000007000700070007000701C700CF007E0000000001E000E000E000E000E380E708D
:2008C0000EE00FC00EE00E700E381E3800000000000000000FC001C001C001C001C001C0BF
:2008E00001C001C001C001C001C00FF8000000000000000000000000000000001FF81C9C5D
:200900001C9C1C9C1C9C1C9C1C9C1C9C000000000000000000000000000000001FE01C70FC
:200920001C701C701C701C701C701C70000000000000000000000000000000000FE01C70F4
:200940001C701C701C701C701C700FE0000000000000000000000000000000001BF00E389B
:200960000E380E380E380E380FF00E000E001F000000000000000000000000001FB038E03E
:2009800038E038E038E038E01FE000E000E001F00000000000000000000000001EF00FF832
:2009A0000F380E000E000E000E001F00000000000000000000000000000000000FE01C305E
:2009C0001C300F8003E0187018700FE0000000000000000000000100030007001FF0070039
:2009E0000700070007000770077003E0000000000000000000000000000000001C701C70F9
:200A00001C701C701C701C701C700FD8000000000000000000000000000000001C701C701B
:200A20001C701C701C700EE007C00380000000000000000000000000000000001C1C1C1C6A
:200A40001C1C1C9C1C9C0FF807700770000000000000000000000000000000001CE01CE001
:200A60000FC0078007800FC01CE01CE0000000000000000000000000000000000E380E3846
:200A80000E380E380E3807F003E000E001C01F800000000000000000000000001FE018E073
:200AA00011C0038007000E201C601FE0000000000000000001F803800380038007001C008D
:200AC0001C00070003800380038001F800000000000001C001C001C001C001C001C001C02A
:200AE00001C001C001C001C001C001C001C00000000000001F8001C001C001C000E00038B5
:200B0000003800E001C001C001C01F8000000000000000001F1C3B9C39DC38F80000000084
:200B2000000000000000000000000000000000000000000000000000000000003FF03FF057
:200B4000F03CF03CF03CF03CF3FCF3FCF3FCF3FCF3FCF3FCF3F0F3F0F000F0003FF03FF047
:200B60000000000000000000000000000000000000000000000000001FF83FFC700EE007BE
:200B8000CC33CC33C003C003C003C003CC33CE73C7E3C3C3C003C003E007700E3FFC1FF89E
:200BA0000000000000000000000000000000000000000000000000001FF83FFC7FFEFFFF68
:200BC000F3CFF3CFFFFFFFFFFFFFFFFFF3CFF18FF81FFC3FFFFFFFFFFFFF7FFE3FFC1FF83C
:200BE0000000000000000000000000000000000000000000000000000000000000000000F5
:200C000038707CF8FFFCFFFCFFFCFFFCFFFCFFFC7FF87FF83FF01FE00FC007800300000061
:200C20000000000000000000000000000000000000000000000000000000000000000000B4
:200C4000030007800FC01FE03FF07FF8FFFCFFFC7FF83FF01FE00FC00780030000000000A2
:200C60000000000000000000000000000000000000000000000000000000000003C003C0EE
:200C80000FF00FF00FF00FF0FC3FFC3FFC3FFC3FFC3FFC3F03C003C003C003C00FF00FF0EC
:200CA00000000000000000000000000000000000000000000000000000000000018003C0F0
:200CC00007E00FF01FF83FFC7FFEFFFFFFFFFFFFFFFF7FFE3BDC03C003C003C00FF00FF08C
:200CE0000000000000000000000000000000000000000000000000000000000000000000F4
:200D0000000000000000000003C007E00FF00FF00FF00FF007E003C0000000000000000083
:200D200000000000000000000000000000000000FFFFFFFFFFFFFFFFFFFFFFFFFFFFFFFFC3
:200D4000FFFFFFFFFFFFFFFFFC3FF81FF00FF00FF00FF00FF81FFC3FFFFFFFFFFFFFFFFF03
:200D6000FFFFFFFFFFFFFFFFFFFFFFFFFFFFFFFF0000000000000000000000000000000083
:200D8000000000000FF01FF83C3C381C300C300C300C300C381C3C3C1FF80FF0000000009F
:200DA00000000000000000000000000000000000FFFFFFFFFFFFFFFFFFFFFFFFFFFFFFFF43
:200DC000FFFFFFFFF81FF00FE3C7C7E3CFF3CFF3CFF3CFF3C7E3E3C7F00FF81FFFFFFFFF3F
:200DE000FFFFFFFFFFFFFFFFFFFFFFFFFFFFFFFF000000000000000003FC03FC007C00FC8D
:200E000001FC03EC07CC0F8C3FC07FE0F9F0F0F0F0F0F0F0F0F0F0F0F0F0F9F07FE03FC0AA
:200E20000000000000000000000000000000000000000000000000000FF01FF83E7C3C3C6A
:200E40003C3C3C3C3C3C3C3C3C3C3E7C1FF80FF003C003C03FFC3FFC03C003C003C003C062
:200E60000000000000000000000000000000000000000000000000000FFF0FFF0F0F0F0F1A
:200E80000FFF0FFF0F000F000F000F000F000F000F000F003F003F00FF00FF00FC00FC004A
:200EA0000000000000000000000000000000000000000000000000003FFF3FFF3C0F3C0F20
:200EC0003FFF3FFF3C0F3C0F3C0F3C0F3C0F3C0F3C0F3C0F3C3F3C3FFC3FFC3FFC3CFC3C62
:200EE000F000F00000000000000000000000000000000000000000000000000003C003C08C
:200F000003C003C0F3CFFBDF1FF80FF0FC3FFC3F0FF01FF8FBDFF3CF03C003C003C003C065
:200F200000000000000000000000000000000000000000008000C000E000F000F800FC00AD
:200F4000FE00FF00FF80FFC0FFFCFFFCFFC0FF80FF00FE00FC00F800F000E000C000800021
:200F600000000000000000000000000000000000000000000004000C001C003C007C00FC91
:200F800001FC03FC07FC0FFCFFFCFFFC0FFC07FC03FC01FC00FC007C003C001C000C000467
:200FA000000000000000000000000000000000000000000000000000018003C007E00FF007
:200FC0001FF83FFC03C003C003C003C003C003C03FFC1FF80FF007E003C0018000000000B1
:200FE0000000000000000000000000000000000000000000000000003C3C3C3C3C3C3C3C11
:201000003C3C3C3C3C3C3C3C3C3C3C3C3C3C3C3C3C3C3C3C000000003C3C3C3C3C3C3C3C40
:201020000000000000000000000000000000000000000000000000003FFF7FFFFBCFF3CF68
:20104000F3CFF3CFF3CFFBCF7FCF3FCF03CF03CF03CF03CF03CF03CF03CF03CF03CF03CFF0
:2010600000000000000000000000000000000000000000003FF03FF0F03CF03C3C003C0042
:201080000FC00FC03CF03CF0F03CF03CF03CF03C3CF03CF00FC00FC000F000F0F03CF03C7C
:2010A0003FF03FF000000000000000000000000000000000000000000000000000000000D2
:2010C00000000000000000000000000000000000FFFCFFFCFFFCFFFCFFFCFFFCFFFCFFFC38
:2010E000000000000000000000000000000000000000000000000000018003C007E00FF0C6
:201100001FF83FFC03C003C003C003C003C003C03FFC1FF80FF007E003C001803FFC3FFCF9
:20112000000000000000000000000000000000000000000000000000018003C007E00FF085
:201140001FF83FFC03C003C003C003C003C003C003C003C003C003C003C003C003C003C093
:2011600000000000000000000000000000000000000000000000000003C003C003C003C063
:2011800003C003C003C003C003C003C003C003C003C003C03FFC1FF80FF007E003C0018035
:2011A00000000000000000000000000000000000000000000000000000000000000000002F
:2011C0000000000001C000E000700038FFFCFFFC0038007000E001C0000000000000000087
:2011E0000000000000000000000000000000000000000000000000000000000000000000EF
:20120000000000000E001C0038007000FFFCFFFC700038001C000E00000000000000000034
:201220000000000000000000000000000000000000000000000000000000000000000000AE
:201240000000000000000000F000F000F000F000F000F000FFFCFFFC0000000000000000F8
:2012600000000000000000000000000000000000000000000000000000000000000000006E
:20128000000000000840186038707878FFFCFFFC78783870186008400000000000000000A8
:2012A00000000000000000000000000000000000000000000000000000000000000000002E
:2012C00003000300078007800FC00FC01FE01FE03FF03FF07FF87FF8FFFCFFFC000000001C
:2012E0000000000000000000000000000000000000000000000000000000000000000000EE
:20130000FFFCFFFC7FF87FF83FF03FF01FE01FE00FC00FC0078007800300030000000000DB
:201320000000000000000000000000000000000000000000000000000000000000000000AD
:2013400000000000000000000000000000000000000000000000000000000000000000008D
:2013600000000000000000000000000000000000000000000000000003C007E00FF00FF0C5
:201380000FF00FF00FF00FF007E007E007E003C003C003C00000000003C003C003C003C047
:2013A00000000000000000000000000000000000000000003C3C3C3C3C3C3C3C3C3C1C3881
:2013C0000C30000000000000000000000000000000000000000000000000000000000000D1
:2013E000000000000000000000000000000000000000000000000000000000003CF03CF095
:201400003CF03CF0FFFCFFFC3CF03CF03CF03CF03CF03CF0FFFCFFFC3CF03CF03CF03CF0D0
:201420000000000000000000000000000000000007800780078007803FF07FF8F87CF03C4A
:20144000F01CF000F000F8007FF03FF8007C003C003C003C003CE03CF03CF87C7FF83FF034
:20146000078007800780078000000000000000000000000000000000000000007878FC78EC
:20148000CCF0CCF0FDE079E003C003C0078007800F000F001E781EFC3CCC3CCC78FC7878C8
:2014A0000000000000000000000000000000000000000000000000000FC01FE03CF03CF006
:2014C0003CF03CF01DE01FC03F1C7FBCFBF8F1F0F0F0F0E0F0E0F0E0F0F0F9F07FF83F3C63
:2014E00000000000000000000000000000000000000000000F000F000F001F003E003C0026
:201500000000000000000000000000000000000000000000000000000000000000000000CB
:20152000000000000000000000000000000000000000000000000000007000F001E003C0A7
:20154000078007800F000F000F000F000F000F000F000F000780078003C001E000F00070F3
:201560000000000000000000000000000000000000000000000000000E000F00078003C004
:2015800001E001E000F000F000F000F000F000F000F000F001E001E003C007800F000E00E0
:2015A00000000000000000000000000000000000000000000000000000000000000000002B
:2015C0000000000038703CF01FE00FC07FF8FFFC7FF80FC01FE03CF03870000000000000DE
:2015E0000000000000000000000000000000000000000000000000000000000000000000EB
:201600000000000007800780078007807FF87FF87FF807800780078007800000000000002D
:201620000000000000000000000000000000000000000000000000000000000000000000AA
:2016400000000000000000000000000000000000000000000000000003C003C003C007C07A
:201660000F800F0000000000000000000000000000000000000000000000000000000000CC
:20168000000000000000000000000000FFFCFFFCFFFC000000000000000000000000000059
:2016A00000000000000000000000000000000000000000000000000000000000000000002A
:2016C00000000000000000000000000000000000000000000000000003C003C003C003C0FE
:2016E000000000000000000000000000000000000000000000000000003C003C0078007882
:2017000000F000F001E001E003C003C0078007800F000F001E001E003C003C0078007800D1
:20172000F000F00000000000000000000000000000000000000000001FE03FF07CF8F87CB3
:20174000F03CF03CF03CF33CF7BCF7BCF7BCF7BCF33CF03CF03CF03CF87C7CF83FF01FE041
:2017600000000000000000000000000000000000000000000000000003C007C00FC01FC031
:201780003FC003C003C003C003C003C003C003C003C003C003C003C003C003C03FFC3FFCED
:2017A0000000000000000000000000000000000000000000000000003FF07FF8F87CF03CE3
:2017C000E03C003C007C00F801F003E007C00F801F003E007C00F800F03CF03CFFFCFFFCF4
:2017E0000000000000000000000000000000000000000000000000003FF07FF8F87CF03CA3
:20180000003C003C003C00780FF00FF00078003C003C003C003C003CF03CF87C7FF83FF0B4
:2018200000000000000000000000000000000000000000000000000000F001F003F007F0DD
:201840000FF01FF03EF07CF0F8F0F0F0FFFCFFFC00F000F000F000F000F000F003FC03FC84
:20186000000000000000000000000000000000000000000000000000FFFCFFFCF000F00092
:20188000F000F000F000F000FFF0FFF8007C003C003C003C003C003CF03CF87C7FF83FF0B4
:2018A0000000000000000000000000000000000000000000000000000FF01FF03E007C0060
:2018C000F800F000F000F000FFF0FFF8F87CF03CF03CF03CF03CF03CF03CF87C7FF83FF0C4
:2018E000000000000000000000000000000000000000000000000000FFFCFFFCF03CF03C9A
:20190000003C003C007C00F801F003E007C00F800F000F000F000F000F000F000F000F0039
:201920000000000000000000000000000000000000000000000000003FF07FF8F87CF03C61
:20194000F03CF03CF03C78783FF03FF07878F03CF03CF03CF03CF03CF03CF87C7FF83FF0A3
:201960000000000000000000000000000000000000000000000000003FF07FF8F87CF03C21
:20198000F03CF03CF03CF87C7FFC3FFC003C003C003C003C003C007C00F801F03FE03FC0EA
:2019A000000000000000000000000000000000000000000000000000000000000000000027
:2019C00003C003C003C003C000000000000000000000000003C003C003C003C000000000EF
:2019E0000000000000000000000000000000000000000000000000000000000000000000E7
:201A000003C003C003C003C00000000000000000000000000000000003C003C003C007C0AA
:201A20000F800F00000000000000000000000000000000000000000000000000003C007C50
:201A400000F801F003E007C00F801F003E003E001F000F8007C003E001F000F8007C003CD0
:201A6000000000000000000000000000000000000000000000000000000000000000000066
:201A8000000000000000FFFCFFFCFFFC000000000000FFFCFFFCFFFC000000000000000064
:201AA000000000000000000000000000000000000000000000000000000000003C003E00AC
:201AC0001F000F8007C003E001F000F8007C007C00F801F003E007C00F801F003E003C0012
:201AE0000000000000000000000000000000000000000000000000003FF07FF8F87CF03CA0
:201B0000F03CF03C003C007C00F801F003E003C003C003C00000000003C003C003C003C094
:201B2000000000000000000000000000000000000000000000000000000000003FF07FF8FF
:201B4000F87CF03CF03CF03CF1FCF3FCF3FCF3FCF3FCF3FCF3F0F1F0F000F8007FF03FF0AB
:201B6000000000000000000000000000000000000000000000000000030007800FC01FE00D
:201B80003FF07CF8F87CF03CF03CF03CFFFCFFFCF03CF03CF03CF03CF03CF03CF03CF03C54
:201BA000000000000000000000000000000000000000000000000000FFF0FFF83C7C3C3C0F
:201BC0003C3C3C3C3C3C3C783FF03FF03C783C3C3C3C3C3C3C3C3C3C3C3C3C7CFFF8FFF069
:201BE0000000000000000000000000000000000000000000000000001FF03FF87C7CF83C73
:201C0000F01CF000F000F000F000F000F000F000F000F000F000F01CF83C7C7C3FF81FF0DA
:201C2000000000000000000000000000000000000000000000000000FFC0FFE03CF03C7826
:201C40003C783C3C3C3C3C3C3C3C3C3C3C3C3C3C3C3C3C3C3C3C3C783C783CF0FFE0FFC0EE
:201C6000000000000000000000000000000000000000000000000000FFFCFFFC3C3C3C1C9E
:201C80003C0C3C003CC03CC03FC03FC03CC03CC03C003C003C003C0C3C1C3C3CFFFCFFFC10
:201CA000000000000000000000000000000000000000000000000000FFFCFFFC3C3C3C1C5E
:201CC0003C0C3C003CC03CC03FC03FC03CC03CC03C003C003C003C003C003C00FF00FF002C
:201CE0000000000000000000000000000000000000000000000000001FF03FF87C7CF83C72
:201D0000F01CF000F000F000F000F000F1FCF1FCF03CF03CF03CF03CF83C7C7C3FFC1FEC0B
:201D2000000000000000000000000000000000000000000000000000F03CF03CF03CF03CF3
:201D4000F03CF03CF03CF03CFFFCFFFCF03CF03CF03CF03CF03CF03CF03CF03CF03CF03C25
:201D60000000000000000000000000000000000000000000000000001FE01FE00780078057
:201D8000078007800780078007800780078007800780078007800780078007801FE01FE0E3
:201DA00000000000000000000000000000000000000000000000000003FC03FC00F000F045
:201DC00000F000F000F000F000F000F000F000F0F0F0F0F0F0F0F0F0F0F0F9F07FE03FC0DC
:201DE000000000000000000000000000000000000000000000000000FC3CFC3C3C3C3C3C83
:201E00003C3C3C7C3CF83DF03FE03FC03FC03FE03DF03CF83C7C3C3C3C3C3C3CFC3CFC3C04
:201E2000000000000000000000000000000000000000000000000000FF00FF003C003C002C
:201E40003C003C003C003C003C003C003C003C003C003C003C003C0C3C1C3C3CFFFCFFFCE0
:201E6000000000000000000000000000000000000000000000000000F03CF03CF87CF87C22
:201E8000FCFCFCFCFFFCFFFCFFFCFFFCF7BCF7BCF33CF33CF03CF03CF03CF03CF03CF03C9A
:201EA000000000000000000000000000000000000000000000000000F03CF83CF83CFC3C56
:201EC000FC3CFE3CFE3CFF3CFF3CF7BCF7BCF3FCF3FCF1FCF1FCF0FCF0FCF07CF07CF03CE6
:201EE0000000000000000000000000000000000000000000000000003FF07FF8F87CF03C9C
:201F0000F03CF03CF03CF03CF03CF03CF03CF03CF03CF03CF03CF03CF03CF87C7FF83FF06B
:201F2000000000000000000000000000000000000000000000000000FFF0FFF83C7C3C3C8B
:201F40003C3C3C3C3C3C3C7C3FF83FF03C003C003C003C003C003C003C003C00FF00FF001D
:201F60000000000000000000000000000000000000000000000000003FF07FF8F87CF03C1B
:201F8000F03CF03CF03CF03CF03CF03CF03CF03CF03CF03CF33CF3BCF3FCF9FC7FF83FF021
:201FA00000E000F0007C003C00000000000000000000000000000000FFF0FFF83C7C3C3C83
:201FC0003C3C3C3C3C3C3C7C3FF83FF03FE03DF03CF83C7C3C3C3C3C3C3C3C3CFC3CFC3CF3
:201FE0000000000000000000000000000000000000000000000000003FF07FF8F87CF03C9B
:020000040801F1
:20200000F03CF03CF00078003F000FC003F00078003C003CF03CF03CF03CF87C7FF83FF071
:20202000000000000000000000000000000000000000000000000000FFFCFFFCFFFCC78C5C
:20204000C78C07800780078007800780078007800780078007800780078007801FE01FE054
:20206000000000000000000000000000000000000000000000000000F03CF03CF03CF03CB0
:20208000F03CF03CF03CF03CF03CF03CF03CF03CF03CF03CF03CF03CF03CF87C7FF83FF0EA
:2020A000000000000000000000000000000000000000000000000000F03CF03CF03CF03C70
:2020C000F03CF03CF03CF03CF03CF03CF03CF03CF03CF87C7CF83FF01FE00FC00780030005
:2020E000000000000000000000000000000000000000000000000000F03CF03CF03CF03C30
:20210000F03CF03CF03CF03CF33CF33CF33CF7BCF7BCFFFCFFFCFFFC7CF87CF838703870F3
:20212000000000000000000000000000000000000000000000000000F03CF03C7878787867
:202140003CF03CF01FE01FE00FC00FC00FC00FC01FE01FE03CF03CF078787878F03CF03C5F
:202160000000000000000000000000000000000000000000000000003C3C3C3C3C3C3C3C7F
:202180003C3C3C3C3C3C3E7C1FF80FF007E003C003C003C003C003C003C003C00FF00FF0CD
:2021A000000000000000000000000000000000000000000000000000FFFCFFFCF03CE03CE1
:2021C000C03C007C00F801F003E007C00F801F003E007C00F800F00CF01CF03CFFFCFFFC6A
:2021E0000000000000000000000000000000000000000000000000000FF00FF00F000F00C3
:202200000F000F000F000F000F000F000F000F000F000F000F000F000F000F000FF00FF0EE
:20222000000000000000000000000000000000000000000000000000F000F00078007800CE
:202240003C003C001E001E000F000F000780078003C003C001E001E000F000F00078007886
:20226000003C003C00000000000000000000000000000000000000000FF00FF000F000F008
:2022800000F000F000F000F000F000F000F000F000F000F000F000F000F000F00FF00FF020
:2022A00000000000000000000000000000000000030007800FC01FE03CF07878F03CE01C82
:2022C0000000000000000000000000000000000000000000000000000000000000000000FE
:2022E0000000000000000000000000000000000000000000000000000000000000000000DE
:202300000000000000000000000000000000000000000000000000000000000000000000BD
:2023200000000000FFFFFFFF0000000000000000000000000F000F000F000F8007C003C05B
:2023400000000000000000000000000000000000000000000000000000000000000000007D
:2023600000000000000000000000000000000000000000000000000000000000000000005D
:20238000000000003FC03FE001F000F03FF07FF0F8F0F0F0F0F0F0F0F0F0F9F07FFC3F3C59
:2023A000000000000000000000000000000000000000000000000000FC00FC003C003C00AD
:2023C0003C003C003F803FE03FF03CF83C7C3C3C3C3C3C3C3C3C3C3C3C3C3C7C3FF83FF09E
:2023E0000000000000000000000000000000000000000000000000000000000000000000DD
:20240000000000003FF07FF8F87CF03CF000F000F000F000F000F000F03CF87C7FF83FF090
:2024200000000000000000000000000000000000000000000000000003F003F000F000F0D6
:2024400000F000F00FF01FF03CF078F0F0F0F0F0F0F0F0F0F0F0F0F0F0F079F03FFC1F3CDB
:2024600000000000000000000000000000000000000000000000000000000000000000005C
:20248000000000003FF07FF8F87CF03CF03CFFFCFFFCF000F000F000F03CF87C7FF83FF0BE
:2024A0000000000000000000000000000000000000000000000000000FC01FE03FF03CF0F3
:2024C0003C703C003C003C00FF00FF003C003C003C003C003C003C003C003C00FF00FF00C0
:2024E0000000000000000000000000000000000000000000000000000000000000000000DC
:20250000000000003F3C7FFCF9F0F0F0F0F0F0F0F0F0F0F0F0F0F0F0F0F0F8F07FF03FF056
:2025200000F000F0F0F0F9F07FE03FC0000000000000000000000000FC00FC003C003C0024
:202540003C003C003CF03FF83FFC3F3C3C3C3C3C3C3C3C3C3C3C3C3C3C3C3C3CFC3CFC3CBA
:2025600000000000000000000000000000000000000000000000000007800780078007803F
:20258000000000001F801F8007800780078007800780078007800780078007801FE01FE0B9
:2025A000000000000000000000000000000000000000000000000000003C003C003C003C2B
:2025C0000000000000FC00FC003C003C003C003C003C003C003C003C003C003C003C003C33
:2025E0003C3C3C3C3C3C3E7C1FF80FF0000000000000000000000000FC00FC003C003C0033
:202600003C003C003C3C3C7C3CF83DF03FE03FC03FC03FE03DF03CF83C7C3C3CFC3CFC3C74
:202620000000000000000000000000000000000000000000000000001F801F80078007804E
:20264000078007800780078007800780078007800780078007800780078007801FE01FE01A
:2026600000000000000000000000000000000000000000000000000000000000000000005A
:2026800000000000FCF0FFF8FFFCFFFCF33CF33CF33CF33CF33CF33CF33CF33CF03CF03C91
:2026A00000000000000000000000000000000000000000000000000000000000000000001A
:2026C00000000000F3F0FFF83E7C3C3C3C3C3C3C3C3C3C3C3C3C3C3C3C3C3C3C3C3C3C3C3E
:2026E0000000000000000000000000000000000000000000000000000000000000000000DA
:20270000000000003FF07FF8F87CF03CF03CF03CF03CF03CF03CF03CF03CF87C7FF83FF025
:20272000000000000000000000000000000000000000000000000000000000000000000099
:2027400000000000F3F0FFF83E7C3C3C3C3C3C3C3C3C3C3C3C3C3C3C3C3C3C7C3FF83FF007
:202760003C003C003C003C00FF00FF0000000000000000000000000000000000000000006B
:20278000000000003F3C7FFCF9F0F0F0F0F0F0F0F0F0F0F0F0F0F0F0F0F0F8F07FF03FF0D4
:2027A00000F000F000F000F003FC03FC00000000000000000000000000000000000000005B
:2027C00000000000F3F0FFF83F7C3E3C3C3C3C3C3C003C003C003C003C003C00FF00FF0094
:2027E0000000000000000000000000000000000000000000000000000000000000000000D9
:20280000000000003FF07FF8F07CF03C78003E001F8007E001F00078F03CF83C7FF83FF0CF
:202820000000000000000000000000000000000000000000000000000100030007000F007E
:202840000F000F00FFF0FFF00F000F000F000F000F000F000F000F000F1C0FBC07F803F01C
:20286000000000000000000000000000000000000000000000000000000000000000000058
:2028800000000000F0F0F0F0F0F0F0F0F0F0F0F0F0F0F0F0F0F0F0F0F0F0F9F07FFC3F3CB9
:2028A000000000000000000000000000000000000000000000000000000000000000000018
:2028C000000000003C3C3C3C3C3C3C3C3C3C3C3C3C3C3C3C3E7C1FF80FF007E003C001803D
:2028E0000000000000000000000000000000000000000000000000000000000000000000D8
:2029000000000000F03CF03CF03CF03CF33CF33CF33CF7BCF7BCFFFCFFFCFFFC7CF8387007
:20292000000000000000000000000000000000000000000000000000000000000000000097
:2029400000000000F03CF87C7CF83FF01FE00FC00FC00FC00FC01FE03FF07CF8F87CF03CB7
:20296000000000000000000000000000000000000000000000000000000000000000000057
:2029800000000000F03CF03CF03CF03CF03CF03CF03CF03CF03CF03CF03CF83C7FFC3FFC69
:2029A000003C007C00F801F0FFE0FFC00000000000000000000000000000000000000000D8
:2029C00000000000FFFCFFFCF0F8F1F003E007C00F801F003E007C00F83CF03CFFFCFFFCD0
:2029E00000000000000000000000000000000000000000000000000000FC01FC03E003C038
:202A000003C003C003C007803F003F00078003C003C003C003C003C003C003E001FC00FC73
:202A200000000000000000000000000000000000000000000000000003C003C003C003C08A
:202A400003C003C003C003C00000000003C003C003C003C003C003C003C003C003C003C0CC
:202A60000000000000000000000000000000000000000000000000003F003F8007C003C0CE
:202A800003C003C003C001E000FC00FC01E003C003C003C003C003C003C007C03F803F00DC
:202AA0000000000000000000000000000000000000000000000000003C1C7F3CFFFCF3F81D
:202AC000E0F000000000000000000000000000000000000000000000000000000000000026
:202AE0000000000000000000000000000000000000000000000000000000000000000000D6
:202B0000030007800FC01FE03FF07CF8F87CF03CF03CF03CF03CF03CFFFCFFFC0000000074
:202B20000000000000000000000000000000000000000000000000000FF00FF03C3C3C3CA7
:202B4000F00CF00CF000F000F000F000F000F000F00CF00C3C3C3C3C0FF00FF000F000F017
:202B6000003C003C3FF03FF000000000000000000000000000000000F0F0F0F000000000BF
:202B800000000000F0F0F0F0F0F0F0F0F0F0F0F0F0F0F0F0F0F0F0F0F0F0F0F03F3C3F3CBF
:202BA000000000000000000000000000000000000000000000F000F003C003C00F000F0091
:202BC000000000003FF03FF0F03CF03CFFFCFFFCF000F000F000F000F03CF03C3FF03FF0D3
:202BE0000000000000000000000000000000000000000000030003000FC00FC03CF03CF0D9
:202C0000000000003FC03FC000F000F03FF03FF0F0F0F0F0F0F0F0F0F0F0F0F03F3C3F3C42
:202C2000000000000000000000000000000000000000000000000000F0F0F0F000000000D4
:202C4000000000003FC03FC000F000F03FF03FF0F0F0F0F0F0F0F0F0F0F0F0F03F3C3F3C02
:202C600000000000000000000000000000000000000000003C003C000F000F0003C003C038
:202C8000000000003FC03FC000F000F03FF03FF0F0F0F0F0F0F0F0F0F0F0F0F03F3C3F3CC2
:202CA00000000000000000000000000000000000000000000FC00FC03CF03CF00FC00FC080
:202CC000000000003FC03FC000F000F03FF03FF0F0F0F0F0F0F0F0F0F0F0F0F03F3C3F3C82
:202CE0000000000000000000000000000000000000000000000000000000000000000000D4
:202D00000FF00FF03C3C3C3C3C003C003C003C003C3C3C3C0FF00FF000F000F0003C003C8F
:202D20000FF00FF000000000000000000000000000000000030003000FC00FC03CF03CF099
:202D4000000000003FF03FF0F03CF03CFFFCFFFCF000F000F000F000F03CF03C3FF03FF051
:202D6000000000000000000000000000000000000000000000000000F03CF03C00000000FB
:202D8000000000003FF03FF0F03CF03CFFFCFFFCF000F000F000F000F03CF03C3FF03FF011
:202DA00000000000000000000000000000000000000000003C003C000F000F0003C003C0F7
:202DC000000000003FF03FF0F03CF03CFFFCFFFCF000F000F000F000F03CF03C3FF03FF0D1
:202DE0000000000000000000000000000000000000000000000000003C3C3C3C00000000E3
:202E0000000000000FC00FC003C003C003C003C003C003C003C003C003C003C00FF00FF078
:202E2000000000000000000000000000000000000000000003C003C00FF00FF03C3C3C3C1E
:202E4000000000000FC00FC003C003C003C003C003C003C003C003C003C003C00FF00FF038
:202E600000000000000000000000000000000000000000003C003C000F000F0003C003C036
:202E8000000000000FC00FC003C003C003C003C003C003C003C003C003C003C00FF00FF0F8
:202EA0000000000000000000000000000000000000000000F03CF03C0000000003000300B4
:202EC0000FC00FC03CF03CF0F03CF03CF03CF03CFFFCFFFCF03CF03CF03CF03CF03CF03C4E
:202EE000000000000000000000000000000000000FC00FC03CF03CF00FC00FC0000000003E
:202F00000FC00FC03CF03CF0F03CF03CF03CF03CFFFCFFFCF03CF03CF03CF03CF03CF03C0D
:202F20000000000000000000000000000000000003C003C00F000F003C003C000000000075
:202F4000FFFCFFFC3C3C3C3C3C003C003FF03FF03C003C003C003C003C3C3C3CFFFCFFFCDF
:202F6000000000000000000000000000000000000000000000000000000000000000000051
:202F800000000000F0F0F0F03F3C3F3C0F3C0F3C3FFC3FFCF3C0F3C0F3C0F3C03CFC3CFC33
:202FA0000000000000000000000000000000000000000000000000000FFC0FFC3CF03CF0A3
:202FC000F0F0F0F0F0F0F0F0FFFCFFFCF0F0F0F0F0F0F0F0F0F0F0F0F0F0F0F0F0FCF0FCA3
:202FE0000000000000000000000000000000000000000000030003000FC00FC03CF03CF0D5
:20300000000000003FF03FF0F03CF03CF03CF03CF03CF03CF03CF03CF03CF03C3FF03FF03C
:20302000000000000000000000000000000000000000000000000000F03CF03C0000000038
:20304000000000003FF03FF0F03CF03CF03CF03CF03CF03CF03CF03CF03CF03C3FF03FF0FC
:2030600000000000000000000000000000000000000000003C003C000F000F0003C003C034
:20308000000000003FF03FF0F03CF03CF03CF03CF03CF03CF03CF03CF03CF03C3FF03FF0BC
:2030A00000000000000000000000000000000000000000000F000F003FC03FC0F0F0F0F034
:2030C00000000000F0F0F0F0F0F0F0F0F0F0F0F0F0F0F0F0F0F0F0F0F0F0F0F03F3C3F3C7A
:2030E00000000000000000000000000000000000000000003C003C000F000F0003C003C0B4
:2031000000000000F0F0F0F0F0F0F0F0F0F0F0F0F0F0F0F0F0F0F0F0F0F0F0F03F3C3F3C39
:20312000000000000000000000000000000000000000000000000000F03CF03C0000000037
:2031400000000000F03CF03CF03CF03CF03CF03CF03CF03CF03CF03CF03CF03C3FFC3FFCE9
:20316000003C003C00F000F03FC03FC00000000000000000F03CF03C000000003FF03FF043
:20318000F03CF03CF03CF03CF03CF03CF03CF03CF03CF03CF03CF03CF03CF03C3FF03FF069
:2031A0000000000000000000000000000000000000000000F03CF03C00000000F03CF03C5F
:2031C000F03CF03CF03CF03CF03CF03CF03CF03CF03CF03CF03CF03CF03CF03C3FF03FF029
:2031E000000000000000000000000000000000000000000003C003C003C003C00FF00FF0C5
:203200003C3C3C3C3C003C003C003C003C003C003C3C3C3C0FF00FF003C003C003C003C05C
:2032200000000000000000000000000000000000000000000FC00FC03CF03CF03C303C30C0
:203240003C003C00FF00FF003C003C003C003C003C003C003C003C00FC3CFC3CFFF0FFF0CA
:203260000000000000000000000000000000000000000000000000003C3C3C3C3C3C3C3C6E
:203280000FF00FF003C003C03FFC3FFC03C003C03FFC3FFC03C003C003C003C003C003C0A6
:2032A0000000000000000000000000000000000000000000FFC0FFC0F0F0F0F0F0F0F0F010
:2032C000FFC0FFC0F030F030F0F0F0F0F3FCF3FCF0F0F0F0F0F0F0F0F0F0F0F0F03CF03CFA
:2032E000000000000000000000000000000000000000000000FC00FC03CF03CF03C003C0AC
:2033000003C003C003C003C03FFC3FFC03C003C003C003C003C003C003C003C003C003C08D
:20332000F3C0F3C03F003F0000000000000000000000000003C003C00F000F003C003C008D
:20334000000000003FC03FC000F000F03FF03FF0F0F0F0F0F0F0F0F0F0F0F0F03F3C3F3CFB
:20336000000000000000000000000000000000000000000000F000F003C003C00F000F00C9
:20338000000000000FC00FC003C003C003C003C003C003C003C003C003C003C00FF00FF0F3
:2033A000000000000000000000000000000000000000000003C003C00F000F003C003C00F1
:2033C000000000003FF03FF0F03CF03CF03CF03CF03CF03CF03CF03CF03CF03C3FF03FF079
:2033E000000000000000000000000000000000000000000003C003C00F000F003C003C00B1
:2034000000000000F0F0F0F0F0F0F0F0F0F0F0F0F0F0F0F0F0F0F0F0F0F0F0F03F3C3F3C36
:203420000000000000000000000000000000000000000000000000003F3C3F3CF3F0F3F0D0
:2034400000000000F3F0F3F03C3C3C3C3C3C3C3C3C3C3C3C3C3C3C3C3C3C3C3C3C3C3C3C06
:20346000000000000000000000000000000000003F3C3F3CF3F0F3F000000000F03CF03C38
:20348000FC3CFC3CFF3CFF3CFFFCFFFCF3FCF3FCF0FCF0FCF03CF03CF03CF03CF03CF03C92
:2034A00000000000000000000000000000000000000000000FF00FF03CF03CF03CF03CF05E
:2034C0000FFC0FFC000000003FFC3FFC000000000000000000000000000000000000000060
:2034E00000000000000000000000000000000000000000000FC00FC03CF03CF03CF03CF07E
:203500000FC00FC0000000003FF03FF00000000000000000000000000000000000000000AF
:203520000000000000000000000000000000000000000000000000000F000F000F000F004F
:20354000000000000F000F000F001F003E007C00F800F000F03CF03CF03CF87C7FF83FF0DF
:2035600000000000000000000000000000000000000000000000000000000000000000004B
:203580000000000000000000FFFCFFFCF000F000F000F000F000F000F000F00000000000B5
:2035A00000000000000000000000000000000000000000000000000000000000000000000B
:2035C0000000000000000000FFFCFFFC003C003C003C003C003C003C003C003C0000000015
:2035E0000000000000000000000000000000000000000000F000F000F000F000F00CF00C13
:20360000F03CF03CF0F0F0F003C003C00F000F003C003C00F3F0F3F0C03CC03C00F000F0D8
:2036200003C003C00FFC0FFC000000000000000000000000F000F000F000F000F00CF00C36
:20364000F03CF03CF0F0F0F003C003C00F000F003C3C3C3CF0FCF0FCC3FCC3FC0FFC0FFC52
:20366000003C003C003C003C0000000000000000000000000000000003C003C003C003C04E
:203680000000000003C003C003C007E007E007E00FF00FF00FF00FF00FF00FF007E003C088
:2036A00000000000000000000000000000000000000000000000000000000000000000000A
:2036C000000000000E1C1E3C3C7878F0F1E0F1E078F03C781E3C0E1C000000000000000008
:2036E0000000000000000000000000000000000000000000000000000000000000000000CA
:2037000000000000E1C0F1E078F03C781E3C1E3C3C7878F0F1E0E1C00000000000000000D9
:203720000000000000000000000000000000000003030303303030300303030330303030F1
:20374000030303033030303003030303303030300303030330303030030303033030303039
:203760000303030330303030030303033030303033333333CCCCCCCC33333333CCCCCCCCB9
:2037800033333333CCCCCCCC33333333CCCCCCCC33333333CCCCCCCC33333333CCCCCCCC39
:2037A00033333333CCCCCCCC33333333CCCCCCCCF3F3F3F33F3F3F3FF3F3F3F33F3F3F3F81
:2037C000F3F3F3F33F3F3F3FF3F3F3F33F3F3F3FF3F3F3F33F3F3F3FF3F3F3F33F3F3F3FC9
:2037E000F3F3F3F33F3F3F3FF3F3F3F33F3F3F3F03C003C003C003C003C003C003C003C021
:2038000003C003C003C003C003C003C003C003C003C003C003C003C003C003C003C003C078
:2038200003C003C003C003C003C003C003C003C003C003C003C003C003C003C003C003C058
:2038400003C003C003C003C003C003C0FFC0FFC003C003C003C003C003C003C003C003C040
:2038600003C003C003C003C003C003C003C003C003C003C003C003C003C003C003C003C018
:2038800003C003C0FFC0FFC003C003C0FFC0FFC003C003C003C003C003C003C003C003C008
:2038A00003C003C003C003C003C003C003C003C00F3C0F3C0F3C0F3C0F3C0F3C0F3C0F3C98
:2038C0000F3C0F3C0F3C0F3C0F3C0F3CFF3CFF3C0F3C0F3C0F3C0F3C0F3C0F3C0F3C0F3C58
:2038E0000F3C0F3C0F3C0F3C0F3C0F3C0F3C0F3C0000000000000000000000000000000070
:20390000000000000000000000000000FFFCFFFC0F3C0F3C0F3C0F3C0F3C0F3C0F3C0F3C59
:203920000F3C0F3C0F3C0F3C0F3C0F3C0F3C0F3C000000000000000000000000000000002F
:2039400000000000FFC0FFC003C003C0FFC0FFC003C003C003C003C003C003C003C003C0CD
:2039600003C003C003C003C003C003C003C003C00F3C0F3C0F3C0F3C0F3C0F3C0F3C0F3CD7
:203980000F3C0F3CFF3CFF3C003C003CFF3CFF3C0F3C0F3C0F3C0F3C0F3C0F3C0F3C0F3CD5
:2039A0000F3C0F3C0F3C0F3C0F3C0F3C0F3C0F3C0F3C0F3C0F3C0F3C0F3C0F3C0F3C0F3C57
:2039C0000F3C0F3C0F3C0F3C0F3C0F3C0F3C0F3C0F3C0F3C0F3C0F3C0F3C0F3C0F3C0F3C37
:2039E0000F3C0F3C0F3C0F3C0F3C0F3C0F3C0F3C000000000000000000000000000000006F
:203A000000000000FFFCFFFC003C003CFF3CFF3C0F3C0F3C0F3C0F3C0F3C0F3C0F3C0F3C6A
:203A20000F3C0F3C0F3C0F3C0F3C0F3C0F3C0F3C0F3C0F3C0F3C0F3C0F3C0F3C0F3C0F3CD6
:203A40000F3C0F3CFF3CFF3C003C003CFFFCFFFC00000000000000000000000000000000EC
:203A6000000000000000000000000000000000000F3C0F3C0F3C0F3C0F3C0F3C0F3C0F3CEE
:203A80000F3C0F3C0F3C0F3C0F3C0F3CFFFCFFFC000000000000000000000000000000006E
:203AA0000000000000000000000000000000000003C003C003C003C003C003C003C003C0EE
:203AC00003C003C0FFC0FFC003C003C0FFC0FFC000000000000000000000000000000000DE
:203AE0000000000000000000000000000000000000000000000000000000000000000000C6
:203B0000000000000000000000000000FFC0FFC003C003C003C003C003C003C003C003C00F
:203B200003C003C003C003C003C003C003C003C003C003C003C003C003C003C003C003C055
:203B400003C003C003C003C003C003C003FF03FF00000000000000000000000000000000CF
:203B60000000000000000000000000000000000003C003C003C003C003C003C003C003C02D
:203B800003C003C003C003C003C003C0FFFFFFFF0000000000000000000000000000000097
:203BA000000000000000000000000000000000000000000000000000000000000000000005
:203BC000000000000000000000000000FFFFFFFF03C003C003C003C003C003C003C003C0D1
:203BE00003C003C003C003C003C003C003C003C003C003C003C003C003C003C003C003C095
:203C000003C003C003C003C003C003C003FF03FF03C003C003C003C003C003C003C003C0F6
:203C200003C003C003C003C003C003C003C003C0000000000000000000000000000000006C
:203C4000000000000000000000000000FFFFFFFF0000000000000000000000000000000068
:203C60000000000000000000000000000000000003C003C003C003C003C003C003C003C02C
:203C800003C003C003C003C003C003C0FFFFFFFF03C003C003C003C003C003C003C003C07E
:203CA00003C003C003C003C003C003C003C003C003C003C003C003C003C003C003C003C0D4
:203CC00003C003C003FF03FF03C003C003FF03FF03C003C003C003C003C003C003C003C0B8
:203CE00003C003C003C003C003C003C003C003C00F3C0F3C0F3C0F3C0F3C0F3C0F3C0F3C54
:203D00000F3C0F3C0F3C0F3C0F3C0F3C0F3F0F3F0F3C0F3C0F3C0F3C0F3C0F3C0F3C0F3CED
:203D20000F3C0F3C0F3C0F3C0F3C0F3C0F3C0F3C0F3C0F3C0F3C0F3C0F3C0F3C0F3C0F3CD3
:203D40000F3C0F3C0F3F0F3F0F000F000FFF0FFF00000000000000000000000000000000F7
:203D6000000000000000000000000000000000000000000000000000000000000000000043
:203D8000000000000FFF0FFF0F000F000F3F0F3F0F3C0F3C0F3C0F3C0F3C0F3C0F3C0F3CF5
:203DA0000F3C0F3C0F3C0F3C0F3C0F3C0F3C0F3C0F3C0F3C0F3C0F3C0F3C0F3C0F3C0F3C53
:203DC0000F3C0F3CFF3FFF3F00000000FFFFFFFF00000000000000000000000000000000D5
:203DE0000000000000000000000000000000000000000000000000000000000000000000C3
:203E000000000000FFFFFFFF00000000FF3FFF3F0F3C0F3C0F3C0F3C0F3C0F3C0F3C0F3CD2
:203E20000F3C0F3C0F3C0F3C0F3C0F3C0F3C0F3C0F3C0F3C0F3C0F3C0F3C0F3C0F3C0F3CD2
:203E40000F3C0F3C0F3F0F3F0F000F000F3F0F3F0F3C0F3C0F3C0F3C0F3C0F3C0F3C0F3C1E
:203E60000F3C0F3C0F3C0F3C0F3C0F3C0F3C0F3C00000000000000000000000000000000EA
:203E800000000000FFFFFFFF00000000FFFFFFFF000000000000000000000000000000002A
:203EA000000000000000000000000000000000000F3C0F3C0F3C0F3C0F3C0F3C0F3C0F3CAA
:203EC0000F3C0F3CFF3FFF3F00000000FF3FFF3F0F3C0F3C0F3C0F3C0F3C0F3C0F3C0F3CFC
:203EE0000F3C0F3C0F3C0F3C0F3C0F3C0F3C0F3C03C003C003C003C003C003C003C003C052
:203F000003C003C0FFFFFFFF00000000FFFFFFFF0000000000000000000000000000000023
:203F2000000000000000000000000000000000000F3C0F3C0F3C0F3C0F3C0F3C0F3C0F3C29
:203F40000F3C0F3C0F3C0F3C0F3C0F3CFFFFFFFF00000000000000000000000000000000A3
:203F6000000000000000000000000000000000000000000000000000000000000000000041
:203F800000000000FFFFFFFF00000000FFFFFFFF03C003C003C003C003C003C003C003C011
:203FA00003C003C003C003C003C003C003C003C000000000000000000000000000000000E9
:203FC000000000000000000000000000FFFFFFFF0F3C0F3C0F3C0F3C0F3C0F3C0F3C0F3C8D
:203FE0000F3C0F3C0F3C0F3C0F3C0F3C0F3C0F3C0F3C0F3C0F3C0F3C0F3C0F3C0F3C0F3C11
:020000040801F1
:204000000F3C0F3C0F3C0F3C0F3C0F3C0FFF0FFF00000000000000000000000000000000C2
:204020000000000000000000000000000000000003C003C003C003C003C003C003C003C068
:2040400003C003C003FF03FF03C003C003FF03FF000000000000000000000000000000004C
:20406000000000000000000000000000000000000000000000000000000000000000000040
:204080000000000003FF03FF03C003C003FF03FF03C003C003C003C003C003C003C003C07A
:2040A00003C003C003C003C003C003C003C003C000000000000000000000000000000000E8
:2040C0000000000000000000000000000FFF0FFF0F3C0F3C0F3C0F3C0F3C0F3C0F3C0F3C6C
:2040E0000F3C0F3C0F3C0F3C0F3C0F3C0F3C0F3C0F3C0F3C0F3C0F3C0F3C0F3C0F3C0F3C10
:204100000F3C0F3C0F3C0F3C0F3C0F3CFFFFFFFF0F3C0F3C0F3C0F3C0F3C0F3C0F3C0F3C89
:204120000F3C0F3C0F3C0F3C0F3C0F3C0F3C0F3C03C003C003C003C003C003C003C003C00F
:2041400003C003C0FFFFFFFF03C003C0FFFFFFFF03C003C003C003C003C003C003C003C043
:2041600003C003C003C003C003C003C003C003C003C003C003C003C003C003C003C003C00F
:2041800003C003C003C003C003C003C0FFC0FFC0000000000000000000000000000000000F
:2041A0000000000000000000000000000000000000000000000000000000000000000000FF
:2041C00000000000000000000000000003FF03FF03C003C003C003C003C003C003C003C0C3
:2041E00003C003C003C003C003C003C003C003C0FFFFFFFFFFFFFFFFFFFFFFFFFFFFFFFFB7
:20420000FFFFFFFFFFFFFFFFFFFFFFFFFFFFFFFFFFFFFFFFFFFFFFFFFFFFFFFFFFFFFFFFBE
:20422000FFFFFFFFFFFFFFFFFFFFFFFFFFFFFFFF000000000000000000000000000000008E
:20424000000000000000000000000000FFFFFFFFFFFFFFFFFFFFFFFFFFFFFFFFFFFFFFFF72
:20426000FFFFFFFFFFFFFFFFFFFFFFFFFFFFFFFFFF00FF00FF00FF00FF00FF00FF00FF0056
:20428000FF00FF00FF00FF00FF00FF00FF00FF00FF00FF00FF00FF00FF00FF00FF00FF002E
:2042A000FF00FF00FF00FF00FF00FF00FF00FF0000FF00FF00FF00FF00FF00FF00FF00FF0E
:2042C00000FF00FF00FF00FF00FF00FF00FF00FF00FF00FF00FF00FF00FF00FF00FF00FFEE
:2042E00000FF00FF00FF00FF00FF00FF00FF00FFFFFFFFFFFFFFFFFFFFFFFFFFFFFFFFFFD6
:20430000FFFFFFFFFFFFFFFFFFFFFFFF0000000000000000000000000000000000000000A9
:2043200000000000000000000000000000000000000000000000000000000000000000007D
:20434000000000003F3C3F3CF3F0F3F0F3C0F3C0F3C0F3C0F3C0F3C0F3F0F3F03F3C3F3CB3
:204360000000000000000000000000000000000000000000000000003FC07FE0F9F0F0F016
:20438000F0F0F0F0F0F0F1E0F3C0F3E0F1F0F0F8F07CF03CF03CF03CF03CF07CF0F8F0F00D
:2043A000000000000000000000000000000000000000000000000000FFFCFFFCF03CF03CAF
:2043C000F03CF03CF000F000F000F000F000F000F000F000F000F000F000F000F000F00065
:2043E0000000000000000000000000000000000000000000000000000000000000000000BD
:20440000FFFCFFFC3CF03CF03CF03CF03CF03CF03CF03CF03CF03CF03CF03CF03CF03CF03E
:2044200000000000000000000000000000000000000000000000000000000000FFFCFFFC86
:20444000F03CF83C7C003E001F000F8007C007C00F801F003E007C00F83CF03CFFFCFFFC48
:2044600000000000000000000000000000000000000000000000000000000000000000003C
:20448000000000003FFC3FFCF3C0F3C0F3C0F3C0F3C0F3C0F3C0F3C0F3C0F3C03F003F002A
:2044A0000000000000000000000000000000000000000000000000000000000000000000FC
:2044C0003C3C3C3C3C3C3C3C3C3C3C3C3C3C3C3C3C3C3C3C3FF03FF03C003C003C003C00DE
:2044E000F000F00000000000000000000000000000000000000000000000000000000000DC
:204500003F3C3F3CF3F0F3F003C003C003C003C003C003C003C003C003C003C003C003C0BB
:20452000000000000000000000000000000000000000000000000000000000003FFC3FFC05
:2045400003C003C00FF00FF03C3C3C3C3C3C3C3C3C3C3C3C0FF00FF003C003C03FFC3FFC0D
:20456000000000000000000000000000000000000000000000000000000000000FC00FC09D
:204580003CF03CF0F03CF03CF03CF03CFFFCFFFCF03CF03CF03CF03C3CF03CF00FC00FC077
:2045A0000000000000000000000000000000000000000000000000000FC00FC03CF03CF005
:2045C000F03CF03CF03CF03CF03CF03C3CF03CF03CF03CF03CF03CF03CF03CF0FCFCFCFC83
:2045E00000000000000000000000000000000000000000000000000003FC03FC0F000F009F
:2046000003C003C000F000F00FFC0FFC3C3C3C3C3C3C3C3C3C3C3C3C3C3C3C3C0FF00FF060
:2046200000000000000000000000000000000000000000000000000000000000000000007A
:20464000000000003FFC3FFCF3CFF3CFF3CFF3CFF3CFF3CF3FFC3FFC0000000000000000E2
:2046600000000000000000000000000000000000000000000000000000000000000F000F1C
:20468000003C003C3FFC3FFCF3CFF3CFF3CFF3CFFF0FFF0F3FFC3FFC3C003C00F000F0003A
:2046A00000000000000000000000000000000000000000000000000003F003F00F000F00F6
:2046C0003C003C003C003C003FF03FF03C003C003C003C003C003C000F000F0003F003F020
:2046E000000000000000000000000000000000000000000000000000000000003FF03FF05C
:20470000F03CF03CF03CF03CF03CF03CF03CF03CF03CF03CF03CF03CF03CF03CF03CF03CD9
:20472000000000000000000000000000000000000000000000000000000000000000000079
:20474000FFFCFFFC0000000000000000FFFCFFFC0000000000000000FFFCFFFC0000000077
:20476000000000000000000000000000000000000000000000000000000000000000000039
:2047800007800780078007807FF87FF87FF8078007800780078000000000FFFCFFFCFFFC8B
:2047A00000000000000000000000000000000000000000000000000000003E001F000F800D
:2047C00007C003E001F000F800F801F003E007C00F801F003E00000000007FF87FF87FF862
:2047E000000000000000000000000000000000000000000000000000000001F003E007C01E
:204800000F801F003E007C007C003E001F000F8007C003E001F0000000007FF87FF87FF8C8
:2048200000000000000000000000000000000000000000000000000000FC01FE03CF03CFD9
:2048400003CF03CF03C003C003C003C003C003C003C003C003C003C003C003C003C003C00A
:2048600003C003C003C003C003C003C003C003C003C003C003C003C003C003C003C003C008
:2048800003C003C003C003C003C003C003C003C0F3C0F3C0F3C0F3C0F3C0F3C07F803F0090
